:0200000490006A
:1000000000000000000000000000000000000000F0
:1000100000000000000000000000000000000000E0
:1000200000000000000000000000000000000000D0
:1000300000000000000000000000000000000000C0
:1004000060A300245D42009071480390494200902F
:10041000494200904942009049420090000000008B
:10042000000000000000000000000000994400905F
:100430004942009000000000354400900593009070
:100440004D4600904D4600904D4600904D46009020
:100450004D4600904D4600904D4600904D46009010
:100460004D4600904D4600904D4600904D46009000
:100470004D4600904D4600904D4600904D460090F0
:1006980081F0004102E000BF83F0004330B54FEA2B
:1006A80041044FEA430594EA050F08BF90EA020F98
:1006B8001FBF54EA000C55EA020C7FEA645C7FEA2B
:1006C800655C00F0E2804FEA5454D4EB5555B8BF4E
:1006D8006D420CDD2C4480EA020281EA030382EABF
:1006E800000083EA010180EA020281EA0303362D51
:1006F80088BF30BD11F0004F4FEA01314FF4801C24
:100708004CEA113102D0404261EB410113F0004F35
:100718004FEA03334CEA133302D0524263EB4303EC
:1007280094EA050F00F0A780A4F10104D5F1200E8A
:100738000DDB02FA0EFC22FA05F2801841F10001E5
:1007480003FA0EF2801843FA05F359410EE0A5F1B9
:1007580020050EF1200E012A03FA0EFC28BF4CF0EA
:10076800020C43FA05F3C01851EBE37101F00045A0
:1007780007D54FF0000EDCF1000C7EEB00006EEBAD
:100788000101B1F5801F1BD3B1F5001F0CD3490837
:100798005FEA30004FEA3C0C04F101044FEA44528E
:1007A80012F5800F80F09A80BCF1004F08BF5FEA15
:1007B800500C50F1000041EB045141EA050130BDF5
:1007C8005FEA4C0C404141EB0101013C28BFB1F507
:1007D800801FE9D291F0000F04BF01460020B1FA52
:1007E80081F308BF2033A3F10B03B3F120020CDA25
:1007F8000C3208DD02F1140CC2F10C0201FA0CF003
:1008080021FA02F10CE002F11402D8BFC2F1200C67
:1008180001FA02F120FA0CFCDCBF41EA0C0190401D
:10082800E41AA2BF01EB0451294330BD6FEA040466
:100838001F3C1CDA0C340EDC04F11404C4F1200251
:1008480020FA04F001FA02F340EA030021FA04F363
:1008580045EA030130BDC4F10C04C4F1200220FABA
:1008680002F001FA04F340EA0300294630BD21FAF8
:1008780004F0294630BD94F0000F83F4801306BFBE
:1008880081F480110134013D4EE77FEA645C18BFB2
:100898007FEA655C29D094EA050F08BF90EA020F49
:1008A80005D054EA000C04BF1946104630BD91EA41
:1008B800030F1EBF0021002030BD5FEA545C05D144
:1008C8004000494128BF41F0004130BD14F5800483
:1008D8003CBF01F5801130BD01F0004545F0FE41F7
:1008E80041F470014FF0000030BD7FEA645C1ABF2C
:1008F800194610467FEA655C1CBF0B46024650EA63
:10090800013406BF52EA033591EA030F41F400218E
:1009180030BD00BF90F0000F04BF0021704730B514
:100928004FF4806404F132044FF000054FF00001E9
:1009380050E700BF90F0000F04BF0021704730B5AA
:100948004FF4806404F1320410F0004548BF40427F
:100958004FF000013EE700BF42004FEAE2014FEAD4
:1009680031014FEA02701FBF12F07F4393F07F4FAF
:1009780081F06051704732F07F4208BF704793F0B2
:100988007F4F04BF41F40021704730B54FF46074C5
:1009980001F0004521F000411CE700BF50EA0102C8
:1009A80008BF704730B54FF000050AE050EA010271
:1009B80008BF704730B511F0004502D5404261EBE1
:1009C80041014FF4806404F132045FEA915C3FF422
:1009D800D8AE4FF003025FEADC0C18BF03325FEABF
:1009E800DC0C18BF033202EBDC02C2F1200300FA70
:1009F80003FC20FA02F001FA03FE40EA0E0021FA95
:100A080002F11444BDE600BF70B54FF0FF0C4CF482
:100A1800E06C1CEA11541DBF1CEA135594EA0C0F34
:100A280095EA0C0F00F0DEF82C4481EA030621EA6F
:100A38004C5123EA4C5350EA013518BF52EA0335AA
:100A480041F4801143F4801338D0A0FB02CE4FF05C
:100A58000005E1FB02E506F00042E0FB03E54FF08C
:100A68000006E1FB03569CF0000F18BF4EF0010E84
:100A7800A4F1FF04B6F5007F64F5407404D25FEA80
:100A88004E0E6D4146EB060642EAC62141EA555133
:100A98004FEAC52040EA5E504FEACE2EB4F1FD0C75
:100AA80088BFBCF5E06F1ED8BEF1004F08BF5FEAF3
:100AB800500E50F1000041EB045170BD06F00046A5
:100AC80046EA010140EA020081EA0301B4EB5C0452
:100AD800C2BFD4EB0C0541EA045170BD41F480114A
:100AE8004FF0000E013C00F3AB8014F1360FDEBF6F
:100AF800002001F0004170BDC4F10004203C35DA4B
:100B08000C341BDC04F11404C4F1200500FA05F3CD
:100B180020FA04F001FA05F240EA020001F000426E
:100B280021F0004110EBD37021FA04F642EB0601E4
:100B38005EEA430E08BF20EAD37070BDC4F10C040E
:100B4800C4F1200500FA04F320FA05F001FA04F2D2
:100B580040EA020001F0004110EBD37041F10001BE
:100B68005EEA430E08BF20EAD37070BDC4F12005C9
:100B780000FA05F24EEA020E20FA04F301FA05F231
:100B880043EA020321FA04F001F0004121FA04F2D9
:100B980020EA020000EBD3705EEA430E08BF20EAA9
:100BA800D37070BD94F0000F0FD101F000464000E3
:100BB80041EB010111F4801F08BF013CF7D041EA65
:100BC800060195F0000F18BF704703F00046520069
:100BD80043EB030313F4801F08BF013DF7D043EA3A
:100BE8000603704794EA0C0F0CEA135518BF95EAF0
:100BF8000C0F0CD050EA410618BF52EA4306D1D177
:100C080081EA030101F000414FF0000070BD50EA95
:100C1800410606BF1046194652EA430619D094EA1F
:100C28000C0F02D150EA013613D195EA0C0F05D109
:100C380052EA03361CBF104619460AD181EA03015D
:100C480001F0004141F0FE4141F470014FF0000015
:100C580070BD41F0FE4141F4780170BD70B54FF0B0
:100C6800FF0C4CF4E06C1CEA11541DBF1CEA135530
:100C780094EA0C0F95EA0C0F00F0A7F8A4EB050412
:100C880081EA030E52EA03354FEA013100F0888009
:100C98004FEA03334FF0805545EA131343EA1263D2
:100CA8004FEA022245EA111545EA10654FEA002687
:100CB8000EF000419D4208BF964244F1FD0404F540
:100CC800407402D25B084FEA3202B61A65EB03059C
:100CD8005B084FEA32024FF480104FF4002CB6EB59
:100CE800020E75EB030E22BFB61A754640EA0C00D9
:100CF8005B084FEA3202B6EB020E75EB030E22BF19
:100D0800B61A754640EA5C005B084FEA3202B6EB59
:100D1800020E75EB030E22BFB61A754640EA9C0018
:100D28005B084FEA3202B6EB020E75EB030E22BFE8
:100D3800B61A754640EADC0055EA060E18D04FEAA6
:100D4800051545EA16754FEA06164FEAC30343EA46
:100D580052734FEAC2025FEA1C1CC0D111F4801F13
:100D68000BD141EA00014FF000004FF0004CB6E70C
:100D780011F4801F04BF01430020B4F1FD0C88BFAB
:100D8800BCF5E06F3FF6AFAEB5EB030C04BFB6EBB6
:100D9800020C5FEA500C50F1000041EB045170BDA9
:100DA8000EF0004E4EEA113114EB5C04C2BFD4EBD6
:100DB8000C0541EA045170BD41F480114FF0000E5A
:100DC800013C90E645EA060E8DE60CEA135594EAD6
:100DD8000C0F08BF95EA0C0F3FF43BAF94EA0C0FD9
:100DE8000AD150EA01347FF434AF95EA0C0F7FF44E
:100DF80025AF104619462CE795EA0C0F06D152EAA2
:100E080003353FF4FDAE1046194622E750EA410685
:100E180018BF52EA43067FF4C5AE50EA41047FF496
:100E28000DAF52EA43057FF4EBAE12E74FF0FF3CFB
:100E380006E000BF4FF0010C02E000BF4FF0010CCC
:100E48004DF804CD4FEA410C7FEA6C5C4FEA430C45
:100E580018BF7FEA6C5C1BD001B050EA410C0CBF94
:100E680052EA430C91EA030F02BF90EA020F0020F6
:100E7800704710F1000F91EA030F58BF994208BF5D
:100E880090422CBFD8176FEAE37040F0010070471A
:100E98004FEA410C7FEA6C5C02D150EA013C07D171
:100EA8004FEA430C7FEA6C5CD6D152EA033CD3D0BC
:100EB8005DF8040B704700BF8446104662468C46B6
:100EC8001946634600E000BF01B5FFF7B7FF0028E9
:100ED80048BF10F1000F01BD4DF808EDFFF7F4FF12
:100EE8000CBF012000205DF808FB00BF4DF808ED9D
:100EF800FFF7EAFF34BF012000205DF808FB00BFC0
:100F08004DF808EDFFF7E0FF94BF012000205DF8E1
:100F180008FB00BF4DF808EDFFF7CEFF94BF012096
:100F280000205DF808FB00BF4DF808EDFFF7C4FF8F
:100F380034BF012000205DF808FB00BF4FEA4102E2
:100F480012F5001215D211D56FF47873B3EB625213
:100F580012D94FEAC12343F0004343EA505311F03A
:100F6800004F23FA02F018BF404270474FF00000CC
:100F7800704750EA013005D111F0004008BF6FF00A
:100F8800004070474FF00000704700BF4FEA410231
:100F9800B2F1E04324BFB3F5001CDCF1FE5C0DD9CF
:100FA80001F0004C4FEAC0024CEA5070B2F1004F19
:100FB80040EB830008BF20F00100704711F0804F1C
:100FC80021D113F13872BCBF01F00040704741F4E1
:100FD80080114FEA5252C2F11802C2F1200C10FAE5
:100FE8000CF320FA02F018BF40F001004FEAC123C9
:100FF8004FEAD32303FA0CFC40EA0C0023FA02F36D
:101008004FEA4303CCE77FEA625307D150EA013342
:101018001EBF4FF0FE4040F44000704701F0004012
:1010280040F0FE4040F40000704700BF80F00040F0
:1010380002E000BF81F0004142001FBF5FEA4103A8
:1010480092EA030F7FEA226C7FEA236C6AD04FEAA8
:101058001262D2EB1363C1BFD218414048404140ED
:10106800B8BF5B42192B88BF704710F0004F40F49F
:10107800000020F07F4018BF404211F0004F41F4BB
:10108800000121F07F4118BF494292EA030F3FD087
:10109800A2F1010241FA03FC10EB0C00C3F120039A
:1010A80001FA03F100F0004302D5494260EB400029
:1010B800B0F5000F13D3B0F1807F06D340084FEA94
:1010C800310102F10102FE2A51D2B1F1004F40EB89
:1010D800C25008BF20F0010040EA030070474900F1
:1010E80040EB0000013A28BFB0F5000FEDD2B0FA8E
:1010F80080FCACF1080CB2EB0C0200FA0CF0AABFB1
:1011080000EBC25052421843BCBFD040184370474E
:1011180092F0000F81F4000106BF80F40000013254
:10112800013BB5E74FEA41037FEA226C18BF7FEA2B
:10113800236C21D092EA030F04D092F0000F08BF6D
:101148000846704790EA010F1CBF0020704712F054
:101158007F4F04D1400028BF40F00040704712F193
:1011680000723CBF00F50000704700F0004343F0F8
:10117800FE4040F4000070477FEA226216BF08462E
:101188007FEA23630146420206BF5FEA412390EAF1
:10119800010F40F4800070474FF0000304E000BFE7
:1011A80010F0004348BF40425FEA000C08BF704798
:1011B80043F0964301464FF000001CE050EA01025C
:1011C80008BF70474FF000030AE000BF50EA010271
:1011D80008BF704711F0004302D5404261EB41015E
:1011E8005FEA010C02BF84460146002043F0B64383
:1011F80008BFA3F18053A3F50003BCFA8CF2083AA8
:10120800A3EBC25310DB01FA02FC634400FA02FCB0
:10121800C2F12002BCF1004F20FA02F243EB0200B7
:1012280008BF20F00100704702F1200201FA02FC19
:10123800C2F1200250EA4C0021FA02F243EB02000C
:1012480008BF20EADC7070474FF0FF0C1CEAD05250
:101258001EBF1CEAD15392EA0C0F93EA0C0F6FD011
:101268001A4480EA010C400218BF5FEA41211ED0EF
:101278004FF0006343EA501043EA5111A0FB0131DB
:101288000CF00040B1F5000F3EBF490041EAD371B0
:101298005B0040EA010062F17F02FD2A1DD8B3F12C
:1012A800004F40EBC25008BF20F00100704790F09B
:1012B800000F0CF0004C08BF49024CEA502040EAED
:1012C80051207F3AC2BFD2F1FF0340EAC2507047B3
:1012D80040F400004FF00003013A5DDC12F1190FF1
:1012E800DCBF00F000407047C2F10002410021FA63
:1012F80002F1C2F1200200FA02FC5FEA310040F17B
:10130800000053EA4C0308BF20EADC70704792F0F3
:10131800000F00F0004C02BF400010F4000F013A2B
:10132800F9D040EA0C0093F0000F01F0004C02BF26
:10133800490011F4000F013BF9D041EA0C018FE795
:101348000CEAD15392EA0C0F18BF93EA0C0F0AD09B
:1013580030F0004C18BF31F0004CD8D180EA0100C1
:1013680000F00040704790F0000F17BF90F0004F5A
:10137800084691F0000F91F0004F14D092EA0C0F3C
:1013880001D142020FD193EA0C0F03D14B0218BFCF
:10139800084608D180EA010000F0004040F0FE4015
:1013A80040F40000704740F0FE4040F440007047B1
:1013B8004FF0FF0C1CEAD0521EBF1CEAD15392EA30
:1013C8000C0F93EA0C0F69D0A2EB030280EA010C20
:1013D80049024FEA402037D04FF0805343EA1111B9
:1013E80043EA10130CF000408B4238BF5B0042F117
:1013F8007D024FF4000C8B4224BF5B1A40EA0C00BC
:10140800B3EB510F24BFA3EB510340EA5C00B3EBED
:10141800910F24BFA3EB910340EA9C00B3EBD10FDB
:1014280024BFA3EBD10340EADC001B0118BF5FEA2D
:101438001C1CE0D1FD2A3FF650AF8B4240EBC25056
:1014480008BF20F0010070470CF0004C4CEA502017
:101458007F32C2BFD2F1FF0340EAC250704740F466
:1014680000004FF00003013A37E792F0000F00F058
:10147800004C02BF400010F4000F013AF9D040EAD6
:101488000C0093F0000F01F0004C02BF490011F46A
:10149800000F013BF9D041EA0C0195E70CEAD15362
:1014A80092EA0C0F08D142027FF47DAF93EA0C0F49
:1014B8007FF470AF084676E793EA0C0F04D14B022D
:1014C8003FF44CAF08466EE730F0004C18BF31F0DF
:1014D800004CCAD130F000427FF45CAF31F00043D9
:1014E8007FF43CAF5FE700BF4FF0FF3C06E000BF72
:1014F8004FF0010C02E000BF4FF0010C4DF804CD95
:101508004FEA40024FEA41037FEA226C18BF7FEAA4
:10151800236C11D001B052EA530C18BF90EA010FA6
:1015280058BFB2EB030088BFC81738BF6FEAE17035
:1015380018BF40F0010070477FEA226C02D15FEAD1
:10154800402C05D17FEA236CE4D15FEA412CE1D03D
:101558005DF8040B704700BF844608466146FFE704
:101568000FB5FFF7C9FF002848BF10F1000F0FBDE6
:101578004DF808EDFFF7F4FF0CBF012000205DF8DF
:1015880008FB00BF4DF808EDFFF7EAFF34BF012064
:1015980000205DF808FB00BF4DF808EDFFF7E0FFFD
:1015A80094BF012000205DF808FB00BF4DF808ED4E
:1015B800FFF7D2FF94BF012000205DF808FB00BFB1
:1015C8004DF808EDFFF7C8FF34BF012000205DF893
:1015D80008FB00BF4FEA40024FEA41037FEA226C52
:1015E80002D15FEA402C08D17FEA236C02D15FEA7E
:1015F800412C02D14FF0000070474FF001007047B6
:101608004FEA4002B2F1FE4F0FD34FF09E03B3EB07
:1016180012620DD94FEA002343F0004310F0004F47
:1016280023FA02F018BF404270474FF0000070479D
:1016380012F1610F01D1420205D110F0004008BF3C
:101648006FF0004070474FF00000704742000ED224
:10165800B2F1FE4F0BD34FF09E03B3EB126209D4E5
:101668004FEA002343F0004323FA02F070474FF09B
:101678000000704712F1610F01D1420202D14FF010
:10168800FF3070474FF00000704700BF7BB972B958
:101698000029BEBF00204FF0004106E008BF002827
:1016A8001CBF6FF000414FF0FF3000F057B8ADF1AC
:1016B800080C6DE904CE002909DB002B1ADB00F0C9
:1016C80069F8DDF804E0DDE9022304B07047404220
:1016D80061EB4101002B1BDB00F05CF8DDF804E056
:1016E800DDE9022304B0404261EB4101524263EB61
:1016F80043037047524263EB430300F04BF8DDF8B5
:1017080004E0DDE9022304B0404261EB4101704787
:10171800524263EB430300F03DF8DDF804E0DDE9F5
:10172800022304B0524263EB4303704753B94AB9EA
:10173800002908BF00281CBF4FF0FF314FF0FF30D1
:1017480000F00CB8ADF1080C6DE904CE00F022F8F9
:10175800DDF804E0DDE9022304B07047704700BFFC
:1017680010F8012B11F8013B012A28BF9A42F7D043
:10177800D01A7047034611F8012B03F8012B002AF1
:10178800F9D17047034613F8012B002AFBD1181A28
:10179800013870472DE9F04786468C460846089E72
:1017A800154674461946002B40F0C2808542B2FAAD
:1017B80082F245D94AB1C2F1200300FA02FC2EFA9E
:1017C80003F3954043EA0C0C94404FEA154EA8B237
:1017D800BCFBFEF8230C0EFB18CC08FB00F943EA0F
:1017E8000C43994528D9EB1808F1FF3704D29945DD
:1017F80002D9A8F102072B44A3EB0903A4B2B3FB57
:10180800FEFC0EFB1C330CFB00F044EA0344A04230
:1018180014D92C190CF1FF3304D2A04202D9ACF12F
:1018280002032C44241A43EA07401EB1D440002383
:1018380034607360BDE8F0874746DDE76346F1E74B
:1018480092BB431B01214FEA154EAFB2B3FBFEFC1E
:10185800200C0EFB1C330CFB07F840EA03439845A9
:1018680062D9EB180CF1FF3004D2984502D9ACF1DB
:1018780002002B44A3EB0803A4B2B3FBFEFC0EFB4F
:101888001C330CFB07F744EA0344A7424ED92C1932
:101898000CF1FF3304D2A74202D9ACF102032C4465
:1018A800E41B43EA0040C0E7C2F1200320FA03F139
:1018B800954090402EFA03F303434FEA154EAFB21A
:1018C800B1FBFEFC0EFB1C10190C0CFB07F841EADF
:1018D8000041884504FA02F422D969180CF1FF3056
:1018E80004D2884502D9ACF102002944A1EB0801D1
:1018F8009BB2B1FBFEFC0EFB1C110CFB07F743EA85
:1019080001439F420ED9EB180CF1FF3104D29F42DC
:1019180002D9ACF102012B44DB1B41EA004192E7FA
:101928006046E3E76146F7E76046A3E76346B7E743
:10193800834206D916B9002108467BE7C6E900E0CC
:10194800F9E7B3FA83F78FB9834201D3724508D810
:10195800BEEB020460EB030301209C461EB9002184
:1019680068E73846FAE7C6E9004CF8E7C7F1200C03
:10197800BB4022FA0CF41C432EFA0CF120FA0CF3AB
:10198800B84001434FEA14490EFA07F5B3FBF9F8DA
:101998001FFA84FE09FB18300B0C08FB0EFA43EA09
:1019A80000439A4502FA07F240D9E31808F1FF30DC
:1019B80004D29A4502D9A8F102002344A3EB0A03F2
:1019C80089B2B3FBF9F809FB183308FB0EFE41EAAC
:1019D80003418E452CD9611808F1FF3304D28E4596
:1019E80002D9A8F10203214443EA0040A0FB02986F
:1019F800A1EB0E014145CE46434602D306D14D45E3
:101A080004D2B9EB020E68EB04030138002EA6D00D
:101A1800B5EB0E0261EB030101FA0CFC22FA07F3A5
:101A28004CEA0303F940C6E9003198E74046C5E7A8
:101A38004346D9E7000000002DE9F04390F8A530AF
:101A480085B004460D4623B94FF07E50FFF7F2FAF1
:101A58000546D4F884202E4B9A4212D12846FEF728
:101A68007BFF29A3D3E90023FFF75EFA011E04F1E7
:101A7800840018BF01210CF0E5FF0120C4F898503C
:101A880005E0B4F89C30B3F5807F03D1002005B0A1
:101A9800BDE8F08304F15009484625F071FB0028A1
:101AA800F4D01C492846FFF7CFFB94F89C60FFF759
:101AB800CDFD94F88080C3B2276E206DB8F1000F79
:101AC8000DD08DF80D30022301220021009303ABC5
:101AD8008DF80C60B847484640F081FCCDE78DF89A
:101AE8000B60012641468DF80C3032460DF10B0390
:101AF8000096B847009603AB276E42463146206DE4
:101B0800E8E700BFAFF30080AE47E17A14AEEF3FDD
:101B18007418059000007F432DE9F04F044685B006
:101B2800084615466160062198469DF838709DF86C
:101B38003CA018F00BFFA060067C16F0010602D04E
:101B48007F4810F05BFC9DF8403008FB05F02773D8
:101B580084F82A307D309DF8443084F828307E237C
:101B680090FBF3F0C0010430C4E9045860623AF015
:101B7800ACF806227349A661C4E90706204645F079
:101B8800F7FC022202A92046ADF8085045F0F0FC07
:101B9800022202A92046ADF8088045F0E9FCF623A8
:101BA800032269462046ADF800308DF8026045F002
:101BB800DFFC7B1EDBB2082B05D840F25515DD4053
:101BC80015F0010501D16048BBE7052F09D0072FA3
:101BD80006D0032F7AD1012384F82930002502E0AA
:101BE8002E4684F829604FF000080026574F4FEA28
:101BF8006810C0EB0020FEF79DFE0022544BFEF754
:101C08004DFD32463B46FFF729F8FFF797F95FFA93
:101C180080FBC8F38200C0EB0020FEF78BFE002299
:101C28004C4BFEF73BFD00224B4BFFF717F8FFF735
:101C380085F95FFA80F908F00300C0EB0020FEF791
:101C480079FE0022424BFEF729FD32463B46FFF75C
:101C580005F8FFF773F9C0B2002D61D08DF80800C0
:101C68008DF809B08DF80A9008F10108032202A93D
:101C7800204645F07DFCB8F1800FB8D1BAF1000FCD
:101C88001BD0364D01A920462A88AB78ADF8042030
:101C980003228DF8063045F06BFC0B2230492046B4
:101CA80045F066FCD5F80300EB790522029002A9FD
:101CB80020468DF80C3045F05BFC204645F046FC8C
:101CC800A06945F067FC05B0BDE8F08F092F84F8DE
:101CD800296083D135460FF25809D9E9008916A73A
:101CE800D7E900672846FF35FEF724FE42464B46F3
:101CF800FEF7D4FC32463B46FEF7B0FFFFF71EF96D
:101D08000322C0B202A98DF808008DF809008DF8E9
:101D18000A00204645F02CFCB5F5FF4FE2D1ADE7AF
:101D28008DF808B08DF809908DF80A009CE700BF7F
:101D38000000000000C04F400000000000C05F40ED
:101D480010A805907DBC05906FA205900000084082
:101D58000000F83F00000C4000001C40239904904C
:101D680084BC05900000000030F000422DE9F84FD7
:101D78000146034604D1BDE8F84F012031F038B8D8
:101D8800002803DABDE8F84F31F03AB8B0F1FF4F58
:101D980003DBFFF751F9BDE8F88FB0F5000F35DA2E
:101DA8004FF09841FFF750FA6FF018020346C3F35B
:101DB8001604DE15764B234403F400007F3E80F0C2
:101DC8007E5016444FF07E51204306EBD356FFF762
:101DD80031F9704B04F10F0213400546002B3ED138
:101DE8000021FFF7C5FB98B1002E00F0C8803046EF
:101DF800FFF7D6F968490546FFF726FA674904460A
:101E08002846FFF721FA01462046C2E70022CEE71E
:101E18005DA1D1E90001FFF7B9F82946FFF714FAE7
:101E280001464FF07C50FFF705F92946044628463D
:101E3800FFF70AFA01462046FFF706FA04460EB9EC
:101E480021466FE03046FFF7ABF953490746FFF7E5
:101E5800FBF9524906463846FFF7F6F972E04FF0AB
:101E68008041FFF7E9F801462846FFF7A1FA8146C5
:101E78003046FFF795F9494680464846FFF7E4F9AA
:101E880001468246FFF7E0F94549DFF818B10746F1
:101E9800FFF7DAF94449FFF7CFF83946FFF7D4F9E5
:101EA8004249FFF7C9F83946FFF7CEF94049FFF72D
:101EB800C3F85146FFF7C8F93E4982463846FFF74E
:101EC800C3F93D49FFF7B8F83946FFF7BDF93B4973
:101ED800FFF7B2F83946FFF7B7F901465046FFF762
:101EE800ABF8C4F55713A34403F5227343EA0B0375
:101EF800002B074630DD4FF07C512846FFF7A4F948
:101F08002946FFF7A1F9014604463846FFF794F839
:101F18004946FFF799F9074646B901462046FFF7B3
:101F280089F801462846FFF785F834E71A494046FC
:101F3800FFF78AF9194906464046FFF785F93946F9
:101F4800FFF77AF801462046FFF774F82946FFF7AD
:101F580071F801463046E6E701462846FFF76AF879
:101F68004946FFF771F90446002E3FF469AF0A4964
:101F78004046FFF769F90949064640466CE70020E4
:101F880009E700BFAFF30080555555555555D53F66
:101F980020FB4A00F0FF7F008071313FD1F71737EF
:101FA8009788173E305CCFFF25333A3E2549923E4D
:101FB800ABAA2A3F4FD01C3E298E633ECDCCCC3EE7
:101FC8002DE9F04F31F0004387B080460F46814637
:101FD8000C460ED180F480094FEA490919F5000F23
:101FE80040F2618239464046FFF726F807B0BDE85F
:101FF800F08F20F00046B6F1FF4F02D8B3F1FF4F43
:1020080008D9B9F17E5FEDD184F48004640014F539
:10201800000FE5E7002832463DDAB3F1974F1BD3AE
:10202800B3F1FF4F3AD00225B4F17C5F4DD1B9F13D
:10203800000F80F29780B6F1FF4F28F0004040F083
:102048004982A6F17E562E4340F0A080404607B054
:10205800BDE8F04F30F0D4BEB3F17E5F2ED3D91572
:10206800C1F1960143FA01F505FA01F18B423BD122
:10207800B3F17E5F4AD1002C80F293800021404664
:10208800FFF776FA00284FD04FEAD97007B0BDE8BD
:10209800F04F30F0ADBEB3F1FF4F3CD1B6F17E5FEB
:1020A80000F0018204D9002CC0F2008238469DE776
:1020B800002C80F2FB8107F1004097E7B1F1804FD7
:1020C80038D0B1F17C5F53D0002529F04041B1F1FF
:1020D8007E5F28F000403BD1002C32DA01464FF0F9
:1020E8007E50FFF765F92CE0B3F17E5FC3D0002581
:1020F800B4F1804FE9D1B6F1BF4F1DD2B6F1D05F30
:1021080024D941464046FFF79FF86FE705F00105DF
:10211800C5F10205ECE7B3F17E5FACD0B1F1804FB9
:102128004FF00005E7D07FE741464FF07E50FFF7BC
:102138003FF95BE70025DEE7B6F1FF4F28F00040E6
:1021480031D1B9F1000FBFF651AF7AE728F000405E
:102158004EBB002C22DAB9F1000F1DDA6B1E584273
:10216800584193E7404607B0BDE8F04F47F079B8CB
:10217800B6F1FF4F20F000403FF438AFB6F17E5F74
:102188003FF464AF002E3FF431AF5FE7012D7FF4D9
:102198002DAF00F1004029E7304677E7012D7FF4A5
:1021A80025AF404622E74FEAD97101390291294308
:1021B8003FF44CAFB3F19A4F40F29981604B9E4285
:1021C80007D8002C0ADA002007B0BDE8F04F30F03D
:1021D80007BE5C4B9E4207D9002CF4DC002007B0F8
:1021E800BDE8F04F47F09CB84FF07E51FEF722FF54
:1021F80055490646FFF728F8544980463046FFF708
:1022080023F881464CA1D1E90001FEF7BFFE4FF04B
:102218007A5182463046FFF717F801465046FEF7D6
:1022280009FF3146FFF710F801464FF07C50FEF7E2
:1022380001FF314682463046FFF706F80146504610
:10224800FFF702F84249FEF7FFFF01464846FEF74E
:10225800F1FE014606464046FEF7EEFE20F47F6B8F
:102268002BF00F0B41465846FEF7E4FE0146304678
:10227800FEF7E0FE24F47F64029B013D24F00F0486
:102288001D430646214638460CBF324D4FF07E5559
:10229800FEF7D0FE5946FEF7D7FF3946804630464E
:1022A800FEF7D2FF01464046FEF7C6FE2146064627
:1022B8005846FEF7C9FF014607463046FEF7BCFE02
:1022C80000280446804620F0004320DDB3F1864F05
:1022D8000BD900212846FFF755F9003818BF01200F
:1022E80072E700210EE1012221E139D11A49304675
:1022F800FEF7A2FE394681462046FEF79BFE0146C0
:102308004846FFF75DF90028E3D186232DE0134AFC
:10231800934207D900212846FFF734F9003818BF3F
:1023280001205CE71CD13946FEF784FE3146FFF7F1
:102338003DF90028E9D0EDE7E13D55555555D53F24
:10234800F3FF7F3F0700803F00AAB83F70A5EC3637
:102358003BAAB83F000080BF3CAA383300001643B0
:10236800B3F17C5F40F29B80DB157E3B4FF40004A9
:102378001C414444C4F3C7534D497F3B1941214094
:10238800C4F31604C3F1170344F400041C41B8F164
:10239800000F3846B8BF6442FEF74CFE0746314688
:1023A8003846FEF749FE20F47F6828F00F084149B7
:1023B8004046FEF749FF394681464046FEF73AFE59
:1023C80001463046FEF736FE3B49FEF73DFF3B49E6
:1023D80006464046FEF738FF01463046FEF72CFE1B
:1023E800074601464846FEF727FE49460646FEF7D9
:1023F80021FE01463846FEF71DFE3146804630462E
:10240800FEF722FF2E490746FEF71EFF2D49FEF76D
:1024180011FE3946FEF718FF2B49FEF70DFE394627
:10242800FEF712FF2949FEF705FE3946FEF70CFFB5
:102438002749FEF701FE3946FEF706FF01463046FA
:10244800FEF7F8FD074601463046FEF7FDFE4FF061
:10245800804181463846FEF7EDFD01464846FEF7C5
:10246800A7FF414607463046FEF7EEFE4146FEF717
:10247800E3FD01463846FEF7DDFD3146FEF7DAFD9D
:1024880001464FF07E50FEF7D5FD00EBC453B3F57F
:10249800000F06DA214630F045FC294633E60024D1
:1024A8007DE71846F9E74FF07E509FE500209DE54F
:1024B800000080FF0072313F1872313F8CBEBF357B
:1024C8004CBB31330EEADD3555B38A38610B363BE8
:1024D800ABAA2A3EB6F17E5F3FF4B3AD002E3FF4BF
:1024E8005DAE002D3FF4B2AD00230225029319F032
:1024F800FF4F7FF4F6AE4FF09741FEF7A5FE6FF061
:1025080017010246D3157F3B0B440393804BC2F35C
:1025180016029A4242F07E5608DD7E4B9A427FF7B9
:10252800E2AE039B01330393A6F5000600227A4B23
:10253800049253F822B030465946FEF77BFD3146E7
:1025480081465846FEF778FD01464FF07E50FEF76B
:102558002FFF014605904846FEF776FE6F49019029
:10256800019B049AB24601EA660646F0005623F437
:102578007F6806F5800606EB425628F00F084146AC
:102588003046FEF761FE01464846FEF753FD5946C0
:1025980081463046FEF74EFD01465046FEF74AFD9D
:1025A8004146FEF751FE01464846FEF743FD059BAE
:1025B8001946FEF749FE019983460846FEF744FE90
:1025C80057490646FEF740FE5649FEF735FD3146A7
:1025D800FEF73AFE5449FEF72FFD3146FEF734FE6A
:1025E8005249FEF729FD3146FEF72EFE5049FEF707
:1025F80023FD3146FEF728FE4E49FEF71DFD314604
:1026080081463046FEF720FE01464846FEF71CFE8E
:10261800414606460198FEF70FFD5946FEF714FE9F
:102628003146FEF709FD414681464046FEF70CFE5D
:1026380041498246FEF700FD4946FEF7FDFC20F4BD
:102648007F6626F00F0641463046FEF7FDFD3A4903
:1026580080463046FEF7EEFC5146FEF7EBFC01469D
:102668004846FEF7E7FC0199FEF7EEFD3146814644
:102678005846FEF7E9FD01464846FEF7DDFC82466E
:1026880001464046FEF7D8FC20F47F6626F00F0688
:102698002A493046FEF7D8FD414681463046FEF7C6
:1026A800C9FC01465046FEF7C5FC2549FEF7CCFD9E
:1026B800244980463046FEF7C7FD01464046FEF7EE
:1026C800BBFC049A204B019253F82210FEF7B4FC8D
:1026D80006460398FEF764FD1C4B019A53F822A0A6
:1026E800804631464846FEF7A7FC5146FEF7A4FC53
:1026F8004146FEF7A1FC20F47F6B2BF00F0B4146FF
:102708005846FEF797FC5146FEF794FC4946ABE560
:1027180071C41C00D6B35D009041059000F0FFDF46
:1027280042F1533E55326C3E05A38B3EABAAAA3EFE
:10273800B76DDB3E9A99193F000040400040763F54
:102748004F38763FC623F6B88041059088410590FA
:102758002DE9F04F91B0840705460E46009302F02C
:102768000403DDF868800293C2F3C203039203F105
:102778000103059340F0BA81041D30B1072909D837
:102788006FF01B0011B0BDE8F08F01F0070634446C
:10279800C6F10806009B4FF000094FF0040A591EC5
:1027A8004FF0FF334F46CB4601935346CDF8109078
:1027B8000DB1009A22600598002800F3E880984837
:1027C800009A824203D397488242C0F0E080039A7D
:1027D800A4EB050E92074FEA9E0000F103810F2F2C
:1027E80000F2B180002D00F0058107F140020DEBE9
:1027F800020C019A0CF8200C0CF8102C04980130EB
:102808000490E7E07A285DD84B280ED8472859D895
:1028180029282DD8252852D054D820287AD02338D2
:10282800D0F1000B4BEB000B74E04C382E2849D844
:10283800DFE800F070484848484848484848484851
:102848004B484848484848484859484B4B595959B3
:10285800704B6D487048184B184848827F4B484861
:102868004B487F0000204FF0000B4FF0040A38E07F
:102878002A380122C0B202FA00F010EA0E0F49D13C
:1028880010F0625C2FD110EA020B43D06046013C85
:102898005444B4FBFAF40AFB04F4002D61D0A3EB12
:1028A800050CA444B4453FF66BAF002868D1042B4F
:1028B80047D158F8043B2360043404232AE0019AE2
:1028C800013A01924FF0000B24E011F8010C6C283A
:1028D80034D111F8023C00206C2B8346C5D14FF04F
:1028E800080A5346D3E708F10708073428F0070811
:1028F80024F00704F8E802AB35B106982044B0424A
:102908003FF63EAFC4E900AB08344FF0000B4FF080
:10291800080A534611F8010F002878D0BBF1000FC0
:102928007FF470AF2528F5D1019B4FF0010B0133DF
:1029380001934FF0040AECE7584694E700208346D9
:10294800A5E7082B02D06FF015001BE708F1070870
:1029580028F00708F8E80223C4E90023083408230C
:10296800D8E768B9042B02D108F10408A4E7082BBA
:10297800E9D108F1070828F0070808F10808EDE789
:10298800059A013A059258F8042B009210E7039A29
:10299800900720D5A4EB050E4FF0010C4FEA9E00DE
:1029A800BEF5007FCFD20F2FCDD8F5B107F1400289
:1029B800C0B20DEB020E019A0EF8200C0EF8102C86
:1029C800BCF1000F3FF41AAF60F07F0009F1010974
:1029D8000EF8200C0137C5F1080204344FF6DA7EF0
:1029E800069297E74FF0000CDAE7BCF1000F01D030
:1029F8000136EFE7029802360028EBD10098CDE9BE
:102A08000631FEF7BFFE0644DDE90631E2E7631B47
:102A1800B3F5806F97D23DB9A6F10804E018B1E686
:102A28004C93049080C105909B08029A28602B70F3
:102A38009DF81030C2B1EB7085F80290B9F1000F23
:102A480005D008A80022C5F1010C97420ED1C5F1A6
:102A580001030DF120084FF0000A0DF1300B01932E
:102A6800574512D1601B8DE66B70E5E710F8013B06
:102A7800190608D50CEB040E03F07F03B6453FF6A4
:102A88007FAE04F8013B0132DFE7B9F1000F03D054
:102A980098F90020002A17DB029BD3B11AF80B2003
:102AA80004F8012B0022019B18191044B0423FF68C
:102AB80067AE98F80000009904F8010B20460392CD
:102AC80046F0EEFA039A14440AF1010A08F10108E3
:102AD800C6E798F8002055F822300093029B00982A
:102AE80045F82230FEF74EFE421CDCE76FF00D0081
:102AF80048E600BF2DE9F04F97B00446894600AF7D
:102B080090F802A0D7F880B03B62CBF3C003FA621A
:102B1800BB6141B9457800780AEB800020444D45F7
:102B280017D8A0EB0409E378FB61BAF1000F02D0D3
:102B38001BF0010F16D1FB6953BBFB6A1BB13A6A44
:102B48004946204698474D4628465C37BD46BDE86D
:102B5800F08F461C09F101093046FEF713FE0130DB
:102B68003044DCE72378626899007A62FA6A79610E
:102B780004EB8301002A40F000814D460E4601EB2C
:102B88000A094FF000084E454CD101EB0A0610E047
:102B98001BF0020FD1D023789A0004EB83017A61ED
:102BA80062687A62FA6A002A77D14D4601EB0A0612
:102BB80090461BF0050F0CBF02230123FB62FB6943
:102BC80006EB430A0BF00203BB625645BCD016F86D
:102BD800021B16F8013C54F82390994B994502D3EF
:102BE800984B994536D3BB69002B40D0786A31F0B1
:102BF8007EF900283BD0E9468AB06A46924B536179
:102C08007B6AC2E906314FF4007313848F4B42F894
:102C1800103F00234FF412518D48023D00F0B4FCE0
:102C2800CD46D2E716F8013BF96254F82300FEF7C7
:102C3800A9FDD7F884300130F96A4BB1D7F888304C
:102C480098453EBFD7F8843023F8180008F10108EA
:102C5800054498E7BB6923B1786A31F048F9002840
:102C6800C9D11BF0010F05D1FB6AED1AADE7BB6AAC
:102C7800002BAAD04846FEF785FDD7F8843053B11B
:102C8800D7F8883098453FBF431CD7F8842022F8EE
:102C9800183008F10108054497E7BAF1000F72D01F
:102CA8001BF0040672D0D046002607F148005246B1
:102CB8003B61B96246F0F4F9B96A3B6901EB0A0273
:102CC800F969BA62FA695200FA60BA6A02EB41021B
:102CD8003A610BF00202BA603A69B96A8A4257D17E
:102CE8001BF0020F62780CBF4FEA580100217A628C
:102CF8001BF0010F3244D2B240F09F801BF0040F4A
:102D080014BF40460020BB616270A0702046E1708D
:102D18003A6A7969FB6A9847051EFFF615AFBB69E1
:102D280041463A6A07F1480023707B6A84F802A09A
:102D38006370FB69E370FB6A9847B0F10008C0F262
:102D4800BB807B69A9EB0A013A6AC91AFB68C91AF0
:102D5800D7E90A0398470028C0F2B080A8444FF08A
:102D6800000B07F1380A08EB0005B34572D30021C0
:102D78003A6AFB6A08469847E6E656464FF0000866
:102D880007F1380093E75646D04697E7B04695E7EF
:102D9800BA6A12F8021B12F8015CBA6254F82500EC
:102DA800274A904202D3274A90421ED3BA6932B1C9
:102DB800786A7B6031F09BF87B6800288CD1BA6810
:102DC80002BB08F1280207F1300C08F1010008F1F4
:102DD8000208944407F158025FFA88F852FA80F022
:102DE8000CF8101C00F8105C76E7BA693AB1786AFA
:102DF8007B6031F07CF87B6800287FF46DAF1BF0B6
:102E0800010F09D006F1280207F13000711C1618CD
:102E180006F8205CCEB25FE71BF0040F3FF45CAF0E
:102E280008F1280207F1300008F1010102EB00085F
:102E380008F8105C5FFA81F84EE7002063E700BFEE
:102E48004C93049080C10590704B059004000001DC
:102E5800009804901BF80A3054F8239087F837300C
:102E6800D7F884302BB3D7F888309B4521D2D7F8D0
:102E7800843033F81B803A6A012107F13700FB6A76
:102E8800984700281ADB0544B8F1000F06D14846D8
:102E9800FEF778FC00F101081FFA88F83A6A414603
:102EA8004846FB6A9847002808DB05440BF1010BEC
:102EB8005BE74FF00008DEE7454645E6054643E692
:102EC800014B1860704700BF3000002480B50546EC
:102ED8000E461746984608F0A9FEDFF820900346EC
:102EE80001F0C2FB0446424649F8003039463046F4
:102EF800A84754F8090001F083FA00BF0800000051
:102F0800044608B5EFF31183102383F31288BFF347
:102F18006F8F01F0DDFB01F037FC33F0B7F9204685
:102F280001F0C2F9024831F009F831F0BAFCFCE7C7
:102F3800244C0590054B00205A6822F002025A6082
:102F48005A6822F001025A60704700BF0010005C06
:102F5800EFF31180102383F31288BFF36F8F094BAF
:102F68001A683AB9084A116841F480711160116809
:102F7800C905FCD51A6801321A6080F31188BFF3BD
:102F88006F8F7047AC1F00240048025810B5EFF34C
:102F98001184102383F31288BFF36F8F134B1A68C1
:102FA800C2B9134B0122BFF35B8F53E8001F0029FE
:102FB80003D143E800200028F7D1BFF35B8F04D189
:102FC8000C4A02210C4831F0EBFA84F31188BFF364
:102FD8006F8F10BD012A04D108490A6822F4807253
:102FE8000A601A68013A1A60EFE700BFAC1F0024B4
:102FF800A81F0024584C0590909804900048025847
:1030080008B501F0A7FB01F035FB0C4B0C4A1A6020
:103018000C4AD36823F0070343F00203D3600A4B3A
:103028001A6841F20303B3EB124F06D1074AD2F8EC
:10303800083143F00103C2F8083108BDB003002489
:103048000090D003004802580010005C0080005136
:103058002DE9F047044607464FF00109DFF8508094
:1030680014B93846BDE8F08794FAA4F5B5FA85F5A1
:1030780009FA05F32E0108EB05156FEA030A24EA9D
:1030880003042B7B002BEBD058F806301B694BB997
:1030980046440222284607EA0A077368196831F08D
:1030A8000FFADDE7284698470028D9D1F0E700BF96
:1030B8000899049030B5002289B00F490F4834F0C0
:1030C800B2FA0022002300240D4D0E492846009430
:1030D800CDE906230E234FF44072CDE90334CDE940
:1030E8000144094B08F0D8FA0849284634F0D7F8C3
:1030F800204609B030BD00BF19310090681900247E
:10310800C0140024002D002435340090A74C0590ED
:10311800014808F00FB800BF980C00242DE9F047CB
:10312800804620480F4631F0A3F90646002832D0E1
:1031380000252846BDE8F087237B83B12368DB6838
:103148000BB120469847636883F8069023681B698B
:10315800CBB9636802222046196831F0B1F901360B
:1031680010345445E8D3B8F1000FE2D0002DDFD079
:103178002846FFF76DFF0546002FF7D00021642091
:1031880034F041F9F2E7204698470028E1D009FADF
:1031980006F31D43E3E7044C0546DFF810A04FF0A3
:1031A8000109DEE7C01F00240899049018990490CB
:1031B800014B53F8200070477499049008B50346F2
:1031C80008462BB1044A136000F074FC002008BDC7
:1031D8006FF01500FBE700BF3400002410B5044C65
:1031E800237813B9034807F0A5FF0123237010BD06
:1031F8009E280024980C002410B504460B4831F092
:1032080037F95CB10A4BBFF35B8F53E8001F0139F4
:1032180043E80012002AF8D1BFF35B8F054834F069
:103228000EFA0548BDE8104007F084BFB81F002417
:10323800BC1F002468190024980C00240020064BA9
:10324800BFF35B8F014653E8000F43E80012002AE2
:10325800F9D1BFF35B8F7047B81F002470B5FFF733
:10326800EDFF084C0546084EB44200D370BD6368B4
:103278005B792BB123685B6813B1294620469847D0
:103288001034F1E7089904901899049010B5044C8B
:103298000449204630F062FF034B1C6010BD00BF9C
:1032A800B00B002460990490B01F002400230D4A3D
:1032B8004FF47A710C4810B513700C4A13600C4A1D
:1032C8001360FFF77BFFFFF7E1FF0A4B0A49184637
:1032D8008B4200D310BD1A1A5C68103312110132E8
:1032E8002271F5E79F28002493440390B81F002417
:1032F800BC1F0024089904901899049001460022E4
:103308000023014830F04BBFB00B0024014830F0D7
:10331800E4BF00BFB00B0024024B0146186831F02F
:1033280037B800BFB01F0024014831F06CB800BFA7
:10333800B00B0024264B70B51878002846D0FFF74C
:10334800E5FF054600283ED1224B234C1B68002B85
:1033580012DD34F020F90A220023FEF7E7F9D4E958
:103368000032C01A40F2E93361EB0201984271F170
:10337800000101D3FFF772FFD4E9003213F57A7325
:1033880042F10002C4E90032BDE87040FFF7CCBF4B
:1033980063685B7923B12368294620461B689847F0
:1033A8001034B442F4D32846FFF7B6FF0B4BBFF3F3
:1033B8005B8F53E8001F013943E80012002AF8D157
:1033C800BFF35B8FC0E7064C064EEAE770BD00BF4F
:1033D8009E280024B81F002460190024BC1F002464
:1033E800089904901899049070B50D4D297861B921
:1033F8000C4C01200C4EFFF791FEB44206D3FFF7A8
:1034080099FF0028FBD101232B7070BD63685B799D
:103418001BB1236820469B6898471034EDE700BF2E
:103428009F280024089904901899049000212DE9F8
:10343800F0470846FFF772FE044658B34FF4FA788F
:103448004FF000091C4B01F00FF91C4A1B58136080
:1034580033B11B4B1B68092B02DD1A4807F06AFEC3
:103468000025194FDFF85CA044B12046FFF7F0FDB6
:10347800044618B94FF0FF384FF0FF39FFF75AFFED
:10348800064628B9B5B942464B46504607F08EFE67
:103498003546E9E74FF0FF384FF0FF39D2E72B68A0
:1034A8009B691BB100222846114698471035BD423A
:1034B800F5D3E8E7054DFAE708000000B41F00243B
:1034C800BC1F0024980C00241899049008990490B3
:1034D80013B5184830F0CCFF174B1B7873B1EFF3D6
:1034E8001184102383F31288BFF36F8FFFF722FF35
:1034F80084F31188BFF36F8F02B010BD0F4B1B68A8
:10350800002BF9D050B9002200230D48CDE9002343
:1035180042F21072002308F09BFEEDE70928EBD178
:10352800074834F08CF8074802B0BDE8104007F0AF
:1035380001BE00BFBC1F00249F280024B41F002424
:1035480068190024980C0024064B10B504461B6823
:1035580098472146A060044830F0A0FEBDE810401E
:10356800FFF7B6BF34000024B00B0024044A054B13
:103578009B1AB1EBD30F34BF52F8310000207047CB
:10358800F8970490089904902DE9F04F8FB0C1F393
:103598004A280D46914604AF0C0DB8607B60B8F11F
:1035A800000F63D0002607F114034FF0040B4FF00F
:1035B8000A0AC7F80C8032467E624846C7E90766A1
:1035C800019307F11C03CDF808B0CDF800A0F96805
:1035D800FFF790FAB0F5006F03461CD36C468AB02B
:1035E800D9F8041004AB26481A46C3E9050140F28D
:1035F800FF71D9614FF400711984224B42F8103FD2
:103608004FF4125133462048FFF7BEFFA5462C372A
:10361800BD46BDE8F08FC0F30A0804F117003B600F
:10362800184468F3532520F007008008FFF766FE6A
:10363800044690B13B6800F11001144A4846F9610C
:10364800C7E9083607F11403CDF808B0CDE900A39F
:1036580007F11C03F968FFF74DFA68F353257B68F7
:10366800B96820462A4630F04BFFD0E704F117002E
:1036780020F007008008FFF741FE0446EDE700BF91
:10368800BC4C05900400000140980490DB44039072
:103698002DE9F04F87B00446934698460391DDE93B
:1036A8001279DDE9105ABFB13B465246102100207D
:1036B800CDF80090CDF81490FFF74AF8B0F5006FF8
:1036C80006460AD340F2FF73174A0221174807B08B
:1036D800BDE8F04F30F06DBF3E4604F0070405F139
:1036E80017000BF0070BE400304444EA8B1420F079
:1036F800070044EA4624800844EA0554FFF7FEFD23
:10370800054640B13FB13B46524631461030CDF8F0
:103718000090FFF71DF8434622460399284607B054
:10372800BDE8F04F30F0ECBEFB4C0590409804909B
:10373800406820B1034BC01A40F3CF0070474FF0E8
:10374800FF307047F89704900EB403B503AB0146F9
:10375800054853F8042B019301F0AEF902B05DF867
:1037680004EB03B0704700BF1D460390CA0605D49A
:103778008B064CBF02490349FFF7E6BF704700BFFD
:10378800089F0590776205902DE9F04F89B09B4618
:1037980004460D46149B90469DF84CA00693159B35
:1037A800179E0593169B0493BAF1000F00F09D80B5
:1037B80006F4807306F00209079330F07FFE024694
:1037C80000283ED091492046FFF7BEFF0746B9F1D1
:1037D800000F08D016F0440F35D12A468C492046F0
:1037E800FFF7B2FF074406F0010353B1894B2046A7
:1037F800894953F82A20894B002A08BF1A46FFF73F
:10380800A3FF06F48073002B49D006F00803002BB1
:1038180063D1B8F1000F66D0424681492046FFF7D0
:1038280093FF0546069B3D44002B6DD1049B002B5E
:1038380073D1F30700F1E48031462046FFF796FF85
:10384800D8E00746C3E7774B18680028CAD0764BFC
:103858004FF47A794FF03C0C1B68B5FBF3F5B5FBD8
:10386800F0F100FB11554FF4616309FB05F5B1FB5D
:10387800F3F2B5FBF0FE03FB121100FB1E55B1FB82
:10388800FCF309FB05F50CFB1311B5FBF0F50091F2
:1038980020466649CDE901E5FFF756FFA2E706F0A5
:1038A8000803EBB1624B2046624953F82A20FFF720
:1038B8004BFF0546B8F1000F05D04246584920464F
:1038C800FFF742FF0544BBF1000FABD05A465A49F7
:1038D8002046FFF739FF0544A4E74FF0000BE1E766
:1038E80006F00805E6E745469CE7BBF1010F069B95
:1038F80006D1002B64D1049B002B7BD000250CE063
:10390800002BF8D04D485CE04D48069B22464D49B7
:1039180030F0BCFA049B002B68D0DFF82C81DFF86C
:103928002C91049F4FF0000B31462046102F28BFE2
:103938001027FFF71BFF5D4545DC059B4FF0010B8A
:10394800494620461A78FFF7FFFE1BF0070F03D100
:1039580041462046FFF7F8FE5F453BD9059B49469F
:10396800204613F80B20FFF7EFFE0BF1010BBBF11C
:10397800100FEAD14FF0000B35492046FFF7E4FE5F
:103988005A46059B20469A5CA2F120015F293149DD
:1039980028BF2E22FFF7D8FE0BF1010BBBF1100F49
:1039A8001DD01BF0070F03D141462046FFF7CCFE80
:1039B8005F455A46E5D841462046FFF7C5FEEBE786
:1039C8001F485546A1E7414620460BF1010BFFF77A
:1039D800BBFEB0E720492046FFF7B6FEC5E7059BCA
:1039E8003B440593049BDB1B04939AD1BAF1000F67
:1039F8007FF41FAF204609B0BDE8F04F30F0FDBDA1
:103A0800064A20460449FFF79FFE15E7384D059002
:103A18003C4D059084990490EE9E0590334D059099
:103A2800614D0590C81F0024C41F0024454D059012
:103A380098990490654D05906B4D059053460390F9
:103A48001D460390C14A0090E3B70590704D05905C
:103A5800764D059073660590E1B7059042F20F73B5
:103A6800114A8B4273B5044628BF0B4605680521E9
:103A780068462DF0D5FC636806460B2228465B682D
:103A88000A4930F0ACFD63683246694628465B68EF
:103A980030F0A5FD63681B2205495B68284630F0B5
:103AA8009EFD02B070BD00BF829F0590944D0590A9
:103AB800784D059000210123064A904206D8064A0F
:103AC80001B901231360054B1860704740080121B4
:103AD8005B00F2E740420F00C41F0024C81F002407
:103AE800F8B50D4604464618054FB44201D128469C
:103AF800F8BD14F8011BBB6801485B689847F4E7F8
:103B080030960490014B036002207047E0990490BE
:103B1800104B70B51C680D46B4B10F4B19680023E3
:103B28008B4202DB6FF0010070BD224612F8146B65
:103B3800864202D001331446F2E7E06833F04FF9C9
:103B480028B100202C60EFE76FF00C00ECE76FF075
:103B58001200E9E740000024009A04902DE9F84398
:103B68000646FDF70FFE0546EFF31188102383F391
:103B78001288BFF36F8F114B1C68D3F804909C42D6
:103B880008BF002434B988F31188BFF36F8F20462B
:103B9800BDE8F883A7683846FDF7F4FDA84206D1CA
:103BA8002A463946304645F0C8FA0028EBD04C453D
:103BB80001D02468E6E70024E5E700BF44000024BC
:103BC8002DE9F0410E461546FFF7C8FF044628B315
:103BD800C3681BB35F690FB3062E07D0072E20D02A
:103BE8002A4631463B46BDE8F0411847838A3BB92F
:103BF8002A463146B84750B9A38A0133A38206E062
:103C08004FF6FF72934204D00133A3820020BDE82F
:103C1800F081124A0121124830F0C2FC6FF0150001
:103C2800F5E745B12A7832B10022314682822A4628
:103C38005B699847EAE7A38A012B08D12A4607213E
:103C48002046B8470028E2D1A38A013BD6E70BB14A
:103C5800013BDAE7034A0221DDE700BF134E059076
:103C680008980490354E059003480021034A08B58A
:103C7800121A30F0F1FD08BD800D0024D42C002468
:103C88000748084A0849121A08B530F0E7FD0748FE
:103C9800074A0849121ABDE8084030F0DFBD00BFE6
:103CA80000000024440D002480C105900000002479
:103CB8000000002480C105902DE9F047064600AFBA
:103CC8000C46002936D0E9468AB0A3686D46D1E98A
:103CD800001221484FF0050AA846C5E90501C5E9C3
:103CE800072348F810AF002342464FF421511B48E0
:103CF800FFF74AFCCD466369AD46D4E9031218487C
:103D0800C5F810A0C5E90501C5E907230023424607
:103D18004FF421511148FFF737FCCD46E369114AAA
:103D280001210E4830F045FCA3690F4A01210B48D8
:103D380030F03FFC012E07D1EFF305830B4A103B0F
:103D48003146064830F035FC2146304606F040FE44
:103D5800BD46BDE8F08700BF5E4E05908098049090
:103D68008D4E0590BC4E0590CB4E0590F94E0590B2
:103D780030BFFFF7FDBF00BF2DE9F0410B4E0546F0
:103D8800DFF82C80324606EB0807CC1B0949204691
:103D980045F086F9A019083C4246002145F0A8F9EB
:103DA80007F10800C5F89040BDE8F0810000000068
:103DB8000800000018990490054B5A699B689A42BC
:103DC80004D0044A536843F080535360704700BFDF
:103DD8006021002400ED00E070B5294C06460D4630
:103DE8002848294930F047FDA36AD9043CD525481D
:103DF800264930F040FD1720A36A1A0504D521484A
:103E0800234930F038FD18201D4CA36A9B0512D5B4
:103E18001C48204930F02FFDA36BA26A100409D575
:103E28001D4A0121174830F0C4FB1EB1A36A23F4D0
:103E38000043A3621920124CA36A590504D51148FE
:103E4800164930F018FD1A20A36ADA050ED50D4878
:103E5800134930F010FD1B20094A936A43F47F434D
:103E6800936200232B7070BD1620C5E7A36A9B04DC
:103E7800F2D504480B4930F0FEFC1C20ECE700BFEB
:103E880000ED00E0809804900C4F0590224F0590BB
:103E9800334F0590464F05905F4F0590744F05903E
:103EA8008F4F0590A74F059010B5204C2049214809
:103EB80030F0E1FCA36A990136D51E481E4930F05E
:103EC800DAFC1E20A36ADA0104D51A481B4930F02F
:103ED800D2FC1F20154CA36A1B0304D515481849AA
:103EE80030F0C9FC2120A36A590304D511481549AB
:103EF80030F0C1FC22200D4CA36A9A0304D50D486A
:103F0800114930F0B8FC2320A36ADB0304D5094823
:103F18000E4930F0B0FC2420044A936A6FEA034348
:103F28006FEA1343936210BD1D20CBE700ED00E05C
:103F3800D64F059080980490EE4F0590015005905B
:103F48001B500590395005905E50059078500590AB
:103F58002DE9F843364D8046894636483649174696
:103F680030F089FCAB6ADE0627D511243349314885
:103F780030F081FCAB6A1D0704D5122430492D4866
:103F880030F079FC2A4DAB6A980718D52D49294895
:103F980030F071FC6E6BAB6A190646D52A4A334677
:103FA8000121244830F005FBB9F1000F03D0AB6ABA
:103FB80023F08003AB62132403E01024DAE76FF0E8
:103FC80015061B4DAB6ADA0704D514241F49194896
:103FD80030F051FCAB6A9B0604D515241C491548E2
:103FE80030F049FC124B9A6AD50602D49A6A9007B7
:103FF8000AD55B68190507D54146304600F0D8FA5E
:1040080010B180F309880224094B9A6A920603D5F5
:104018005A6A22F400525A629A6A204642F0FF0213
:104028009A6200233B70BDE8F8836FF01506C2E77B
:1040380000ED00E080980490A3500590B9500590D9
:10404800334F0590EC500590045105901A51059096
:10405800A74F05902DE9F041664B8AB0044600262B
:10406800D3F8048000AFC8F3080586F31188BFF3BE
:104078006F8F02F07F43B3F17F4F07D102F00C033B
:10408800082B12D15C495D4830F0F5FB0026344618
:104098000023FB71EB1E092B00F28B80DFE803F095
:1040A8000A81847D89898989898710074CBF0C46D4
:1040B8000126EDE75249514830F0DDFB4D4D002314
:1040C800FB71EB6A9A0705D54E494C4830F0D3FB93
:1040D800002332E0EB6A002B01DA4B49F5E7EB6A83
:1040E8005B00F5D54949454830F0C5FB6B69A269C5
:1040F80043F480736B61BFF34F8FBFF36F8F6B69AE
:1041080032F8022C23F480736B61BFF34F8FBFF337
:104118006F8F4DF602739A4208D0AB6ADBB27BB35D
:10412800FA1D01212046FFF713FF38E02368384ABB
:104138000121324830F03DFA2368FA79E2B907F1F3
:10414800080504F1200C2068083454F8041C2A4699
:10415800644503C21546F6D17A6A002E45D0C2F3EB
:10416800080121B96FEA52226FEA42227A6207F106
:1041780008011846FFF7A0FD2837BD46BDE8F081C5
:10418800AB6A13F47F4F04D0F91D0120FFF724FE1A
:1041980005E0AB6AB3F5803F9AD3FFF785FE034687
:1041A800CBE7FA1D0021BDE7F91D0020EEE719490C
:1041B8008BE718F4F87F184AE8468AB0174B18BFFF
:1041C80013466A461649103DC2E905134FF40073B9
:1041D800D5611384134B42F8103F00234FF411515B
:1041E8000648FFF7D1F9C54672E722F4FF7222F0BC
:1041F8000102BBE700ED00E067510590809804904C
:1042080092510590A9510590CA510590D851059031
:10421800F7510590135205904E510590395105906C
:104228003752059004000001044B5A6942F010020D
:104238005A615A6922F008025A61704700ED00E09D
:10424800EFF30880EFF3098101B57246FFF702FF2B
:1042580001BD00BF002080F31488BFF36F8F0F48A3
:1042680080F3088830F0F1F800200D490860BFF3AA
:104278004F8F00F03DF8102080F3118809484FF463
:104288000461401880F30988EFF314800221084381
:1042980080F31488BFF36F8F00F05CF960A30024EB
:1042A80094ED00E0C03A0024BFF34F8F0549064B58
:1042B800CA6802F4E0621343CB60BFF34F8F00BFBC
:1042C800FDE700BF00ED00E00400FA050749002300
:1042D800D1F890201846C2F30722934200DB7047BA
:1042E800C1F898300133C1F8A000F6E700ED00E00E
:1042F80070B572B6002484F31388FFF7E7FF3E4BCE
:104308004FF0FF32C3F88020C3F88420C3F8882018
:10431800C3F88C20C3F89020C3F89420C3F89820E1
:10432800C3F89C20C3F88021C3F88421C3F88821EE
:10433800C3F88C21C3F89021C3F89421C3F89821BD
:10434800C3F89C212D4A536913F4803339D0C2F83D
:104358008440BFF34F8F536923F480335361BFF315
:104368004F8FD2F8803043F6E074C3F3C900C3F32B
:104378004E335B0103EA0406014646EA81750139BA
:10438800C2F87452F9D2203B13F1200FF2D1BFF3D7
:104398004F8FBFF36F8FBFF34F8FBFF36F8F174BE5
:1043A8005A6922F400325A610022C3F85022BFF33E
:1043B8004F8FBFF36F8F62B6BFF34F8FBFF36F8F0F
:1043C80070BDC2F88430BFF34F8FD2F8803043F607
:1043D800E074C3F3C900C3F34E335B0103EA040678
:1043E800014646EA81750139C2F86052F9D2203B8C
:1043F80013F1200FF2D1CAE700E100E000ED00E080
:10440800084B9B6883420BD1EFF3058343B1064BFE
:104418005A6842F080525A605A6A22F400425A623C
:1044280007F00ABC6021002400ED00E015498A6805
:104438004FF030001044EFF3098C80E8F01F102093
:1044480080F31288BFF36F8F0F4F4FF000664A69F1
:104458008A603E60D2F890000C4C2060D2F894003C
:104468000023C2F8943080F3118804B5104600F098
:10447800ABF9BDE8044002F1300090E8F01F8CF37E
:10448800098870476021002404ED00E0F81F00242B
:104498001EF0040F0CBFEFF30880EFF30980816969
:1044A80011F8021C0229FFD001B5724630F0D8F984
:1044B80001BD00BF09010028C9B206DB00F1604058
:1044C80000F5614080F80013704700F00F00014BC1
:1044D8001954704714ED00E000B2002807DB0123EF
:1044E800410900F01F00024A834042F8213070471A
:1044F80000E100E000B200280CDB4309012200F0D3
:104508001F0005492033824041F82320BFF34F8F15
:10451800BFF36F8F704700BF00E100E04209054B11
:1045280000F01F0053F82220012303FA00F0104086
:10453800704700BF00E100E0044B054A23F07F0309
:104548009360BFF34F8FBFF36F8F704700040090E5
:1045580000ED00E008B5FFF7EFFF084AD2F8883011
:1045680023F47003C2F88830FFF77EFBFFF788FB5F
:1045780000F05CF830F0A2F906F04EFB00ED00E028
:1045880042F8203C203A009B08495360019B21F0E7
:1045980001019360029B9161D3604FF08073D361F6
:1045A80000230265C0F89430704700BFD52E0090F4
:1045B8000A4A0346906878B113F1160FD0F88000C4
:1045C80005D0A0F140029A4205D8834203D2814225
:1045D80028BF002070470020704700BF60210024DA
:1045E80015460D4A0E4608B50C4B9060D0F8902041
:1045F8001A6000F0E9F82C4686F309880020044B7D
:1046080098472046002100220023024C2047000042
:104618009D480390D52E009060210024F81F0024A7
:10462800014B10221A61704700ED00E00023044896
:104638001021C2180133962B82F80013F9D1704764
:1046480000E100E008B5EFF30583064A103B02EBF2
:10465800C30152F8330049688847BDE80840FFF7AE
:10466800ABBB00BFD40600240148006870470000B7
:10467800F81F0024154A70B5536913F4803323D109
:10468800C2F88430BFF34F8FD2F8803043F6E0741D
:10469800C3F3C900C3F34E335B0103EA04060146C2
:1046A80046EA81750139C2F86052F9D2203B13F10C
:1046B800200FF2D1BFF34F8F536943F48033536116
:1046C800BFF34F8FBFF36F8F70BD00BF00ED00E0E9
:1046D800134A002370B5C2F88430BFF34F8F536973
:1046E80023F480335361BFF34F8FD2F8803043F601
:1046F800E074C3F3C900C3F34E335B0103EA040655
:10470800014646EA81750139C2F87452F9D2203B54
:1047180013F1200FF2D1BFF34F8FBFF36F8F70BD2E
:1047280000ED00E0002910DD00F01F030B44BFF38B
:104738004F8F07490344C1F8680220301A1A002A2B
:10474800F9DCBFF34F8FBFF36F8F0020704700BFB6
:1047580000ED00E00B4B5A6912F4003211D1BFF39F
:104768004F8FBFF36F8FC3F85022BFF34F8FBFF344
:104778006F8F5A6942F400325A61BFF34F8FBFF30B
:104788006F8F704700ED00E0BFF34F8FBFF36F8F5F
:10479800064B5A6922F400325A610022C3F85022AB
:1047A800BFF34F8FBFF36F8F704700BF00ED00E07E
:1047B800024B0121024A034800F08CB8000008248B
:1047C80000000024549A0490D0F880204021054B22
:1047D800403A18461A60044AC3E90112012100F060
:1047E80083B800BFFC1F002400000B1508B5034662
:1047F8001048D0F89020C2F30722013A934207D913
:104808000D4801210D4A2FF0D4FE6FF0150008BDA8
:10481800C0F898300A6822F01F021A4342F01002CA
:10482800C0F89C208A6842F00102C0F8A02018460F
:10483800EDE700BF00ED00E0689804904E52059047
:10484800F0B50E4685B01F4604460025B5420DDA80
:10485800606810B397B1431E18420AD0104A2B461D
:10486800012110482FF0A5FE6FF01502104605B083
:10487800F0BD1F28F2D921680B42EFD1236801A9A6
:10488800019330F01CF8A3680343D0B20393FFF7F9
:10489800ADFF10F1160FE7D0421C01350C34D5E7F7
:1048A8007452059068980490044B0522C3F894202C
:1048B800BFF34F8FBFF36F8F704700BF00ED00E06D
:1048C800BFF35F8F024B0022C3F89420704700BFEC
:1048D80000ED00E010B5034C01232278FFF7B0FF8C
:1048E800207010BDA12800240B4A08B500231278B7
:1048F800FFF7A6FF10F1160F07D0084A0021D2F8DB
:104908009030C3F30723984200DB08BDC2F8980033
:104918000130C2F8A010F2E7A128002400ED00E061
:104928005F4860492DE9F043D0F8903085B00D68B4
:10493800C3F307239D4200F2B080FFF7C1FF496827
:104948000022954201F10C011BD1574C6846574F84
:104958002570FFF7D7F800250646DFF85481DFF801
:104968005491AE4220D1237800204D49D1F89020AF
:10497800C2F307229342C0F28A800020FFF794FF17
:104988004FE0C0F8982051F80C3C23F01F03134364
:10499800013243F01003C0F89C3051F8043C43F056
:1049A8000103C0F8A030CCE700984FEA051C00EBE3
:1049B8000511CB683B40B3F5000F49D00AD8B3F5D1
:1049C800001F31D0B3F5800F37D0B3F5801F13D057
:1049D8000135C6E7B3F1007F43D0B3F1805F49D01A
:1049E800B3F1807FF4D150F80C3088682FF067FF5E
:1049F8004A6840F0887009E050F80C3088682FF059
:104A08005EFF40F088504A6840F43020039001A9C6
:104A18002078CDE90123FFF7E9FE002833DA6FF0AB
:104A2800150005B0BDE8F08350F80C3088682FF009
:104A380046FF4A6840EA0900E8E750F80C30886801
:104A48002FF03DFF40F000704A6840F40030DDE789
:104A580050F80C3088682FF032FF4A6840F08270B6
:104A6800D4E750F80C3088682FF029FF4A6840F4E2
:104A78008020CBE750F80C3088682FF020FF4A6878
:104A880040EA0800C2E7237801332370A0E7C1F8A1
:104A980098300133C1F8A00068E74FF0FF30C0E755
:104AA80000ED00E034990490A12800240000F0FFF4
:104AB8000000021100000811F0B587B007460E4645
:104AC80014460021102268461D4644F011FB0223BB
:104AD8002A4621468DF802306846044BCDE9047613
:104AE80001932CF0A3FD07B0F0BD00BFED48039083
:104AF80008B5024B1B689847002008BD0820002411
:104B0800034B044A1860937843F00203937070478C
:104B1800082000244C00002408B505482FF00EFAA0
:104B2800002383F31188BFF36F8F0423184602DF35
:104B38009A5205900649074821F00701C1F1105221
:104B480008B502F500222FF049F9002008BD00BF82
:104B5800CFAF00240C2000244FF0FF324FF0FF337A
:104B6800014806F0F1B900BF5C000024014806F0D6
:104B78005FBA00BF5C00002438B50546FFF7ECFFBC
:104B8800082108482A462FF072F8044628B925B1AA
:104B9800054B0C22FFF768FD1A50FFF7E7FF204688
:104BA80038BD00BF0C2000240C00000038B50446B6
:104BB8000D46FFF7D1FF082221462B4607482FF064
:104BC800D5F8044628B925B1054B0C22FFF74CFD52
:104BD8001A50FFF7CBFF204638BD00BF0C20002439
:104BE8000C00000010B50446FFF7B6FF0348214645
:104BF8002EF0DBFFBDE81040FFF7B8BF0C20002403
:104C080070B541690446867A0A4D59B1437ADB0783
:104C180006D42C2303FB06535B6A1B689B689847E2
:104C2800002363612C20214606FB0050BDE870403C
:104C380032F0AABAD40C00242C22024B02FB00301A
:104C4800704700BFD40C0024827A2C21054B01FB4D
:104C580002339A6A1B7F801A1B3323F00303B0FBCD
:104C6800F3F07047D40C002438B52C24827A064B14
:104C780004FB02335B6AD3E901240C601568FFF773
:104C8800E3FF04FB005038BDD40C00242DE9F043A9
:104C980085B0054690461C466846039132F07DFC77
:104CA800DDE90067EFF31189102383F31288BFF35E
:104CB8006F8F6B8B002B41D02A8B9A4225D900220B
:104CC8000023284606F004FA0446F0B189F3118857
:104CD800BFF36F8F039B002B41D032463B4668469B
:104CE80032F080FCA27A2C21254B204601FB0233AE
:104CF80003A95B6A1B681D68DDE90023A84760619A
:104D080070BB2046FFF77CFF24E0698B4B1E6B834A
:104D180089F31188BFF36F8F2B7F2A8B1B33AC6A03
:104D2800521A23F0030302FB0344154B154AEB1AEE
:104D38009B105343A3722B7FE372CBE789F311884F
:104D4800BFF36F8F23464246284606F0C1F9044652
:104D58000028BFD10024204605B0BDE8F083636178
:104D680001230025E27A04F1180023812946039BD8
:104D78006560638244F0BCF963692582E360EAE711
:104D8800D40C0024A38B2EBA70B50D4C2C2500B979
:104D980070BD037A4668002BFAD0013BDBB2037280
:104DA800002BF5D1C3604360837A05FB03431B6A7C
:104DB80013B198473046EAE7FFF722FFFAE700BF4A
:104DC800D40C0024F7B506460D461446124F384653
:104DD80032F005F8E0B1BB68AAB2314638461B6824
:104DE8009847002802DB002003B0F0BD002CFBD15F
:104DF800AC42F8D22F1B042F28BF042704F04AFB2B
:104E080001A901903A46301944F04AF93C44EFE7C9
:104E18006FF01200E8E700BF149604902DE9F04106
:104E280090F8283004460F4600F1280603F01F03C7
:104E3800012B1BD0022B05D043BB90F829102FF073
:104E48009FFE03E0818DC9B200F056FF0546E8B128
:104E580030462FF0E8FD024668688368A2B99B686F
:104E68004BB13A463146BDE8F0411847818DC9B289
:104E78002FF06DFEEAE76FF08503104AFFF7F4FBA9
:104E880013500020BDE8F081DB68E9E794F82910A9
:104E980020462FF095FD02460028ECD030462FF032
:104EA800C2FD40B91369002BE5D03A463146204689
:104EB80098470346E1E7D368F5E700BF0C00000018
:104EC8002DE9F04F95B00D4600F128030446097E00
:104ED80002AF914631F08008BB600BD06FF0040838
:104EE800A64A0121A6482FF0B4FD40464C37BD46DE
:104EF800BDE8F08F6B7E03F00102B9F1000F17D007
:104F080019F10C0F14D0B2B919F1710F03D1284659
:104F1800FFF73AFFE9E79B4A0B4699480121CDF88C
:104F28000090C8462FF04FFB2846FFF72DFFDCE71F
:104F3800002A00F0C784002940F087842B8A072BB9
:104F48000FD9EA681368A3625368E362D5F804A02E
:104F5800E28DBAF1000F17D18B4A012188482FF052
:104F680078FD8A4A012186482FF073FD2846FFF70D
:104F78000BFFB8682FF057FD0346A069002B00F01F
:104F8800B884802100F0BEBC04F128002FF04BFD4E
:104F9800E0B99AF8193032B198071DD46E4688B036
:104FA80002AA7B4B05E05E0716D46E4688B002AABB
:104FB800784BC2E9053A032342F8103F70480B4684
:104FC8004FF4C251FEF7E0FAB546CAE70AB9724A89
:104FD800C3E79AF81930DFE7294600202FF0A1FC33
:104FE800054628B9684A012165482FF032FDC0E717
:104FF80094F828200023FFF737FB684E12F0600F63
:105008008351C2F3411308D0032B40F0EB816FF0BA
:105018008503FFF729FB335057E004F128002FF0F0
:1050280002FD94F82930002840F07681013B0A2BD4
:10503800EDD801A151F823F00352009017500090C9
:1050480087520090175000906D50009017500090B4
:1050580017500090175000900F5100901750009073
:10506800B5510090A069618D03697F29D3F880301C
:10507800CDD8A28D002ACAD1E28D002AC7D194F8D2
:105088002820D206C3D194F83420022A04D14FF044
:10509800FF33FFF7E9FABEE71A070BD5C9B22FF0BD
:1050A800FDFC804648B1638D3D4A012134482FF00C
:1050B80080FA2CE7012384F83D3094F83430012B32
:1050C8001FD1638DEBB984F83430FFF7CDFA33582C
:1050D800002B7FF44BAF0123B86823632FF0A3FCA8
:1050E800002840F0AB83E38D002B00F0A78329460E
:1050F80000202FF016FC0546002840F09B83294A23
:1051080071E70123DFE720462FF050FC628D01464E
:10511800FF2A3FF67CAFE38D002B7FF478AF94F83D
:105128002830DB067FF473AF94F83430002BAED010
:105138002AB1D2B220462FF0F3FC0028A7D0618D07
:1051480094F83C308B42C0D0C9B2204600F07CFDB8
:10515800638D804630B1144A0121009008482FF031
:1051680032FAD4E61A1E4FF00501204614BF022376
:10517800012384F834302FF00FFEA6E7CD520590B6
:10518800B8980490EE5205901D53059080530590F1
:105198003F5305904E5305905F5305900C00000057
:1051A8009753059087540590B953059094F8283083
:1051B80003F01F03012B7FF42AAFE38D002B7FF44C
:1051C80026AF628DFF2A3FF622AFA18DFF293FF659
:1051D8001EAF94F83430022B7FF459AFD2B2204678
:1051E800C9B22FF036FD10F1020F804640F0FF8063
:1051F800FFF73AFA46F8008067E7E38DA18D002BA8
:105208007FF405AF94F83430002B3FF440AF012B06
:1052180010D100297FF43BAF12F01F020DD1638D2E
:10522800012B7FF452AF94F870306FF3C30384F806
:1052380070304AE712F01F0217D0022A7FF445AFF8
:10524800B4F82A80B8F1000F7FF43FAF5FFA81FA13
:105258002046514600F05AFE0346FFF705FA335040
:10526800013306D14FF0FF3851E600297FF40FAF24
:10527800D5E74246514620462FF0DBFB25E7E38D74
:10528800A18D002B7FF4C3AE638D5FFA81F8022BEA
:1052980013D194F8283003F01F0358EA03037FF46E
:1052A800B6AE0122090AA0692FF0D5FB00287FF4C9
:1052B800AEAE012384F83D3007E794F834000028A7
:1052C8003FF4E5AE01280DD100297FF4E0AE12F0DD
:1052D8001F020AD1012B7FF4F8AE94F8703043F026
:1052E8000803A4E712F01F0212D0022A7FF4EDAEE1
:1052F800002B7FF4EAAE4146204600F0E5FD034668
:10530800FFF7B2F933500133ACD001224146B2E77E
:1053180000297FF4BCAEDDE70A2B3FF678AE01A189
:1053280051F823F0595300901750009017500090EF
:10533800175000901750009017500090D9530090C4
:1053480017500090D55700901750009003580090C0
:10535800E38DA18D022B7FF45AAE94F83430002BE4
:105368003FF495AE012B10D100297FF490AE12F0D6
:105378001F020DD194F870304FEA9308C3F300135D
:1053880008F0020848EA030806E012F01F0210D0ED
:10539800022A12D04FF0000805F10C0A50462FF0EF
:1053A800F4FAE38D98420ED26FF00B03FFF75CF925
:1053B80031E600297FF46BAEDCE7C9B220462FF056
:1053C800E1FC8046E8E7414650462FF0CDFA7CE6FE
:1053D80094F82820B4F82AA0D0064FEA1A235FFAD6
:1053E8008AFA09D029462046FFF718FD8046B8F109
:1053F800000F7FF48CAD68E6013B0E2B3FF607AE3D
:1054080001A252F823F000BF4D5400909754009029
:105418005B5500901750009017500090535500901E
:105428005355009017500090175000901750009057
:105438001750009017500090175000901750009088
:10544800B356009005F10C08B4F82EA040462FF092
:105458009CFA82450AD2B4F82EA020462FF0A6FA6C
:1054680048B101287FF4D3ADA16F05E040462FF085
:105478008CFA8246F1E7616F002900F021810A78F1
:105488004046524528BF52462FF05DFA1DE60AF104
:10549800010820462FF08AFA0146F8605FFA88F280
:1054A80020462FF017FB824630B9C14A43460121F6
:1054B800C0482FF07EF8AAE505F10C08D0F804B032
:1054C80040462FF062FA9BF80020904203D24046F3
:1054D8002FF05BFA0246594640462FF034FADAF8C4
:1054E8000CA0BAF1000F09D1298AE38D99427FF601
:1054F800ECADC91A40462FF041FAE6E5DAF80400A7
:1055080083681B6B13B9DAF800A0EAE7F9689847D3
:105518000028F8D0A0F1040B5BF8043F002BF2D070
:105528001B78002BEFD040462FF02FFADBF8003025
:105538001A78904203D240462FF027FA82B2DBF85D
:10554800001040462FF0FFF9E6E720462FF02EFA2C
:105558005DE55246032120462FF046FA8246002890
:105568003FF455AD2FF05AFAE38DE0B9BAF814209C
:1055780098463A85DAF8102005F10C0A1288504648
:105588007A852FF002FA804509D2E08D97F8282015
:1055980007F12801824228BF0246504674E7504668
:1055A8002FF0F3F9F2E79B460023DAF808203B7561
:1055B8009AF815307B75804B1340804A934263D12B
:1055C800102107F1180003F0B5FA002842DB07F1B3
:1055D8002803102807F11802DFF8E4C19E4628BF07
:1055E8001020404503F102033DD88000C7F80CE0C5
:1055F8000230387505F10C0A50462FF0C6F997F8B5
:105608001480D84528BFD846404503D250462FF0CD
:10561800BCF98046B8F1020FC34607F114015046A1
:1056280028BF4FF0020B5A46A8EB0B082FF08BF956
:10563800D7F80CB04FEA58030BEB58025A452AD159
:1056480018F0010F3FF441ADFA685046D15C2FF0D5
:1056580083F93AE558307FF4DAAC5A4A01215548C3
:105668002FF0F7F9D3E412F8011B08F101084FEA0B
:10567800111A01F00F011CF80AA01CF8011003F818
:1056880002AC03F8011CACE79AF814303B75DAF861
:105698001030FB60AEE71BF8011B5046C7E900322B
:1056A8002FF062F9D7E90032C8E720462FF07EF9DB
:1056B80020B101287FF4ABACA36F00E0636F13B98E
:1056C8006FF0150823E45B88B3F5007F7FF69FAC85
:1056D8003D4B226DBB62002387F82C3004F1500348
:1056E8009342FB6060D105F10C0A50462FF04DF94A
:1056F800B7F82A80E38D984528BF9846404503D2DD
:1057080050462FF042F9804697F8282007F12801E3
:105718005046424528BF42462FF015F9B8F1050F0B
:1057280094BFA8EB0808A8F10508B8F1000F3FF4EA
:10573800CCACD4F850B0FB689B453FF4C6ACBBF189
:10574800000F3FF4C2AC9BF815300F2B15D19BF816
:1057580014205046DBF81010424528BF42462FF06F
:10576800F2F89BF81430434594BFA8EB0308A8EB64
:105778000808B8F1000F3FF4A8AC636D5B453FF42F
:10578800A4ACDBF800B0DAE7537D0F2B08D1137D0A
:10579800798D0B447B8597F82C30013387F82C30B2
:1057A800636D93429FD01268002AEDD19BE700BF3A
:1057B800DC530590B898049000FF02000003020033
:1057C800A454059002540590050F050094F8343050
:1057D80094F83CA0002B3FF45AACE38D012B7FF4E6
:1057E80016AC05F10C0840462FF0CFF8E38D98422F
:1057F800FFF4DAAD5146404629E794F8283003F023
:105808001F03012B7FF443AC20462FF077F90028C3
:105818003FF43DACA38D4268FF2B3FF6F8AB1279FD
:105828009A42FFF4F4AB0F2B3FF6F1AB234493F805
:105838003EA0D2E76B7E59077FF559AC2946204632
:1058480000F0FAFA8046FFF750BB5A077FF591AB94
:1058580080297FF48EAB2846FFF796FA256B012D39
:1058680040D194F83D30002B3FF43FAB94F82930F9
:10587800052B0CD1618DA069C9B22FF00FF98046B4
:1058880028B1638D234A294623482EF092FE94F8C6
:105898002930032B11D1638D022B0ED1A18D00224B
:1058A800A0690D0A29462FF0D6F8804628B11B4A70
:1058B8002B46012118482EF07CFE002384F83D3049
:1058C800FFF713BB5B077FF554AB0029C0D1236BEF
:1058D800012B3FF41CAB124A02210F482FF0B9F8F4
:1058E800FFF715BB0F4A02210B482FF0B2F8FFF75C
:1058F800FCBAE38D002B3FF444AB19F10C0118BF3F
:105908000121C9012FF04EFD002380462363FFF7D4
:10591800ECBA00BF97530590B89804904554059089
:10592800245405906354059030B589B000220023B3
:1059380000241E491E480094CDE906236FF0070392
:105948004FF48062CDE90334CDE90144194B05F0E9
:10595800A3FE1949164831F0A2FC184B18498B428E
:1059680007D3184B002018498B4210D3002009B0E8
:1059780030BD03F11402BFF35B8F52E8000F42E819
:105988000045002DF9D11833BFF35B8FE7E703F12A
:105998001402BFF35B8F52E8004F42E80005002D68
:1059A800F9D11833BFF35B8FDEE700BF4030002426
:1059B800A0190024295A0090BE5405902C0D0024EB
:1059C800440D0024440D0024440D002438B50D4630
:1059D8002FF094F830B9104A01211048BDE838403A
:1059E8002EF0DEBDC46804B938BD2B78032B07D070
:1059F800052B0CD0022B08D1606883689B6902E0F4
:105A0800606883685B6903B198472468EBE760685E
:105A18008368DB69F7E700BFC3540590C898049012
:105A28002DE9F04784B0DFF80482102600AF4FF06C
:105A3800FF334FF0FF32391D404605F021FAFB686D
:105A48001B69D3F89C40236A73B1EFF3118386F383
:105A58001288BFF36F8FD4F820A0BAF1000F1BD1C2
:105A680083F31188BFF36F8F3B79062BDFD0072BA9
:105A7800DDD801A252F823F0175B00900B5B009071
:105A88003F5B00901D5B0090755B0090615B009030
:105A9800375A0090255C0090616ADAF800208A4540
:105AA800226208BF626283F31188BFF36F8F9AF88E
:105AB80018305146DAF81E2020465D061ED1FFF741
:105AC800FFF905460028BED0E9468AB09AF8183092
:105AD8006A465749C2E9073A0523C2E9051042F860
:105AE800103F00234FF421515248FDF74DFD2A463F
:105AF80007212046CD462FF04FF9A4E72FF037F8BD
:105B0800DFE70022012120462FF046F98FE7002227
:105B18001146F8E794F8703043F0040384F87030C5
:105B280094F83430022B03D1391D2046FFF74EFF7D
:105B380000220321E7E794F870306FF3820384F8BA
:105B4800703094F83430022B03D1391D2046FFF70A
:105B58003DFF00220221D6E794F83430022B7FF46F
:105B680066AF391D2046FFF731FF60E794F87030C3
:105B7800D4F818906FF3820384F87030D9F8103095
:105B8800D9F808A0BFF35B8FD3F8A030BFF35B8FC1
:105B98009A071BD5DAF83C3048469847DAF824309B
:105BA8000021484698470546DAF840304846984765
:105BB8007DB1214A01211F482EF0F2FC0022042168
:105BC80020462FF0E9F82A4607219CE74FF0FF35D9
:105BD800EFE72946204600F037F8054608B1174A8E
:105BE800E8E7802120462FF0CAF820B1144A0121A5
:105BF80010482EF0D5FCA0692FF087FC831E0022E8
:105C08000421584284F83420584194F8703023F025
:105C1800680343EA401384F8703074E7094A0121A5
:105C280004482EF0BDFCBA6806216CE7680C002415
:105C3800F2540590C89804901C5505904A55059053
:105C480076550590935505902DE9F04105460E4689
:105C58002EF0ACFE804695F83C303BB328462EF03B
:105C68004DFF0746F8B1014628462EF0A0FF102246
:105C78000446002105F13E0043F03AFA002385F876
:105C88003C30FF6847B98CB1194A012119482EF0F8
:105C980087FC2046BDE8F081786883685B6A03B1B9
:105CA80098473F68EEE76FF03C04EDE71EB985F8CA
:105CB8003C600024EDE73246414628462EF00AFFB4
:105CC800074690B1024628462EF09BFF044600285E
:105CD800DFD185F83C60FC68002CEAD060688368F6
:105CE8001B6A03B198472468F6E76FF03C04D0E7D5
:105CF800B7550590B098049001F07F0311F0800F1C
:105D080070B518BF1033012504469D4090F8343013
:105D1800022B06D00C4A01210C482EF041FC002031
:105D280070BD90F83C602EF041FE01462046324698
:105D38002EF0D0FE0028F2D0C0680028EFD083688B
:105D48001D42EDD10068F8E7DE550590C098049033
:105D58002DE9F04F83B00E468146904600AF4C685F
:105D68007B6097F830303B602EF020FEA368014638
:105D78001B6B33B96FF0150420460C37BD46BDE8E0
:105D8800F08F204698470028F4D0051F002406F11C
:105D98000C0A55F8041F09B10B782BB9002C0CBF5D
:105DA8006FF03C040024E7E74B78042B0ED1002C5D
:105DB8003CD18B787A689342EBD1CB783A6893429E
:105DC800E7D10B79002BD7D00124E2E7052BE0D1EE
:105DD800002CDED0B8F1010F91F802B009D0B8F16B
:105DE800020FF1D152465946D9F818002EF096FF05
:105DF80004E05246D9F818002EF075FF0446002832
:105E0800E2D06D468AB0F3686A4609495062C2E931
:105E180007B30623C2E9051842F8103F00234FF4E0
:105E280041510448FDF7B0FBAD46A5E70024A3E7C0
:105E38000E560590E89804902DE9F0410B7E054632
:105E48000C465E0638D119062DD52EF0B4FD40B1AA
:105E58001B4801211B4A2EF0A3FB4FF0FF30BDE881
:105E6800F0812846D5F87480268AEF8D2EF09EFDA5
:105E7800F8B1421E534253419B01228A9AB1BE4255
:105E88003246E98D28BF3A4691420CD9B2FBF3F16C
:105E980003FB11223AB994F91830002BBEBF637E78
:105EA80043F0080363762146A869BDE8F0412FF066
:105EB800D5BA98F80730E0E76FF01500CFE700BFD4
:105EC800E09804904A56059070B5064680690C46DD
:105ED8002FF068FA054638B10A4A234602210A48D3
:105EE8002EF067FB284670BD14F0800F4FF00102BA
:105EF800B36B1CBF24F080041034A2401A43B26371
:105F0800F0E700BF5E560590E098049070B505462E
:105F180080690E462FF071FA044638B1064A3346B6
:105F2800022106482EF045FB204670BD314605F19A
:105F380038002EF0CAFEF7E775560590E0980490F1
:105F480070B50646EFF31181102282F31288BFF371
:105F58006F8F1D4C236881F31188BFF36F8F5B68C7
:105F680093F87030DB0705D40A220023BDE870409F
:105F780005F026BBEFF3118382F31288BFF36F8F0E
:105F8800256865B983F31188BFF36F8F2368D3B190
:105F9800304600220023BDE8704005F0DDBA616894
:105FA8002A688D42226008BF626083F31188BFF3BC
:105FB8006F8F686805F10801C36998472946034847
:105FC80030F0A3FFE2E770BD18200024F40B002492
:105FD80030B585B00546002316486C4684E80600AF
:105FE800002203A904F0AEFE0246E8B9039B94E838
:105FF80003005D60083383E80300EFF3118010238A
:1060080083F31288BFF36F8F039B1A600A4A5168A3
:1060180061B9C2E9003380F31188BFF36F8F0022A2
:106028000023064805F098FA05B030BD0B605360B0
:10603800F1E700BFF40B002418200024000000241E
:10604800D3B50026002704460648CDE900672EF0A0
:1060580055FC20B1230604765CBF0023038202B0FE
:10606800D0BD00BFD40C00242DE9F04383B0002339
:106078001D4C4FF00108056902AF1C4E05F12409BB
:1060880028602B7785F82030B442234601D30020BE
:1060980019E095F820201034CAB16C4688B01B6806
:1060A80002AA1349C2E905134FF400739383114BF5
:1060B80042F8103F104800234FF4E251FDF764FA0C
:1060C8006FF00B00A5460437BD46BDE8F08385F8A0
:1060D8002080484654F8043C009354F8101C54E9B6
:1060E80003232EF0C5FFCFE7C4CE0590C4CE05909C
:1060F8009F56059003000001F89804901FB5CDE95C
:10610800010103924FF0FF324FF0FF3301A903481A
:1061180030F05EFF002005B05DF804FB380C002469
:1061280013B514464A780369FE2A14D14A8892B9ED
:10613800CA8882B193F820300BB1013BDBB201224F
:106148000DF1070104F10C008DF807302EF0FBFB70
:10615800002002B010BD034B6FF08502FEF784FAF1
:106168001A50F5E70C0000001FB500230190CDE997
:1061780002334FF0FF324FF0FF3301A9024830F0ED
:1061880027FF05B05DF804FB380C002408B54B78F0
:10619800FF2B07D14B882BB9CB881BB9FFF7E4FF3E
:1061A800002008BD034B6FF08502FEF75DFA1A5018
:1061B800F6E700BF0C0000002DE9F0410368044633
:1061C80017460E461B695B6893F80B804046FFF73D
:1061D80037FFD4F87B2005460146D21B2068C4F857
:1061E8007B202EF0B1FD88B10B4A434601210B48B4
:1061F8002EF0DFF9314620462EF080FE2846FEF7C5
:10620800C3FD2046BDE8F0412EF034BEA37F013324
:10621800A377BDE8F08100BFB6560590F8980490C2
:106228002DE9F8430368054630274FF024081B6919
:106238005B689E7CEB7F012B20D82B68D3F81090ED
:1062480099F8614017FB04844C4420462EF036FF31
:10625800B0F5007F636A044628BF4FF4007499F8CC
:106268001F2024F03F047BBB3AB1041BB4F5007F28
:1062780028BF4FF4007424F03F040CB9BDE8F8833C
:1062880028462EF097FD2246014681463046FFF704
:10629800D7FE0446014628682EF056FD80B1134A01
:1062A8003346012112482EF084F92046FEF76CFD92
:1062B800494628462EF022FEBDE8F8432EF0DABD06
:1062C800EB7F0133EB77B5E7B4FBF3F45C43002ACB
:1062D800D3D0001BB0F5007F28BF4FF4007020F02A
:1062E8003F00B0FBF3F000FB03F4C6E7B656059099
:1062F800F89804902DE9F04FDFF8EC9287B04FF052
:10630800FF324FF0FF3303A9B84804F0B9FDDDF8B8
:106318000C80049DD8F81040002D40F0978004F1BF
:106328002406257794F820309D42C0F2898004F134
:106338001803BFF35B8F53E8002F22F0020243E8F3
:1063480000210029F7D1BFF35B8FBFF35B8F53E8C0
:10635800001F21F0040143E80012002AF7D1BFF31F
:106368005B8FBFF35B8FA369BFF35B8FDB07C6D57A
:10637800237F022B00F07781032B00F0708143BB51
:10638800DDF80CB0DBF81050EB7F13BB6B682846C8
:1063980093F812802EF00EFD402201460646404634
:1063A800FFF74EFE0746014658462EF0CDFC002862
:1063B80000F051818E4A434601218E482EF0F9F8AB
:1063C8003846FEF7E1FC314628462EF097FD2EF0C0
:1063D80051FDA37F002B92D1237F012B40F06881D0
:1063E800302394F8615004F1630694F8621003FBBB
:1063F80005453046243500F04FFA314602462369F8
:10640800284600F067FA0646C4F8840028462EF0AD
:106418004BFE804628462EF04CFE074628462EF0B6
:106428004DFEE26D3044002A40F02681002840F0FD
:106438001E8128462EF069FE003818BF012017E19A
:106448003046013530362EF026FE6BE7059AD8F82F
:1064580004B02B7E3AB3298A71326648009107BF8F
:106468000221654A0121654A2EF0ADF8D8F81020BE
:106478002B7E5268917C994240F0DF80E37F5A1E60
:10648800E2776A680AB1023BE377696920462EF031
:1064980035FD6B6813B159692EF030FD2946584611
:1064A8002EF06AFC5DE76168887C984240F0918034
:1064B800227FEF68B5F810A0002A48D1BAF11F0F63
:1064C80041D13B684B453ED1394604F1540307F1AD
:1064D8001C0251F8040B914243F8040BF9D10A88C5
:1064E8001A808A7842219A705523E26D84F87330B5
:1064F8005323C4F87B2084F8743084F87630A36D75
:1065080084F87510C4F877300023C4F8803094F804
:1065180060309A060FD194F8612094F820309A429E
:1065280009D294F86230013B0F2B04D8012384F878
:106538007F3023779AE720682EF050FC022384F8F6
:106548007F300423F5E720462EF094FC8EE7032ADB
:106558008CD1302294F8616002FB0646D4F8802082
:1065680052442436C4F88020BAF1000F15D03046C2
:106578002EF0A4FD88B13946524630462EF0B1FDC2
:10658800074628B91E4A534602211A482EF011F828
:10659800D4F87B30DB1BC4F87B30D4F88020E36D63
:1065A8009A420DD230462EF089FD00287FF45EAF66
:1065B800D4F88020E36D9A4202D220682EF014FCB1
:1065C80030462EF0A2FD003818BF012084F87F0065
:1065D800B7E7C97A99427FF449AF237F298A052B07
:1065E80010D1227742E700BF55534243380C0024AC
:1065F800B6560590F8980490DB560590FF5605901E
:1066080020570590022B7FF431AFD4F880302068F2
:106618000B4494F86160C4F880302EF0EBFB00283E
:106628007FF424AFD4F87B3013B120682EF0D6FB6A
:10663800302303FB06402430C3E7D27A9A427FF422
:1066480024AFA37F5A1EA2776A68002A3FF41DAFC1
:10665800023BA37719E7EB7F0133EB77B9E62046D6
:10666800FFF7DEFDB5E620462EF058FCB1E6022025
:1066780084F87F0004231AE094F9601040B90029D7
:10668800206802DA2EF0AAFBD3E62EF0ADFBD0E6A6
:10669800002914DA904202D8B8F1000F06D1206818
:1066A8002EF09CFB022384F87F30E3E70223237754
:1066B800237F022B0CD120462EF030FC1FE690429F
:1066C80000D81FB920682EF08FFBEBE70323EEE715
:1066D800032B03D12046FFF7A3FD10E6042B7FF41C
:1066E8000EAEA37F2BB11E4A01211E482DF058FF84
:1066F80005E6236820461B695B68DF7A2EF05AFBA3
:1067080004F173030546024604F17F0153F8040BB4
:106718008B4242F8040BF9D11B782946384613708E
:106728000D22FFF78DFC0646014620682EF00CFB73
:1067380078B10D4A3B4601210A482DF03AFF304610
:10674800FEF722FB294620462EF0D8FB2EF092FBBE
:10675800D5E5A37F0133A37705232377CFE500BFD2
:1067680046570590F8980490B6560590802938B594
:106778000D46144621D083290DD019BB8023032050
:1067880011715371832393710023E0700430657095
:106798002370A37038BD02231371012353710023A2
:1067A80093710A23D37108224168A01842F0D7FCDC
:1067B800064B0E201B882382E6E7044B02201B8829
:1067C8009380E1E76FF08500E4E700BFE2B705904A
:1067D8002DE9F04187690446D0F82480BA4228BFE1
:1067E8003A46B2FBF8F5C2692B4600682EF01DF850
:1067F800064648B9B7FBF8F7AF4207D0E3692B4420
:10680800E361606A684312E0002501260022052141
:106818002068FDF7D5F960B1094A012109482DF032
:10682800BFFEE3692B44E361074B0020A362BDE888
:10683800F081E3692B44E361002EF5D1E1E700BF65
:1068480067570590F89804900203000C81420B46A4
:1068580007B509D30D4A02210D482DF0AAFE6FF0A5
:10686800150003B05DF804FB6AB101391144814297
:1068780001D28B4207D90221009305481346054AE5
:106888002DF0A1FEEBE70020EBE700BF7E57059057
:10689800F8980490955705900C290346084616D198
:1068A8001B78252B12D009D8122B10D8084A42FA87
:1068B80003F313F0010F08BF0620704703F0FD0231
:1068C800282A03D05A2B08BF0A2070470A2070478D
:1068D800F6FFFBFF2DE9F0411E4690F82C30062A02
:1068E80086B023F00C030446884680F82C304FF01D
:1068F80000038361C0E904330B7840F00C81D3B9FD
:106908004D7915F0040540F0168290F82C309B075D
:106918000AD402234FF468521D4684F829500025F2
:1069280084F8283062853AE02EF026FB0028F0D162
:106938002B462A46F1E7032B35D14F7917F0040788
:1069480040F0F98190F82C308DF8077043F004037B
:106958008DF808708DF8097080F82C3070230D7947
:1069680001A9ADF8043090F82930122D8DF80A707D
:1069780003F00F0328BF122503978DF806300A236A
:106988002A46ADF812708DF80B30438D3046ADF8BD
:1069980014705BBAADF8103042F082FBA76228464B
:1069A80006B0BDE8F081122B4BD14B795F0700F19F
:1069B800C28190F82C3043F0040380F82C304B78D7
:1069C80013F0020723D113F0010F8B7819D0B1F817
:1069D8000350324619466DBAFFF7C8FEADB285427C
:1069E80006DAB8F8030040BA80B200231A4613E06A
:1069F800324698F802102046FFF7B8FE0028F4DA6D
:106A080005E083B1AB4A0221AB482DF0D2FD022349
:106A180005274FF410520020054684F8283084F8E2
:106A280029706285BBE7B1F8035031462EF0D7FADA
:106A38006DBAADB28542D4DB314620462EF0CFFA8E
:106A4800DCE71A2B27D14D7915F0040540F0738146
:106A580090F82C3043F0040380F82C308B783F2BCF
:106A680014D1CF7897B90D79032301A93046042DA5
:106A7800019328BF04252A4642F012FB3A463B46BA
:106A880084F8282084F82970638588E7022205277E
:106A98004FF41053F4E71B2B23D14D7915F004055F
:106AA80040F04981097990F82C200809C2F3400385
:106AB8000AD18E0708D5C80711D402F00302032AA9
:106AC80000F03E81002301E0002BF6D094F82C2042
:106AD80063F3410284F82C2000231A461DE70123A2
:106AE800F4E71E2B40F022814D7915F0040540F0A3
:106AF80022810B7913F0030306D0012BECD190F817
:106B08002C3043F0010303E090F82C3065F30003C8
:106B180084F82C30E0E70A2A40F00881232B40D182
:106B28004B7A13F0040340F0068190F82C20ADF85E
:106B3800043042F004028DF80630082380F82C2037
:106B48008DF807302EF018FA002801A93046ABBF9F
:106B5800236A4FF0FF3302220322A8BF1BBA8DF825
:106B68000C200293636A1BBAC3F307228DF80D3019
:106B7800C3F307438DF80E208DF80F3094F82C30AE
:106B880043F0040384F82C30B8F807506DBAADB25E
:106B98000C2D28BF0C252A4642F082FA0023A36256
:106BA800FDE6252B2ED14F7A17F0040740F0C3805D
:106BB80090F82C3043F00403990780F82C3006D461
:106BC80002274FF46853002584F828705AE72EF0FE
:106BD800D3F90028F4D1236A93B1013B1ABA1B06F2
:106BE80022F07F4294F82C001A43616A002340F097
:106BF8000400082509BA84F82C0032607160E3E7C4
:106C08001A46EFE7282B2BD14D7A15F0040540F0F2
:106C1800928090F82C30D1F8027043F00403B1F858
:106C280007609A0780F82C307FF573AE2EF0A4F930
:106C380000287FF46EAE76BA3FBA206AB6B23946FB
:106C48003246FFF703FE20B1022305254FF4045214
:106C580063E61A4BE7612361636A7343A36167E6DE
:106C68002A2B2FD14D7A15F0040564D190F82C30D9
:106C7800D1F8027043F00803B1F8076080F82C30AF
:106C88009B077FF546AE2EF077F900287FF441AEDA
:106C980076BA3FBA206AB6B239463246FFF7D6FD11
:106CA8000028D1D1064BE7616361636A7343A3612E
:106CB80012E700BFBF570590F89804904B50039017
:106CC800D96700905A2B31D14D7A15F0040532D18D
:106CD80090F82C3043F0040380F82C308B783F2B4D
:106CE80019D1CF78E7B94FF4C0633046CDE9013503
:106CF800B1F8075001A96DBAADB2082D28BF082513
:106D08002A4642F0CDF900231A4684F8283084F840
:106D18002970628543E6022305274FF41052F4E7F1
:106D2800022305274FF410520025EEE7074A0121F8
:106D380007482DF03EFC022305254FF41052ECE5E0
:106D48000223052545F20232E7E500BFDC5705902E
:106D5800F898049007B5094A6B4692E8030083E85F
:106D6800030007488268126822B11946904703B0A9
:106D78005DF804FB6FF05700F9E700BF189904901D
:106D88005494049000F01F0201215F2801FA02F2D6
:106D980008B5034605D90C480C4A2DF00AFC00201A
:106DA80008BD1F284FF0B04106D8D1F888309A4363
:106DB8000CBF01200020F3E73F2802D8D1F8983013
:106DC800F5E7D1F8A830F2E718980490F75705903E
:106DD80000F01F0201215F2801FA02F208B50346FC
:106DE80006D90B480B4A2DF0E4FB6FF0150008BDDF
:106DF8001F284FF0B04103D8C1F888200020F6E7DB
:106E08003F2802D8C1F89820F8E7C1F8A820F5E78C
:106E180018980490F7570590044B03EB40000023A3
:106E2800013320F8022B9942FADC70475C060024F3
:106E38002DE9F041054600260F4F4FF00108F4B246
:106E48006B78A34201D8BDE8F0812B781C4420461A
:106E5800FFF798FF68B12046FFF7BAFF57F83430BC
:106E68003BB107EBC40204F01F04516808FA04F0B0
:106E780098470136E3E700BF20200024034680B18D
:106E8800B0FA80F2C2F11F02D2B2074931F91200FA
:106E98004FF0B042D2F880100B43C2F88030FDF7B3
:106EA8001BBBFF22F1E700BF5C06002430B5B0B180
:106EB800B0FA80F3C3F11F03DBB20B4850F833403C
:106EC8008C4204D100EBC3056D68954205D044B9E6
:106ED80040F8331000EBC3004260002030BDFF23B0
:106EE800EBE76FF00F00F9E72020002460B1B0FA5B
:106EF80080F3C3F11F03DBB2044A002142F83310C8
:106F080002EBC30251607047FF23F5E720200024FD
:106F180000F003020F23043292009340094A43EA27
:106F2800900000F00303023352F82320030C93FA75
:106F3800A3F3B3FA83F302EA104003F01F03D84027
:106F4800704700BF000400582DE9F0470546894600
:106F580090461F46D0F808A02EF0D6F90446D0B1C6
:106F6800067FF3070AD590F8203018480121184AFF
:106F78002DF01FFB6FF07700BDE8F0873B464246D7
:106F880049462EF07BF948B994F82030114A01217E
:106F98000E482DF00EFB6FF01200EDE79DF8203043
:106FA80026F0060684F8218021466784284684F85E
:106FB80024302677DAF818309847B0FA80F3227F21
:106FC8005B0963F300022277D6E700BFA898049014
:106FD800455805905F58059070B5054686682EF0AF
:106FE80093F90446D8B1037FDB0709D490F8203021
:106FF8000C4801210C4A2DF0DCFA6FF0770070BDC7
:107008000146F3692846984738B1237F03F0010306
:10701800227F63F300022277F1E70346F8E76FF077
:107028001200ECE7A898049081580590064B1B695C
:1070380003F03803102B05D0182B044818BF002084
:10704800400870470248FBE70044025800389C1C7F
:1070580040787D01354B10B518680B88C3F30B03D6
:10706800132B38D813B96FF0850033E0013B122B8E
:10707800F9D801A454F823F00B710090CD7000905A
:107088006F700090217100906F7000906F70009089
:107098006F7000901171009015710090157100903B
:1070A8006F7000906F7000906F7000901171009079
:1070B800197100901D7100906F700090037100901D
:1070C800037100904FF4004010600B68B3F5805FC7
:1070D80024D2002010BDD42B0FD003F62873C3F39D
:1070E8000B031C2BBFD8012404FA03F3104C2342D2
:1070F80005D140F211142342B5D04008E4E78008D6
:10710800E2E7FFF793FFDFE70A48DDE70A48DBE736
:107118000A48D9E70A48D7E70A48D5E7C3F313333B
:107128000133B0FBF3F01060D3E700BFB0030024D5
:107138000010111100389C1C001C4E0E006CDC0263
:10714800C9F6930040787D0137B5984CD4F8E03003
:1071580043F00073C4F8E030D4F8E03003F0007373
:107168000193019B236843F480232360236843F43D
:107178008033236023689803FCD5FBF7E9FE236F6F
:107188008A4A23F018032367236F43F00103236718
:10719800136F9907FCD5FBF7F9FE854B9A6942F402
:1071A80040429A619A699204FCD5804B1A6902F0B0
:1071B8003802182A16D11A68550706D41A6842F0F8
:1071C80001021A601A685407FCD5784B1A6922F034
:1071D80007021A611A6912F0380FFBD19A6922F076
:1071E8000F029A61714B1A6822F080721A601A684D
:1071F80022F080621A601A6822F080521A609A6A35
:1072080022F0030242F002029A629A6A22F47C7225
:1072180042F050029A62DA6A22F00C0242F0080246
:10722800DA62DA6A22F00202DA621A6B22F4FF7278
:1072380022F0010242F0BF021A63DA6A22F0010268
:10724800DA621A6B22F47E4242F400721A63DA6A36
:1072580042F48032DA621A6B22F4FE0242F44032BF
:107268001A63DA6A42F40032DA621A6B22F0FE42DA
:1072780042F040721A63DA6A42F48022DA621A68CB
:1072880042F080721A601A689001FCD59A6A474CDD
:1072980022F07C7242F4A0029A62DA6A22F4406216
:1072A80042F40062DA62DA6A22F40072DA621A6C74
:1072B80022F4FF7222F0010242F0BF021A64DA6A75
:1072C80022F48072DA621A6C22F47E4242F400726E
:1072D8001A64DA6A42F48002DA621A6C22F4FE0254
:1072E80042F498121A64DA6A42F40002DA621A6CFA
:1072F80022F0FE4242F0C4421A64DA6A42F0807216
:10730800DA621A6842F080521A6023689900FCD544
:10731800FFF78CFE05462748854201D202F070FA35
:10732800A369224A23F47063A361A36923F00F03BE
:1073380043F00803A361E36923F0700343F04003BB
:10734800E361E36923F4E06343F48063E361A369E1
:1073580023F0700343F04003A361236A23F0700312
:1073680043F040032362236923F0070343F0030338
:107378002361136903F03803182BFAD10D488542AD
:1073880001D302F03DFA0A4B9A6942F440429A61ED
:107398009A699204FCD5054A0020136923F4004336
:1073A8001361054B054A1A6003B030BD004402580A
:1073B80000480258001C4E0EB003002400389C1CE4
:1073C800132808D8054BC34013F0010F14BF002041
:1073D8006FF0850070476FF08500704716C70D0085
:1073E80008B507482FF0FBFC38B10648FDF788FBC5
:1073F8000448FBF765FD002008BD6FF01200FBE7AD
:1074080030960490117400900A2838B50446074D48
:1074180004D1AB680D2128465B689847AB68E1B298
:1074280002485B689847204638BD00BF30960490F4
:1074380098B5406800AF046B0369DCB133BB2046E4
:107448002FF0CDFC034640BB21686C4688B06A46E5
:107458001548C2E905014FF400719183134942F8B8
:10746800101F13484FF4E251FCF78EF86FF012002A
:10747800A54602E01BB96FF05700BD4698BD2146EE
:1074880010302EF00DF900EAE070F6E70021103018
:107498002EF006F90028D2DAEFE7A3681B68002B64
:1074A800E9D020469847E8E7AD5805900300000169
:1074B8001098049098B5406800AF046B0369DCB17C
:1074C80033BB20462FF08BFC034640BB21686C463B
:1074D80088B06A461548C2E905014FF400719183E6
:1074E800134942F8101F13484FF4E251FCF74CF8C7
:1074F8006FF01200A54602E01BB96FF05700BD46B9
:1075080098BD012110302EF0CBF800EAE070F6E7C4
:10751800012110302EF0C4F80028D2DAEFE7A36872
:107528005B68002BE9D020469847E8E7AD580590FE
:1075380003000001109804902DE9F8431C46D0F888
:1075480004809B88D8F800500B440669089FAB421A
:10755800D6F8B80005D8E388D8F804C013446345C2
:1075680008D919480121194A2DF01AF86FF01500A9
:10757800BDE8F88396F8A93005FB02114FF0000921
:1075880001FB0305E2881FFA89F39A4201D800201B
:10759800EEE7A388294696F8A92038465A4341F0D1
:1075A8007FFDA18896F8A9305943384609F10109A9
:1075B800FDF7B8F896F8A930D8F8002002FB035573
:1075C800228903FB0277DDE710980490C9580590DB
:1075D8002DE9F843D0F804801D46B3F804E00469A7
:1075E8000EEB0103D8F80000089F834205D8EE8807
:1075F800D8F804C09319634508D930480121304AA6
:107608002CF0CEFF6FF01500BDE8F88352EA0109AF
:1076180094F8A93029D1704527D1B44525D12E89B0
:10762800864222D10CFB06F1384604F1BC055943C9
:10763800FDF778F8284603F0DFFD23680122C4F837
:10764800B470DA632268536B43F0010353634FF05D
:10765800FF324FF0FF33284603F0A8FD2268536B32
:1076680023F0010353630020CEE75843D4F8AC60FD
:107678004B434FF0000902FB00321644EA881FFA18
:1076880089F39A42EFD9AB88394694F8A920304655
:107698005A4341F005FDA98894F8A930594330466A
:1076A80009F10109FDF73EF894F8A930D8F800204F
:1076B80002FB03662A8903FB0277DFE71098049030
:1076C800C95805902DE9F743476806460569BB6820
:1076D80083B14FF4D01107F108002DF0C6FF041E46
:1076E80008DA3D4A01213D482CF05AFF204603B0F4
:1076F800BDE8F0833B694BB14FF4B01107F11000BE
:107708002DF0B3FF041E01DA354AEBE701AA002188
:10771800B86A2EF0F2FB041E07DB019B00221979E0
:10772800186801F055FA041E01DA2E4ADAE7DFF884
:10773800B880B969D8F80890D9F800302BB140461C
:107748009847041E04DA294ACCE76FF05704FAE791
:10775800FB69012B0ED9B969D9F81830083133B152
:10776800002240469847041E04DA214ABAE76FF01F
:107778005704FAE7D7E908018368DB6803B198473B
:107788004FF40473A5F8A8300122002105F1BC00CC
:107798002FF004FDFB6A30469847164A28461368BE
:1077A80023F00D0313602EF013FE044600289DD12C
:1077B800024605F1380128462EF068FE04460028E6
:1077C80094D12A68D2F8043123F00103C2F80431B5
:1077D800094B18648AE700BFF15805901098049087
:1077E800255905905C590590549404907659059054
:1077F8009D5905900040005200100050064A11683B
:107808000B6823F004030B60044B50681968836805
:107818005B6803B11847704734020024A0020024B3
:10782800094B10B5D3E90040084B196883681B68F9
:1078380003B19847236843F004032360236843F0A7
:107848000803236010BD00BF34020024A0020024F6
:1078580008B5EFF31181102383F31288BFF36F8FFC
:10786800084B012093F8482083F8480081F31188D9
:10787800BFF36F8F22B9FFF7D3FF5020FCF72CFE20
:10788800002008BD34020024F8B51646837890F825
:1078980003C0EFF31182102484F31288BFF36F8FB3
:1078A800077890F801E0DB1B3C4603EA0C039E4294
:1078B80088BF9EB2BD190CEA0505057082F31188D0
:1078C800BFF36F8F8A198A421AD177450CD1EFF32B
:1078D8001182102181F31288BFF36F8F01784170F4
:1078E80082F31188BFF36F8F02799B1B9A4205D3ED
:1078F8002FF0CFFC60B1084803F0BEFD3046F8BD5C
:10790800051901346D7904EA0C0401F8015BDAE722
:10791800FFF79EFFF2E700BF6C0200242DE9F84351
:10792800134F0D46144607F1560807F1180914B904
:107938002046BDE8F8834FF0FF324FF0FF3338465A
:1079480003F034FC224629464046FFF79DFF0646D1
:1079580030B94FF0FF324FF0FF33484603F026FCB2
:10796800A41B3846354403F0E5FBA4B2DFE700BFAB
:107978003C02002438B543680469224860601968ED
:1079880083681B6803B19847012204F10800114677
:107998002FF004FC0122002104F1200000252FF023
:1079A800FDFB04F1380018492FF047FC07232A464D
:1079B800294684F861300423502084F85E5084F806
:1079C80062300F2384F85F5084F84C300C2384F81D
:1079D800605084F84D3084F8495084F84A5084F84F
:1079E8004B502CF04CFF094B1B681A6842F00402FC
:1079F8001A601A6842F008021A60FFF729FF284641
:107A080038BD00BF54940490B55703903402002445
:107A1800164B014610B51A68EFF31184102383F34F
:107A28001288BFF36F8F53685B0605D45368D80775
:107A380013D46FF00A000BE06FF0400353600C237F
:107A4800013B9068FCD153685B06EFD56FF00400EA
:107A580084F31188BFF36F8F10BD506810F0400099
:107A6800F4D193680B60002BF2D1E2E734020024D2
:107A78002DE9F347D8070F46144605D42E48FFF7DB
:107A880003FF02B0BDE8F087002A37D0EFF3118575
:107A9800102383F31288BFF36F8F5020FCF73EFD4D
:107AA80006465020FCF726FD85F31188BFF36F8F3B
:107AB800DFF88880FFF7B4FED8F800305A6851071D
:107AC80014D45B685A0611D4DFF874904FF4803AE6
:107AD8002546C9F888A1D8F800305B68DB070FD4C1
:107AE800BFF34F8F20BF40BF20BFF4E7002401A899
:107AF800FFF78EFFE6B15020FCF7EEFC2046C0E70A
:107B080001A8FFF785FF0028C9F888A1E3DB6A1EF2
:107B1800291F019B17FA82F289B2013D02F8013947
:107B28001B0AADB2002DE5D08D42F6D10193D2E704
:107B3800FFF764FEE2E700BF7D0200243402002460
:107B480000E100E02DE9F74301A8FFF761FF0028F5
:107B580044DB284C0021019A042794F84B308846CE
:107B680094F84CC0084694F84AE0A3EB0E055FFA77
:107B780082F93CEA05051ED194F8600094F85F602C
:107B880094F86150861B35EA06062AD109B184F8B3
:107B98004B30B8F1000F00D001925020FCF7AAFC3E
:107BA800FFF72CFE002384F84830134803B0BDE8E3
:107BB800F04303F0BFBAE118013381F84E900CEAA4
:107BC80003030121013F4FEA12224FF00108CCD1F3
:107BD80009B184F84B3001920028E6D103B0BDE822
:107BE800F08326180130054086F86390012084F858
:107BF8006050E7E73402002454020024C3780F2BB6
:107C080014D9C96B0B480B0E00EA911013708B0244
:107C1800090603F47C0301F0FE41034310680B439B
:107C28000549014000200B43136070476FF0850041
:107C3800704700BF00FF0300FF0000800048704746
:107C4800589C0490F0B5154602681E468FB013681C
:107C580004460F4602A823F0400300211360302297
:107C680041F046FA5A23082141F288322046CDE9EC
:107C780000374FF4005303934FF48073CDE9051395
:107C88004FF48063694607934FF08073CDE9093656
:107C98002EF03FFD034668B10D4A0E4801212DF034
:107CA8008CFE6FF004002268136843F040031360F1
:107CB8000FB0F0BD41F28832294620462EF0B0FDC3
:107CC800034608B1044AE8E7C4F89000EBE700BFB0
:107CD800035A059028980490275A059038B58B6266
:107CE800002304461546C0F890302EF056FD034692
:107CF80038B10D4A0D4801212DF05FFE6FF00400E8
:107D080038BD294620462EF0ECFD034608B1084A46
:107D1800F0E74FF0FF324FF0FF3304F1640003F057
:107D280045FAD4F89000EBE73F5A0590289804905C
:107D3800635A0590002310B5C0F8903004462EF021
:107D48002CFD034638B109480121094A2DF035FEBA
:107D58006FF0040010BD4FF0FF324FF0FF3304F115
:107D6800640003F023FAD4F89000F3E7289804900D
:107D78003F5A059038B58B62002304461546C0F873
:107D880090302EF00AFD034638B10D4A0D48012106
:107D98002DF013FE6FF0040038BD294620462EF062
:107DA800D8FD034608B1084AF0E74FF0FF324FF01C
:107DB800FF3304F1640003F0F9F9D4F89000EBE71D
:107DC8003F5A059028980490635A05902DE9F04F82
:107DD8000D1E91B0064614467CDBD0F80490AA1814
:107DE8004FEAE5734FF00001D9F80C0043F10003A6
:107DF800904271EB03036DD3002C39D0382202A8CE
:107E0800D6F8108041F074F94FF480724FF4806313
:107E1800DFF8C8A04FF0FF3B4046CDE9082398F8AB
:107E2800BF3013F0010F0CBF4FF400534FF4405311
:107E380005932DF0D2FD514630690395FFF77AFF7F
:107E4800D9F80C300027A34216D1C72302A93069FC
:107E580002930997FFF76EFFD9F80C30E41A304601
:107E68002DF02CFE002CE6D130694C302DF0A3FD0E
:107E7800204611B0BDE8F08F08F1840308F18C00AA
:107E880045EA040C5A785AB10BFA02F13CEA0101AE
:107E980006D117B17978914202D21A781F46029218
:107EA80002339842EED147B102A93069FFF742FF89
:107EB8007A78012393401D44D0E7094A23460121DB
:107EC800084800956FF015042CF07DFB30462DF026
:107ED800F5FDC9E76FF01504CAE700BF609C049080
:107EE8007B5A0590289804902DE9F0470D1E8EB016
:107EF800074690461E4665DB4068AA194FEAE573B7
:107F08004FF00001C06843F10003904271EB030396
:107F180058D3002E59D0342201A841F0E9F8386925
:107F28004FF48073DFF8A890069390F8BF3013F0F1
:107F3800010F0CBF4FF400534FF44053039390F8D4
:107F4800BC30322B009314BF4FF440634FF480636E
:107F580007934FF0407309932DF03FFDB6F5007F6E
:107F6800B2464FEA5522494628BF4FF4007A38698D
:107F78000AEB0503013BB2EB532F1CBFC5F3080AFC
:107F8800CAF5007AFFF7D6FE044698B9534642462A
:107F9800694638690195FFF7A1FE044650B938468D
:107FA800A6EB0A062DF08AFDD0445544044608B9CC
:107FB800002ED3D138694C302DF0FDFC20460EB090
:107FC800BDE8F0876FF01504F8E73446F6E700BF20
:107FD800609C04902DE9F04FB5B0476806690446E7
:107FE80020AA0021B8692DF088FF051E07DB209B19
:107FF80000221979186800F0EBFD051E06DA2B46F9
:10800800AB4A0121AB482DF0D8FC08E0DFF8A88284
:10801800D8F80890D9F800302BB96FF00405284635
:1080280035B0BDE8F08F39464046984705460028E8
:10803800F3D1D9F80C30002BEFD008AA39464046C6
:1080480098470028E9DB089A2846034601303D692D
:10805800B2FBF0F18D4203D2B0F5807FF5D1034633
:1080680073604025FA68304692FAA2F3002AB3FA00
:1080780083F308BF4FF0FF33013B33613B7D013B86
:1080880073610023C6E9073501F018FA8046002815
:10809800C3D1012206F14C0011462FF07FF80122CE
:1080A800414606F1640066262FF078F8BB68204642
:1080B80098473422414621A841F01AF84FF44073FA
:1080C80020A9206926932096FFF734FE034628B19D
:1080D8007A4A012177482DF070FC1CE0992520A9E7
:1080E80020692095FFF726FE034608B1744AF0E799
:1080F8004FF4807320A9206926932096FFF71AFE73
:1081080003460028E4D120A920692095FFF712FE34
:1081180003460028EAD10A202EF03AFE18230CAABA
:1081280000212069FFF78EFD054610B10346654A18
:1081380067E70C9B644A934207D0644A01215D4873
:108148006FF015052DF039FC69E79DF836300EAA59
:108158004FF0010B012B164697BF01331023DBB2FA
:10816800DB00D3180293029B2069B34200F0F2802F
:10817800F279337843EA0223B3F57F4F40F0DD818B
:10818800F37871799B00B27909023779502B41EA6B
:10819800024120AA28BF50233943FFF753FD8246E6
:1081A800002840F0D180219A2769002A616807F1E8
:1081B800840973DA22F000420123A2F1200AC2F1F5
:1081C800200003FA02F203FA0AFA23FA00F04AEA54
:1081D800000AD208C96842EA4A72B1EB420F4FEA74
:1081E800420304D03A4A012132482DF0E6FB00232D
:1081F8004FF0010AC7F88430C9F804304A4651469E
:1082080020A82DF05BFB20B999F80130013389F8DB
:1082180001300AF1010A09F102095FFA8AFABAF192
:10822800050FEBD1F3780A2B89BF2A9B4FF4807393
:10823800C3F303130BFA03F35B00A7F88C30209BFE
:10824800C3F34143012B49D10AAA20A93046FFF7BD
:10825800D5FC002844D19DF82830980740D09907CC
:10826800206904D51B49FFF765FD8246C0B9342251
:10827800002113A840F03CFFB72312A920691293EC
:108288004FF480731893FFF755FD824640B997F86D
:10829800BF3043F0010387F8BF3021E0013298E78F
:1082A80053460D4A012103482DF087FB4CE000BFDF
:1082B800945A05902898049054940490B35A0590C1
:1082C800CF5A0590EC5A059053464450015B0590EF
:1082D800195B0590609C0490335B0590022BD6D007
:1082E80040F204730DF1140A4FF00009ADF8143090
:1082F800FF2387F88F301AF8012B07AB20A93046E7
:1083080003922DF06DFA002810DB039A9DF81C30BB
:1083180087F88F2087F8BD309DF81D209DF81E3006
:1083280087F8BE3012B1134487F8BE30B9F1000F98
:1083380037D097F88F30FF2B36D16FF0850A854AF2
:10834800012185482CF02CF95346844A01218248A2
:108358002DF033FB22696368B2F88C0002F108063D
:10836800D968134693F884403CB193F88540B8F136
:10837800000F01D0444500D2A04602339E42F1D1FD
:10838800B8F1000F00F0DB80012303FA08F35C1E4C
:10839800044208BF0346C2F88030B1FBF3F3D36749
:1083A8003DE64FF00109A6E709AA20A930462DF0BD
:1083B80099FA031E10DA6A4A022167482DF0FDFA7D
:1083C800236993F88E30062B00F2B480DFE803F0BF
:1083D800B58C0B908C8C8C009DF82430C3F3420331
:1083E80087F88E30ECE740274FF0010906AA494686
:1083F80020462DF046FBB0F1000A7EDB9DF81820E0
:108408009DF81930174202D03B4240F096803A431B
:108418003B43544920698DF818208DF81930FFF72F
:1084280089FC8246002865D112AA012120462DF038
:1084380028FB824600285DD19DF848309B07F3D57C
:108448009DF849309807EFD50021342213A8D4F8B5
:1084580010A0CDE90A1140F04BFE0123B9F1010F3C
:10846800BDF8182012934FF4807318934FF080735F
:108478001B939AF88E3043D1012BADF8282053D1A5
:108488000DF12A02022120462DF0FBFAB0F1000A74
:1084980033DB0AAA042312A92069FFF71FFCB0F1F5
:1084A800000A2ADB20462DF009FBB0F1000A24DB84
:1084B80006AA494620462DF0E4FAB0F1000A1CDB72
:1084C8009DF818209DF81930174201D03B4234D14D
:1084D800BDF81830244A012100934B461E486FF01E
:1084E800040A2CF070F808E002274FF002097DE733
:1084F8008027FAE7BAF1000FA6DA53461B4AD1E6FD
:108508003121012BADF82A20129102D0043B012B16
:108518000DD80AAA012120462DF0B3FAB0F1000ABD
:10852800EBDB01231293B4E70AAA0223B3E70DF1A8
:108538002A02FAE76FF0850ADFE7083613E66FF0DC
:1085480085030B4A012104486FF012052DF035FA16
:1085580065E500BF505B059028980490E15B0590A5
:10856800735B0590609C04909E5B0590C25B0590D0
:10857800F55B059000487047989C0490044BB3F84D
:1085880080389B020B60002318464B60704700BF81
:1085980000E0F11F064B186828B94FF0010C4FF4A2
:1085A8000030C3E900C0012010600B60704700BFB5
:1085B800A02000240B4A5369DB0312D5002910DDE3
:1085C80000F1006300F01F000144BFF34F8F203912
:1085D800C2F85C3220330029F9DCBFF34F8FBFF3B8
:1085E8006F8F704700ED00E037B505682C6914F00F
:1085F800C06F0AD02B6EC3F30E030C4A02210C483D
:108608005B01009301232BF0DEFF0A480A4B204050
:108618006B6108D001230648084A194600942BF0DC
:10862800D2FF6FF0040003B030BD00BF365C059088
:10863800309804900000EE150F00EF1F515C059074
:1086480070B5054610461A46EFF31186102383F3DA
:108658001288BFF36F8F012383F31388104C63696B
:1086680043F480736361BFF34F8FBFF36F8F01F1E2
:10867800006140F015FD002383F31388636923F438
:1086880080736361BFF34F8FBFF36F8F86F31188D9
:10869800BFF36F8F2869BDE87040FFF7A5BF00BF23
:1086A80000ED00E0F7B517461A4606460D461C468B
:1086B8002DF039FA50B90B482B460B4A012100948A
:1086C8002BF081FF6FF0150003B0F0BD44B12346D5
:1086D8003A462946304603B0BDE8F040FFF7B0BF40
:1086E8002046F1E730980490675C059007B50BB118
:1086F800CB0604D103B05DF804EB2DF014BA2023A7
:10870800054A064800930B4601212BF05CFF002028
:1087180003B05DF804FB00BF915C059030980490AD
:10872800D3B50446154A002368462EF036FF206963
:10873800DDE90067FFF758FF00280EDB00222369F8
:108748001B68186910F0040009D052B14FF4FA53AD
:108758000B4A01210B482BF02CFF6FF0040002B0EC
:10876800D0BD32463B4668462EF03CFFDDE900327C
:1087780013430CBF01220022E1E700BF803801004B
:10878800E35C0590309804902DE9F84FB1F5003F6F
:10879800036907460D4690461E6809D32F480B46C5
:1087A8002F4A01212BF005FF6FF01500BDE8F88F67
:1087B800F46814F0010402D06FF00400F6E7FFF744
:1087C800AFFF0028F2DB05F1006505F120022B461A
:1087D800D3E90001B1F1FF3F08BFB0F1FF3FEBD192
:1087E80008339342F4D1F36843F00203F360BFF314
:1087F8004F8FDFF868B008EB040158F804204B6885
:108808002919C1E90023BFF34F8F2EF0C4FE0A22B5
:108818000023F8F78BFF10F1640941F1000A33696E
:108828005B070FD52EF0B7FE0A220023F8F77EFF6C
:1088380081457AEB0101F2DA64230A4A012158469C
:108848002BF0B7FE0834202CD5D13846FFF768FF47
:10885800F36823F00203F360A8E700BF30980490A0
:10886800F75C0590115D0590013A2DE9F041074646
:108878000D4600205618DFF87080AE420CD33B69D5
:10888800B5F5003F1C6809D318482B46184A012142
:108898002BF08FFE6FF01500BDE8F081E368DB0771
:1088A8001ED43846FFF73CFF0028F5DBE36823F4C5
:1088B800E063E360E36843F00403E360E36843F0E4
:1088C8008003E360BFF34F8F3846FFF729FFE36863
:1088D800002803EA0803E360DEDB05F50035CCE792
:1088E8006FF00400D8E700BFFBF8FFFF3098049052
:1088F800F75C05902DE9F743012306460F46144619
:10890800FFF7F4FE60B96FF015053B46224A0121D6
:10891800224800942BF057FE284603B0BDE8F083A8
:10892800002C36D030692DF0F7F833691B68DA6807
:10893800D20723D4224604F5FF34DFF86490394681
:1089480004F5FF743046FFF78FFF07EA09083C4437
:108958000546404604EA0901A1EB0801FFF72AFE93
:10896800336930461C68FFF7DBFE68B1002D08BF8D
:1089780005463069043002F0DDFBCDE7094A5A604C
:1089880002F188325A60D5E7E36843F00103E360F7
:10899800ECE72546C0E700BF225D059030980490BB
:1089A8000000FEFF230167452DE9F04104460069F8
:1089B80015461F460E462DF0AFF823691B68DA6886
:1089C800D2071BD43B462A46314620462DF0C0F834
:1089D800236905462046D3F80080FFF7A1FE98B129
:1089E800002D08BF054639463046FFF7E3FD2069EC
:1089F800043002F09FFB2846BDE8F081064A5A6021
:108A080002F188325A60DDE7D8F80C3043F00103F0
:108A1800C8F80C30E4E700BF23016745F7B51C46EA
:108A280017460123064622460D46FFF75FFE50B95A
:108A38000B482B460B4A012100942BF0C4FD6FF024
:108A4800150003B0F0BD44B123463A4629463046E6
:108A580003B0BDE8F040FFF7A7BF2046F1E700BF2D
:108A6800309804904D5D05902DE9F843D0F80490B6
:108A7800904607460D46D9F808001E462CF091FB93
:108A8800B8F5001F044616D1D9F808402846FEF765
:108A98003FFA84420CD129462CF083FB04462CF083
:108AA80085FB2046FEF722FA002120462CF087FBA2
:108AB8000020BDE8F883B8F5800F20D0B6F1806FAC
:108AC80019D0B6F1C06F18D0B6F1007F1AD10226BE
:108AD8003A460F492046FEF7E9F9B0B9D9F8081027
:108AE80028462CF095FB204631462CF068FB2046A2
:108AF800FEF7C4F9DCE70126EAE70326E8E76FF0AA
:108B08008500D6E76FF01500D3E76FF00F00D0E7C8
:108B1800C35D039008B5416805480C3183681B683C
:108B28001BB1984700EAE07008BD6FF05700F9E7FD
:108B3800549404901FB50C4B0C29D3F8082828BF6F
:108B48000C2112BA0C460192D3F8042812BA0292E8
:108B58000A46D3F8003801A91BBA039340F0A0FADB
:108B6800204604B010BD00BF00E0F11F37B54568CE
:108B780001AA0021E8682DF0C0F9041E07DB019B5B
:108B880000221979186800F023F8041E08DA0C4A44
:108B9800234601210B482BF00CFD204603B030BDC5
:108BA8000948696883681B682BB19847041E05DA71
:108BB800064A2346EDE76FF05704F9E70024ECE78F
:108BC8003E5E059058980490549404905C5E05901D
:108BD8002DE9F047044600EBC10600251C4FB442BE
:108BE80001D1002014E02068C30600F01F0911D449
:108BF800656845F02005C0F3481AC0F344201928D9
:108C080023D857F82080B8F1000F0DD16FF012006B
:108C1800BDE8F087B9F1100F04D0B9F1110FEAD10E
:108C28006568E8E73025E6E740462EF0D8F80028E2
:108C3800ECD04B462A460AF00F0140462DF0D3F8F7
:108C4800002804F10804CADAE2E76FF01500DFE74C
:108C5800309F049043681B6803F1080252E8002F14
:108C680042F0010203F1080040E800210029F3D195
:108C7800154A93421BD0A2F54C42934217D002F5F5
:108C88008062934213D002F5806293420FD002F5BE
:108C9800806293420BD002F54442934207D0A2F57A
:108CA8001C42934203D002F58062934203D15A6872
:108CB80042F040025A6053E8002F42F4807243E8C1
:108CC80000210029F7D170470010014043681B6854
:108CD80003F1080252E8002F22F0010203F1080014
:108CE80040E800210029F3D1154A93421BD0A2F590
:108CF8004C42934217D002F58062934213D002F59A
:108D0800806293420FD002F5806293420BD002F545
:108D18004442934207D0A2F51C42934203D002F585
:108D28008062934203D15A6822F040025A6053E8A5
:108D3800002F22F4807243E800210029F7D1704700
:108D4800001001402DE9F04182B080460D4643688D
:108D580000AF1E68002936D0586819698368DB6837
:108D68006BB13A1D9847041E0CDA1A4A01211A48B9
:108D78002BF016FC20460837BD46BDE8F0816FF0A1
:108D88005704F2E7336823F4004333607B6803EB4E
:108D98005503B3FBF5F30F2B18D86C468AB0D8F8F7
:108DA80000306A460D49D561C2E905134FF40073D6
:108DB80013840B4B42F8103F00234FF4115106481F
:108DC800FAF7E2FBA5466FF01504D3E79BB200243F
:108DD800F360CFE7C85E0590A0980490F65E059012
:108DE80004000001F8B50C46036941681D68237941
:108DF800012B15D09F1E7E427E41B6026279022A5F
:108E080096BF464F4FF4005737F81270A279022ADE
:108E180009D0042A30D0003B18BF01231B0306E009
:108E28004FF4C066EAE7B3FA83F35B091B07E279FC
:108E38000968012A14BF4FF0000C4FF4407CA5428A
:108E48001DD10A6822F0805222F4B05232431A43EC
:108E58000A604B6823F440533B434B6043681A68ED
:108E6800936823F4407343EA0C0393602968FFF77F
:108E780069FF00EAE070F8BD4FF48053D7E7D1F8F6
:108E880000E00EF4C06E764506D0D1F800E02EF46E
:108E9800C06E4EEA06060E6041680E68716801F4FD
:108EA80040518F4204D0716821F4405139437160B8
:108EB80041680E68316801F010218B4204D0316896
:108EC80021F010210B433360436819688B6803F461
:108ED80040739C4505D08B6823F4407343EA0C0328
:108EE8008B6043681B689968490405D5032A09D033
:108EF8009A6822F4804204E0032A03D19A6842F473
:108F080080429A6021682B68994205D0FFF71AFFC2
:108F18000028B0DB23682B600020ACE7684505908B
:108F28002DE9F04383B00546466800AF70683169A3
:108F380083681B685BB96FF057046E4A01216E485D
:108F48002BF02EFB20460C37BD46BDE8F083984732
:108F5800044630BB3A1D0021706A2CF0CEFF041E77
:108F6800F0DB7B68002219791868FFF731FE041ED0
:108F7800E8DBD5F804802B69D8F80040D3F80090D6
:108F8800236823F001032360D8F808002DF027FF99
:108F980078B95A4A012158486FF012042BF000FBA7
:108FA800D0E7544A012154482BF0FAFA002CC9DBC7
:108FB800D0E7D8E902018368DB6803B1984754E831
:108FC800003F43F00C0344E80032002AF7D1494639
:108FD8002846FFF707FF002802DA6FF01504B1E70B
:108FE80098F818301BB1A36843F00803A36098F8F9
:108FF80019301BB1636843F40043636098F81A3072
:109008001BB1636843F48033636098F81B301BB16D
:10901800636843F40033636098F81C30002B53D026
:10902800374B9C4233D0A3F54C439C422FD003F5D9
:1090380080639C422BD003F580639C4227D003F5C4
:1090480080639C4223D003F544439C421FD0A3F580
:109058001C439C421BD003F580639C4217D0294BCC
:109068009C4214D06C4688B02B686A462649C2E9EF
:1090780005134FF400739383244B42F8103F0023E9
:109088004FF4E2511C48FAF77FFAA546A5E76B684A
:109098001A68936843F480439360236898F81D2006
:1090A80023F0787343EA42532360236898F81E201C
:1090B80023F4F81343EA0243236098F81F301BB1E6
:1090C800A36843F40043A36098F820301BB12368D9
:1090D80043F000532360236843F001032360E369EE
:1090E8009A02FCD5E3695B02FCD5B36A28460024E2
:1090F800984727E70D5F0590A09804902D5F05908D
:1091080000100140000C0058485F05900300000162
:10911800F8B5436802460E4691F805E01C680369F5
:1091280008791D6801288B7913D1BEF1020F6CD91B
:10913800022B1F464FF4C0614FF4005C7DD0042B16
:1091480076D000287ED0C31E012B73D86FF085001F
:10915800F8BD02280AD1BEF1020F62D9022B1F46C0
:109168004FF480610BD04FF4005CE8E7BEF1020FCA
:109178005AD9022B1F4659D100286ED00021C31E90
:10918800012BE3D90020022703237345DED12CF0FD
:1091980000FFB842DAD1F3791BB3012B65D1344B08
:1091A8009C421ED0A3F54C439C421AD003F5806321
:1091B8009C4216D003F580639C4212D003F580636D
:1091C8009C420ED003F544439C420AD0A3F51C43AD
:1091D8009C4206D003F580639C4202D0254B9C42FA
:1091E800B4D123683146104623F001032360FFF70A
:1091F800F9FD0028AADB236843F00103236096E801
:10920800030085E803000020A2E74FF4C0611A4F6D
:10921800022B37F81EC01F4691D170B94FF080500D
:1092280010E04FF48061F2E70021F0E700219AE7AF
:1092380000288BD14FF4805004E0C31E012B85D940
:1092480002270020BCF5805F0BD0BCF5405F0AD038
:10925800BCF1000F98D1012397E701464FF08050E9
:1092680092E7002391E702238FE7032B97D06DE75E
:1092780000100140000C0058684505904FF0E023AD
:109288000F4910B59C691A6908689B6902F4803215
:109298000C4934B993B903464AB90A681044C01A4C
:1092A80010BD002B08BF03460AB9A342F5D90A68C6
:1092B80002440A604FF0E0221269EEE70446F3E741
:1092C8005C21002458210024094B1022002083F837
:1092D80023204BF68032074B1A604BF67F32064B41
:1092E80018604FF0E0235A61072298611A617047AD
:1092F80000ED00E05C21002458210024684620F09D
:1093080007018D4619B5FFF7B9FF1149114B0868D8
:10931800D3E90042001942F10002C3E900020E4AF3
:1093280000230B604BF68033D2E90041001BB0FBF1
:10933800F3F043431B1941F10001C2E9003102F087
:109348008DFEFAF739FDBDE819408546704700BF24
:1093580058210024E81A0024E01A00242DE9F041DD
:10936800DFF8E08099B1421C0BD14FF0E02213697D
:1093780023F0010313614FF07F43C8F80030BDE8C4
:10938800F081D8F80060012807DC00270BE0431CB7
:10939800D8F80060F7D14FF4AE7040F25D139842F0
:1093A800A8BF1846471EEFF31185102383F31288D0
:1093B800BFF36F8FFFF762FF234C4FF0E0239969EB
:1093C800D4E9002380184FF0000243F10003C4E9F8
:1093D80000031E4B1A601E4B1A68831A2ED44BF6D4
:1093E800803C0CFB073303F53B437F33B3FBFCF7AF
:1093F800131A40F6B8320CFB0733934238BF1346B2
:10940800144A934228BF1346C8F800304FF0E022B0
:10941800013B90695361002381429361A1EB0003F2
:10942800D4E9001238BF9B195B1842F10002C4E965
:10943800003285F31188BFF36F8FA0E740F6B83389
:10944800E2E700BF5C210024E81A00245821002428
:10945800E01A002400E2FE0038B5EFF3118510236E
:1094680083F31288BFF36F8F084B1C68084B1B6887
:10947800E41AFFF703FF85F31188BFF36F8F4BF6EC
:1094880080332044B0FBF3F038BD00BFE81A002455
:10949800E01A002438B5EFF31185102383F31288FE
:1094A800BFF36F8F044B1C68FFF7E8FE85F3118844
:1094B800BFF36F8F204438BDE81A002437B504463F
:1094C8002AF0BBFF0546002C41D094F841302BB957
:1094D80020462DF01DF941F28833A3642168204607
:1094E800A3680A68013B22F4F85242EA03220A60A0
:1094F8000022A36C202100932B462DF0E2F820BB1C
:109508002168E569E3680A682B43256A22F07F42EF
:109518002B43656822F0D00243EA056313430B60CE
:109528002168D4E905324D681343226943EA0243AE
:10953800084A2A4013434B602268136843F001032A
:1095480013600123606484F8413003B030BD01200A
:10955800FBE700BFFEF8E0FF38B5036804469968EA
:109568001A68480734D5550332D594F84120122A91
:1095780014D122689168480703D420462DF044FA94
:1095880038BDE16AF9B1626A127883F82020626A0C
:1095980001326262E26A013AE262EAE794F8412043
:1095A800222AEAD1226891684907E6D5A16B51B110
:1095B80093F82010226B1170226B01322263A26B88
:1095C800013AA263EEE7136823F480231360D4E71B
:1095D8008D076CD590036AD50222DA602268136879
:1095E80023F4E023136094F84130122B14D123683C
:1095F8001A68510709D51A6822F004021A60E36B49
:109608001A68D36823F00103D3600123204684F845
:1096180041302CF070FAB3E794F84130222B27D16F
:1096280023681A6852071DD51A6822F004021A60C6
:10963800E36B1A68D36823F00103D3600123204643
:1096480084F841302CF054FA9AE7A26B002AF5D03E
:1096580093F82010226B1170226B01322263A26BE7
:10966800013AA2632268926812F47C5FEDD1E5E7C3
:1096780094F84130022B06D10123204684F841306A
:109688002CF033FA7CE794F84130082B7FF478AF5C
:1096980022682046536923F040635361012384F80C
:1096A8004130636C002B3ED12DF0ADF968E70D0712
:1096B80012D5100310D50822DA6023681A685502FB
:1096C80006D51A6822F410221A60012384F8413062
:1096D80020462CF013FA53E7C80727D5D50325D51C
:1096E8000125DD602268136823F470231360636C1E
:1096F80043F00203636423681A68500710D51A6898
:1097080022F004021A600F4AE36B9A65E06B2CF0B2
:109718000BFF00283FF434AF636C43F00403636429
:10972800204684F841502CF0DAF929E7C9067FF57C
:1097380027AFD2027FF524AF10222046DA602CF042
:10974800E0F91DE7D569039038B50D460446F0B138
:1097580090F82C3003F0FF021BB980F82D202DF073
:1097680054F90223211D206884F82C3000F014F8E5
:109778006268294620682DF080F9064A002013689F
:1097880043F000431360012384F82C3038BD0120D6
:10979800FCE700BF0040005230B50A684D6AD1E9C5
:1097A80007342343154C92B902682B4322401343D4
:1097B8004A6813438A681343CA6813430A69134300
:1097C8004A6913438A6913430360002030BD026865
:1097D8002B4322F4F8421343036043684A6823404A
:1097E80013438A681343CA6813430A6913434A69CF
:1097F80013438A6913434360E7E700BF0080FFFF14
:10980800002854D02B4A936903F44043B3F5404FE2
:109818001FD1294B294A0344934242D9284B294A4C
:10982800034493423FD9284B984240D80020274A06
:10983800136823F00F0303431360136803F00F0347
:10984800984232D0136803F00F03C01A18BF0120E2
:109858007047936903F44043B3F5004F0ED11C4A97
:109868001C4B02449A421AD91B4A02449A4218D9FC
:109878001A4A02449A4216D90133D5E7184A194BB5
:1098880002449A4209D9184A02449A4207D9174A07
:1098980002449A4205D9164AEBE70420C7E7032099
:1098A800C5E70220C3E70120C1E70346CDE7012051
:1098B800704700BF00480258FFC4A7F7FFE0F5054E
:1098C8007FE2D3FB7F1D2C04801D2C040020005256
:1098D800BF4C2AF6BF3B47037F8871F93FC4B8FCE9
:1098E800FF6A45F53FA5AE023F10F4F77FB5A2FA2F
:1098F800BF5A51FD10B50A46044619B1024B002162
:109908001B68984710BD00BFB403002403460A4AE9
:1099180000209A6002F18832DA6002F12942A2F549
:109928009612A2F68B621A61A2F188325A61034A32
:10993800C3E900009A61704701234567F0E1D2C38B
:109948002DE9F04F4B68AFB0D1F800E01BBA8E6834
:10995800CD689EFA8EFE089336BA0B692DBA01902F
:1099680093FA83F84B6993FA83FA8B691BBA0A93C3
:10997800CB691BBA12930B6A93FA83FB4B6A1BBA27
:109988000B938B6A1BBA0C93CB6A1BBA0D930B6BA8
:109998001BBA0E934B6B1BBA03938B6B1BBA0493C6
:1099A800CB6B1BBA059383680F93C3680293036953
:1099B8000F9906934369029F10938369109A139332
:1099C800069B83EA0200029B1840E04B5040139A22
:1099D80003EBB7071A442F4402EBF16202991044D3
:1099E800069A82EAB1020F9970448EEA060E0A407E
:1099F80006998EEA0B0E4A40109919440A440899B0
:109A08000A440F994FEAB10C029902EBF0628CEA12
:109A1800B104044084EAB10406991944314486EA41
:109A280008060C448CEAB001114004EBF2644FEADA
:109A3800B20281EA0C019C4482EAB409394482EA00
:109A4800B007C444274001EBF46187EAB00709EA8C
:109A5800010967440AEB030C89EA020907EBF1677D
:109A68000CEBB00C0A984FEAB101E144184481EAC2
:109A7800B40C104409EBF7690CEA070C129A8CEA4B
:109A8800B40C1A44844481EAB70002EBB40200EA39
:109A980009000CEBF96C484010444FEAB9020BEB93
:109AA800030982EAB704894400EBFC6004EA0C0469
:109AB80084EAB70404EB090182EABC04DDF82C90BF
:109AC800044001EBF06199444FEAB000544009EBBF
:109AD800B7090C9F4C4480EABC091F4409EA0109F4
:109AE80004EBF16417440D9A89EABC091A44B94495
:109AF80080EAB10702EBBC02DDF838C0274009EB69
:109B0800F4694FEAB4049C444740844484EAB900A9
:109B1800174484EAB10202EA090207EBF96782EA0C
:109B2800B10238406244DDF80CC060409C4402EB4E
:109B3800F7624FEAB7070CEBB10C0499604487EA67
:109B4800B90C19440CEA020C00EBF2602144059CA4
:109B58008CEAB90C1C448C4487EAB20104EBB904C2
:109B680001400CEBF06C4FEAB0007940214480EAE8
:109B7800B20401EBFC69039904EA0C048EEA0101C2
:109B880084EAB20403EBF17E07910899BE4481EAA6
:109B980005070B99744485EA0A054F40049904EBBC
:109BA800F964794080EABC0703EBF17E07EA09070C
:109BB80008914FEAB9010EEBB20E0C9A4740564095
:109BC800059A7744564007EBF46703EBF67E4FEAB5
:109BD800F67286440D98149281EABC0245400798B3
:109BE800224085EAF07082EABC0211904FEAF070D8
:109BF800119D7244159081EAB40003EBF573384067
:109C080002EBF76203EBBC0348404FEAB70718447E
:109C18000A9B87EAB40988EA03080E9B89EA0209C5
:109C280000EBF26088EA0308089B88EAF37309935B
:109C3800099D474B03EBF57C039D8C4412998AEAF6
:109C48000101E14487EAB20A6940129D8AEA000AE2
:109C580009EBF06981EAF6714FEAB00003EBF17C99
:109C68000CEBB40C0A9C84EA0B08049CE24488EAD6
:109C78000408119C0AEBF96A88EAF47803EBF87C8B
:109C88004FEAF874BC440B9F169480EAB20485EA44
:109C9800070E059D84EA09048EEA050E099D6444B1
:109CA80080EAB90C8EEAF57E04EBFA648CEA0A0CB9
:109CB80003EBFE774FEAFE7507EBB2070C9A129595
:109CC8004FEABA0A079D8BEA0202BC448AEAB9073E
:109CD80082EAF57267400CEBF46C82EAF17203EBEE
:109CE800F27B0A920B9A83440D9D07EB0B0082EAE4
:109CF8000507089A0E9D00EBFC6087EAF27787EA71
:109D0800F8728AEAB4070B9203EBF27B0C9A87EAA3
:109D18000C070BEBB90B82EA05090D9A5F444FEA71
:109D2800BC0C89EAF6768CEAB40986EAFE7689EAFA
:109D3800000907EBF0674FEAF67503EBF67B17951A
:109D4800039DD34482EA050A04E000BF9979825A48
:109D5800A1EBD96E119AD9448AEAF2750A9A8CEA6B
:109D6800B00A85EAF2758AEA070A09EBF76903EB94
:109D7800F57B4FEAF5720BEBB40B0D924FEAB70780
:109D88000E9A0AEB0B04DDF810A004EBF96482EAE2
:109D98000A0A099A8AEAF27A0B9A8AEAF27287EA36
:109DA800B00A03EBF27B0C928AEA090A039AE344AD
:109DB8000AEB0B0CDDF814A082EA0A0A0CEBF46C2F
:109DC8008AEAF17A8AEAF67287EAB90A03EBF27B41
:109DD80003928AEA040A049A0BEBB00B0798DA4458
:109DE8004FEAB40B82EAF0748BEAB90084EAF8749B
:109DF80080EA0C000AEBFC6A84EAF57403EBF47859
:109E08004FEAF472B8440E9200EB0807059A0898D6
:109E180007EBFA6782EAF0700C9A80EAFE708BEA28
:109E2800BC0E80EAF2708EEA0A0E4FEABA0A03EB19
:109E3800F0784FEAF07208EBB9081192C644149A08
:109E4800DDF81C800EEBF76E82EAF8780A9A88EA49
:109E5800F278039A88EAF2728AEABC0803EBF2798C
:109E6800049288EA0708159AD944C844DDF8209076
:109E780082EAF9790B9A08EBFE6889EAF27989EAAD
:109E8800F4728AEAB70903EBF27B059289EA0E09B4
:109E9800149A0BEBBC0B4FEABE0E09EB0B0CDDF86A
:109EA800249082EAF9790CEBF86C89EAF6798EEA63
:109EB800B70689EAF07986EA08064FEAF97203EBF1
:109EC800F97B1492D344159A06EB0B0A82EAF176D1
:109ED800049A86EAF5768EEAB80586EAF27685EA85
:109EE8000C050AEBFC6A4FEAF67203EBF67B159257
:109EF8004FEABC0C169A0BEBB70B099F5D4482EA3C
:109F0800F7770C9A05EBFA6587EAF277059A87EAFC
:109F1800F2728CEAB807079203EBF27B129A87EA8F
:109F28000A07F3448CEABA0E82EAF171039A5F4495
:109F38008EEA050E81EAF271169A07EBF56781EA57
:109F4800F97B4FEAB50503EBFB7101EBB8018E44D1
:109F58000A9982EAF1710EEBF76E81EAF47485EAE8
:109F6800BA0184EAF67479404FEAF47203EBF478A4
:109F78001692E044129ADDF82CC0414482EAFC7C37
:109F8800079A01EBFE618CEAF07085EAB70C80EA6B
:109F9800F2708CEA0E0C01EABE0803EBF0734FEA8C
:109FA800F07203EBBA0312929C440A9A179B0CEBCB
:109FB800F16C83EAF272049B82EAF37282EAFB7321
:109FC8000893089AE74B03EBF272154441EABE0284
:109FD80002EAB70205EBFC6542EA0802DDF82C80CC
:109FE8002A440D9D85EAF875DDF8148085EAF87530
:109FF8004CEAB10885EAF47508EABE0809950CEA46
:10A00800B10548EA0505DDF8248003EBF87808EB8C
:10A01800B70805EB0807179DDDF8308007EBF267F6
:10A0280085EAF87888EAF97802EABC0988EAF078DB
:10A038004FEAF8750B9503EBF87505EBBE0E42EA8F
:10A04800BC050EEBF76E05EAB10545EA0905DDF832
:10A058000C90AE440D9D85EAF97547EAB20985EA88
:10A06800F676089D09EABC0986EAF5764FEAF675A0
:10A078000D9507EAB20549EA050503EBF67909EB00
:10A08800B1090E994D44DDF8309081EAF971DDF897
:10A098001C9005EBFE6581EAF971DDF8249081EAF0
:10A0A800F9710EEAB7090A9103EBF17101EBBC0CE7
:10A0B8004EEAB7010CEBF56C01EAB20141EA09017D
:10A0C800DDF80C906144DDF844C08CEAF97C45EA7F
:10A0D800BE098CEAFB7C09EAB7098CEAF87CCDF862
:10A0E8000CC005EABE0C49EA0C0CDDF80C9003EB39
:10A0F800F97909EBB2090E9ACC44DDF8109082EA9E
:10A10800F9720CEBF16C82EAF47401EAB50984EA9D
:10A11800F6744FEAF4720E9203EBF47202EBB7078F
:10A1280041EAB50207EBFC6702EABE0242EA09020D
:10A13800DDF814901744119A82EAF9724CEAB109D1
:10A1480082EAF0700A9A09EAB50980EAF2704FEAE1
:10A15800F07211920CEAB10249EA020203EBF079BB
:10A1680009EBBE09DDF850E04A44DDF810908EEAAC
:10A17800F97EDDF8209002EBF7628EEAF97EDDF8D1
:10A188000C908EEAF97E03EBFE79CDF810E007EA31
:10A19800BC0E09EBB50947EABC0509EBF26905EA0B
:10A1A800B10545EA0E05DDF814E0A944159D85EAD8
:10A1B800FE75DDF824E085EAFE7502EAB70E85EA49
:10A1C800F475059542EAB70505EABC0545EA0E0EA1
:10A1D800059D03EBF57505EBB1051499AE44079D94
:10A1E80081EAF5710EEBF96E81EAF87809EAB205B1
:10A1F80088EAF0784FEAF871149103EBF87101EBF3
:10A20800BC0C49EAB2010CEBFE6C01EAB701294328
:10A218000EEAB9058C44159981EAFB7A04998AEA11
:10A22800F67A079E8AEAF17A4FEAFA7115914EEAB0
:10A23800B90101EAB2010D4303EBFA7101EBB70171
:10A248000D44169981EAF6710A9E05EBFC6581EAD0
:10A25800F671059E81EAF671089E03EBF177079186
:10A268000CEABE0107EBB2074CEABE0207EBF56742
:10A2780002EAB9020A4305EABC011744129A82EAC3
:10A28800FB7B039A8BEAF27B45EABC028BEAF87BFC
:10A2980002EABE02114303EBFB7202EBB90211445E
:10A2A800169A82EAF67601EBF76186EAF47686EA90
:10A2B800FA764FEAF67203EBF674169247EAB5029D
:10A2C80004EBBE0402EABC0207EAB50E04EBF16433
:10A2D80042EA0E02DDF824E01444129A82EAFE7281
:10A2E80041EAB70E82EAF070079A0EEAB50E80EAE4
:10A2F800F2720C924FEAF2720C98129201EAB702CB
:10A308004EEA020203EBF07E08980EEBBC0E02EB5D
:10A318000E0C0B9A04EAB10E82EAF07204980CEB68
:10A32800F46C82EAF0720D9882EAFB72089203EBF1
:10A33800F27202EBB50244EAB10502EBFC6205EAEF
:10A34800B70545EA0E050CEAB40E2A44099D80EAD1
:10A35800F575059885EAF07585EAF6704CEAB40556
:10A3680002E000BFDCBC1B8F099005EAB10545EA95
:10A378000E0E03EBF07505EBB705AE44DDE90A50A8
:10A388000EEBF26E80EAF5750C984EEAB20985EA92
:10A39800F87502EABC0885EAF075039809EABC0971
:10A3A8004FEAF577179703EBF57707EBB10742EA22
:10A3B800BC0107EBFE6701EAB40141EA08010EEAB5
:10A3C800B2080F440D9949EA080881EAF071089823
:10A3D80081EAFA714FEABE0A81EAF0718AEAB20E9E
:10A3E80003EBF1734FEAF1708EEA070E03EBB40347
:10A3F8000D9008EB03040A980E9B04EBF76483EABC
:10A40800F073079883EAF073099883EAF0730A9364
:10A418000A98DF4B03EBF078119808EBBC08DDF8DD
:10A428000CC080EAFC7CC6448AEAB7088CEAFB7C4C
:10A438000EEBF46E88EA04088CEAF5704FEAB4046F
:10A4480003EBF07C0B9004980CEBB20C0E9A82EAAA
:10A45800F079E04484EAB70C059889EAF6798CEA41
:10A468000E0C08EBFE6889EAF1794FEAF9720E9250
:10A4780003EBF97252449444119A82EAF0760C9AEA
:10A488000CEBF86C86EAF2760A9A86EAF2764FEADC
:10A49800F67203EBF6700C9284EABE0200EBB7008A
:10A4A800149F82EA080202444FEAB800DDF81080DF
:10A4B80080EABE0A87EAF877DDF820808AEA0C0A83
:10A4C80002EBFC6287EAF877DDF82C8087EAF877F8
:10A4D8004FEAF777039719971F442744159CBA4406
:10A4E800059F84EAF774099F0AEBF26A84EAF77415
:10A4F80084EAF9744FEAF4740494049F1A9480EA85
:10A50800BC041F4454404FEAB20207EBBE07059251
:10A518003C44149A079F04EBFA6482EAF778059A98
:10A5280088EAF57882EABC05159A88EAF67885EA19
:10A538000A054FEAF87808EB0307CDF86C80074462
:10A548003D4482EAFB77059A87EAF177039982EA24
:10A55800BA00169A4F4005EBF46560404FEAB40420
:10A568004FEAF77784EABA0EF9181C978EEA050EB7
:10A5780001EBBC010844079982EAF1710A9A00EBE1
:10A58800F56081EAF271049A5140059A4FEAF17137
:10A5980001EB030C1D919444129AE64482EAFB7283
:10A5A800DDF82CC00EEBF06E82EAFC7284EAB50C82
:10A5B80082EA08028CEA000C4FEAB0004FEAF27215
:10A5C80002EB030B1E920BEBBA0BDDF858A0DC4430
:10A5D800DDF820B08AEAFB7A0CEBFE6C8AEAF97A9D
:10A5E8008AEA070A4FEAFA7980EAB50ACDF81490A0
:10A5F800CDF87C9099448AEA0E0AA144129CCA4478
:10A60800DDF8249084EAF9740AEBFC6A84EAF674AB
:10A6180080EABE064C4086EA0C064FEABC0C4FEABC
:10A62800F4748CEABE09079420941C4489EA0A0948
:10A6380004EBB504039D2644179C84EAFB7406EBDF
:10A64800FA666C4054404FEAF474E51821940544C6
:10A658000D98A944099D80EAF570049D09EBF669F7
:10A668006840059D68408CEABA054FEAF07075406D
:10A678004FEAB60600EB030B22900BEBBE0BDDF89E
:10A688005CE05D44DDF828B08EEAFB7E05EBF965F9
:10A698008EEA080EDDF81C808EEA080E86EABA08F3
:10A6A8004FEAFE7E88EA09080EEB030BCDF88CE032
:10A6B800E344DDF834C0D844DDF82CB08CEAFB7CE8
:10A6C80008EBF5688CEA070C8CEA040C86EAB904F6
:10A6D8004FEAFC776C404FEAB50507EB030C24976B
:10A6E8000CEBBA0CDDF828A06444DDF838C08CEA1D
:10A6F800FA7C04EBF8648CEA010C8CEA000C85EA1D
:10A70800B9004FEAFC7180EA080001EB030C2591BF
:10A71800B4440C9E86EAFB766044564085EAB8024B
:10A7280000EBF46086EA0E0662404FEAB4044FEA92
:10A73800F6762D9426961E4406EBB9063244039EFF
:10A7480002EBF06C0E9A5640059A56400C9A7E40E1
:10A7580084EAB8074FEAF67647404FEAB0002796F2
:10A768001E442C902E44049D5540079A374455406A
:10A778004FEABC0207EBFC674D4084EA00012A97C8
:10A7880018954FEAF57581EA0C012B9202E000BF9B
:10A79800D6C162CA28951D4405EBB8054B190F9917
:10A7A80003EBF76329930B4401998B60029B1F44C9
:10A7B800069B1A44109BCF601844139B0A611C44E3
:10A7C800486118A88C615821FFF794F800202FB031
:10A7D800BDE8F08F03460846C1B90E4ADFF838C015
:10A7E800C3E910110D49C3E912120D4A0D49C3E915
:10A7F80014C20D4AC3E916120C4A1A6602F17452C1
:10A80800A2F52302A2F692425A6670476FF07300CF
:10A81800704700BF85AE67BB72F36E3C67E6096A96
:10A828003AF54FA57F520E518C68059BABD9831F13
:10A838002DE9F04FCFB0044600F1480300F1680657
:10A8480046AD03911868083353F8041C2A46B342EE
:10A8580003C21546F6D1DDF834B104AA4A984FF080
:10A86800000CDDE94883DDE94B9601933D4BDDE9BA
:10A8780046150293BCF10F0F5CD8039B53F82C309C
:10A888001BBA4FEAF02E86EA0907DDF808A00CF19A
:10A89800010C8EEAB01E07409360BCF1400F8EEAAF
:10A8A800706E87EA060702F1040277445AF804EB4F
:10A8B800774445EA010ECDF808A005EA010A3B44B1
:10A8C8004FEA71370EEA080E87EAB1075B444EEA91
:10A8D8000A0EB34687EAB1577744DDF804E0CDF8AD
:10A8E80004809E443B441ED1CDE94631CDE904376E
:10A8F80045A904F144036434CDE94C96CDE94AE016
:10A90800CDE9485853F8042F51F8040FA3420244E4
:10A918001A60F7D104A84FF49471FEF7EBFF0020FA
:10A928004FB0BDE8F08FA8464E460D468146194601
:10A9380070469FE7136852F834AC4FEAF34E52F86A
:10A94800387C8EEA734E8EEA932E52F8143C3B44C0
:10A958004FEABA4787EAFA17734487EADA073B44AB
:10A968008FE700BF44A0049070B5044688B103780F
:10A97800C3B10D4D0D4EB54201D3002409E029683D
:10A98800A14208D128462CF02AFA002814BF2C46E8
:10A998000024204670BD2046F6F7E2FE0028F1D0DC
:10A9A8001C35E8E71C46F4E754940490BC960490E0
:10A9B80010B50446F8F718FD03480121034A29F0A9
:10A9C800EFFD20462CF016FA80980490955F0590CC
:10A9D8002DE9F843044600AF0D46EFF31188102324
:10A9E80083F31288BFF36F8F0428294AE9468AB097
:10A9F80098BF284B9668117C6A4694BF53F820305C
:10AA0800254BC2E9073140F2013324489384244B93
:10AA1800C2E9050442F8103F00234FF431512148A0
:10AA2800F8F7B2FDCD4645B1EB69C3F3080323B18E
:10AA38001D4A01211B4829F0B3FD2EB130462CF0E8
:10AA480031FC08B1037803B91848E9468AB06A4668
:10AA5800174BD061C2E9053640F201331384154B18
:10AA680042F8103F00234FF411510E48F8F78CFDBF
:10AA780029462046CD46FFF79BFF88F31188BFF390
:10AA88006F8F3046F9F7BCFCBD46BDE8F88300BFC0
:10AA98006021002444A10490A45F0590BA5F05904A
:10AAA8000500000180980490E25F0590B25F059070
:10AAB800036005900400000138B50A4B53F82040A4
:10AAC800013053F82050A54200D838BD606830B135
:10AAD800037EDB0701D42CF06AF90834F3E7236816
:10AAE8009847FAE758A104902A4B0122032070B531
:10AAF800294C86B0294D1A70FFF7DEFF01F038FCAB
:10AB08000420FFF7D9FF26463034AE4210D3224C3A
:10AB180000F082FF224EAC4226D300F091FF28F0CD
:10AB28003AFE204A938923F00103938106B070BD51
:10AB380054F80C3C059354F8103C049354F8143C16
:10AB4800039354F8183C029354F81C3C019354F8AE
:10AB5800203C009354E90A2354E90C0100F036FD27
:10AB680054F8303C5E65CEE7D4E90A23B3F1FF3FE1
:10AB780008BFB2F1FF3F05D052EA0301206803D1B4
:10AB880001F030F83034C6E73146183001F0D6F914
:10AB9800F8E700BFA2280024C0960490F09604901D
:10ABA8008D730390901B002470B5A023154E86B0BA
:10ABB800012203FB00660023134D04460193134949
:10ABC800CDE904230F22CDE9023214234FF4A072F9
:10ABD80003FB00554FF4C0700D4B00FB04113046C9
:10ABE800009500F0F3FC337C0A4A23F00403EE607E
:10ABF8002C7433744FF4046304FB033313446B6005
:10AC080006B070BDF01A002460210024004300241F
:10AC1800836F0390C03A0024BFB50020FFF74CFFB4
:10AC2800274B83F30888274D0024F023264F85F807
:10AC38002230EC772C766C76AC7685F820406B6AFF
:10AC480043F4E0236B62F9F7EFFAF9F7E9FC4FF008
:10AC5800FF33AB62EB62F9F763FE1C4DF9F7A8FD11
:10AC6800F8F724FB1A4800F043FDF8F7C9F901206A
:10AC7800FFF722FF0220FFF71FFF00F015FF154B1B
:10AC880015494FF4BE425D612846144B0094059364
:10AC98000123CDE90144CDE903433B4600F096FC8E
:10ACA8002A7C0646284622F004022A742CF036FB39
:10ACB8002046FFF779FF3A4631462846F9F790FCD7
:10ACC8000043002400ED00E0F1AA0090901B00244E
:10ACD800301C00246021002480440024904C0590FE
:10ACE80038B5064C064DAC4201D3002038BDD4E936
:10ACF8000112204614342CF0C7F8F4E7100C002495
:10AD0800240C002430B585B0044BDDE908450293D6
:10AD1800CDE900452CF076F805B030BD773C0390BE
:10AD280038B50020054C064DAC4200D338BD20464E
:10AD38002CF0CEF80028F9DB1C34F5E7F40B0024DE
:10AD4800100C002473B50C46EFF31181102585F320
:10AD58001288BFF36F8FC5685DB125602B68C3602B
:10AD6800836901338361002081F31188BFF36F8FFA
:10AD780011E052EA030603D16FF00B002560F3E7F8
:10AD8800CDE900230246083000F08CFD18B9034BCA
:10AD98009B685B69236002B070BD00BF602100241E
:10ADA8002DE9F34104460E469DF8200004F10808F9
:10ADB800EFF31187102181F31288BFF36F8F256A93
:10ADC800E1688D4246D22568AC4218D0BDB128460C
:10ADD8002CF0DEF805F118002CF0B1FBA268314622
:10ADE80068693EF05DF900232846C5F898302CF0D4
:10ADF80095FA4046394600F0E9FD002037E0A268A0
:10AE0800D8B13146E0693EF04BF9E369A2681344D2
:10AE180062699342E36101D12369E361236A1021E6
:10AE280004F12400013323622CF068FC0028E0D1EF
:10AE380087F31188BFF36F8F19E0A16923699942DD
:10AE4800314604BF6369A361A069801AA0613EF01E
:10AE580027F9E3E752EA03010CD00849404689681C
:10AE68004E613946CDE90023224600F01BFD02B0B1
:10AE7800BDE8F0816FF02200DAE700BF602100240E
:10AE8800F7B50446084604F10807EFF311861021C8
:10AE980081F31288BFF36F8F216A00293AD0A26824
:10AEA800A1693EF0FDF8A369A268256813446269A8
:10AEB8009342A36104BF2369A361AC42236A03F1EF
:10AEC800FF33236234D02846002D32D02CF060F8AE
:10AED80005F118002CF033FBA2686969E0693EF0BF
:10AEE800DFF8E369A2682846134462699342E36184
:10AEF80004BF2369E361236A013323620024C5F890
:10AF080098402CF00BFA3846314600F05FFD204699
:10AF180003B0F0BD52EA030110D00A4989684861BC
:10AF280031463846CDE90023224600F0BBFCEFE766
:10AF3800002086F31188BFF36F8FE9E76FF02200D6
:10AF4800F7E700BF602100242DE9F34104461746C6
:10AF58001E46EFF31188102383F31288BFF36F8F17
:10AF6800C368314A7BB180689168884219D057EA32
:10AF7800060318D188F31188BFF36F8F6FF00F00A5
:10AF880002B0BDE8F081916891F90E10013321619A
:10AF9800E3609368A36088F31188BFF36F8F002084
:10AFA800EEE72169F2E790F90E3091F90E10994217
:10AFB800A8BF19468B422DDD2CF054F805462246D1
:10AFC80041461A48CDE9007600F06CFC0028E6D02E
:10AFD800EFF31186102383F31288BFF36F8FA068F5
:10AFE800D0B1236821699C420AD04BB193F90E3045
:10AFF8009942A8BF19466FF07F039942B8BF194616
:10B008002CF030F840B13146084800F0DFFC6FF012
:10B018000A00B5E70025D2E7002DF4D186F31188A0
:10B02800BFF36F8FF3E700BF60210024A32800243B
:10B03800F8B583680546002B40D0234A92689342AE
:10B048003FD1C368012B03D9013BC3600020F8BD81
:10B05800EFF31187102383F31288BFF36F8F016911
:10B0680080682BF0FFFF2C68AC4207D10023C5E9AC
:10B07800023387F31188BFF36F8FE7E7002CF5D011
:10B08800002604F11800D4E9003213605A60237CCA
:10B09800A66023F00203C4E9006623742CF04FFA7B
:10B0A800AC6094F90E3020462B61C4F898602CF0FF
:10B0B80035F93946054800F089FCC7E76FF01500F7
:10B0C800C5E74FF0FF30C2E760210024A328002421
:10B0D80037B51146EFF31185102282F31288BFF3BA
:10B0E8006F8F04689CB123680121426823F0030331
:10B0F8009442036008BF436020462CF039F80446A8
:10B1080085F31188BFF36F8F204603B030BD51EA35
:10B118000302F5D000F10802CDE9001310462946D4
:10B1280000F0C0FB0028EFD1014B9B685C69EBE79E
:10B138006021002470B5EFF31186102383F3128881
:10B14800BFF36F8F0468A0421BD0D4B1002504F16F
:10B158001800D4E9003213605A60237CA56023F0FC
:10B168000203C4E9005523742CF0E9F92046C4F819
:10B1780098502CF0D3F831460B48BDE8704000F0E9
:10B1880025BCD0E90232022110309A4218BF01339F
:10B1980040F8083C2CF0B2FA0028ECD186F311886C
:10B1A800BFF36F8F70BD00BFA328002413B5EFF362
:10B1B8001181102484F31288BFF36F8F846844B11F
:10B1C800013C846081F31188BFF36F8F002002B0C7
:10B1D80010BD52EA030406D181F31188BFF36F8FC3
:10B1E8006FF00F00F3E7CDE900230246014800F0B5
:10B1F80059FBECE7A32800242DE9F8430546EFF3B3
:10B208001188102383F31288BFF36F8F00266FF025
:10B218000A0937462C68A54216D0ACB104F11800CB
:10B228000126D4E9003213605A60237CA76023F01A
:10B238000203C4E9007723742CF081F92046C4F88E
:10B2480098902CF06BF8E5E70023022105F1100037
:10B25800AB602CF053FA30B92EB988F31188BFF3DC
:10B268006F8FBDE8F88341460248BDE8F84300F017
:10B27800ADBB00BFA32800242DE9FF4104461027D9
:10B288004E4EEFF3118887F31288BFF36F8FD4F80F
:10B29800A450F5B9022104F1BC002BF08FFF00285F
:10B2A80068D004F1B4050022012128462CF0DCF80E
:10B2B8000028F8D100234FF0FF324146404802935E
:10B2C8004FF0FF33CDE9002304F1AC0200F056FD46
:10B2D800D7E7D4F8A8202B689542C4F8A43008BF53
:10B2E800C4F8A830D4F8BC3043F00203C4F8BC302A
:10B2F800EB6823F0040343F00103EB606B6888F309
:10B308001188BFF36F8F28469847EFF3118887F3AA
:10B318001288BFF36F8FEB68D80623F0010236D48A
:10B32800EA60EB689A0716D523F002033068EB60F1
:10B3380088B10368002170B14268954235D103682D
:10B3480069BB72683360824200D17360002340F8A1
:10B35800083BFFF7EFFED4F8BC3023F00203C4F833
:10B36800BC3088F31188BFF36F8FDB0589D400F0F8
:10B37800B9FB86E7D4F8BC30D9069BD5C4F8BC0025
:10B3880088F31188BFF36F8F04B0BDE8F08123F014
:10B398001103EB6005F11000FFF7CCFEC1E70B606D
:10B3A8007368834208BF7160D0E723B11A68014609
:10B3B80018461346BFE71A46F9E700BF8421002460
:10B3C800A3280024F8B5C36804460F469A07C3F3B8
:10B3D80040062DD45B071BD40B680BB983680B6040
:10B3E800E368DD0745BFA368022601263B603D6888
:10B3F800002D3CD01F4B9A68D5F8A0309A420AD04D
:10B40800D5F8BC30D807C3F3800214D46FF0120605
:10B4180000233B6025E02BF03CFFD5F8BC3000282A
:10B42800F0D1D907C3F3C002F0D552B15B0708D4F5
:10B438006FF00F06ECE7002AFAD1C3F3C003002B24
:10B44800F6D100232360D5F8A83063B9C5E92944AB
:10B4580028462BF0CDFEE36843F00403E3603B6825
:10B46800A3603046F8BD1C60C5F8A840F0E76FF04F
:10B478001506CDE760210024014601482BF0F9BEEE
:10B48800F01C0024F0B50446002089B0C4E9290066
:10B4980004F1AC000E9DC4E92B0004F1B400C4E92A
:10B4A8002D0055B32879002840F2011008BF01206B
:10B4B800C4F8BC0000204FF0FF364FF0FF3700946F
:10B4C800CDE90330CDE901000D4B2046CDE90667F3
:10B4D80000F0E2F855B1296811B120462BF0DFFEE3
:10B4E8006B791BB1A38943F00103A381204600F0C7
:10B4F80079FBC4F8A04009B0F0BD0120D8E700BF2F
:10B5080081B2009037B501900846EFF311841021FD
:10B5180081F31288BFF36F8FC16811F01E0F17D126
:10B5280053EA020508D101A9FFF74CFF84F31188FB
:10B53800BFF36F8F03B030BD41F00801103040F801
:10B54800041C01998161034900F0F8FC0120EDE732
:10B558000020EBE70772039001460148FFF7D2BFCE
:10B56800F01C0024F7B50C4616461D460190EFF373
:10B578001187102383F31288BFF36F8F08462BF0CF
:10B5880028FE55EA060309D101A92046FFF71AFF4C
:10B5980087F31188BFF36F8F03B0F0BDE3683246BD
:10B5A800064904F1100043F00803E360019BA3621D
:10B5B8002B4600F0C3FC0120EAE700BF07720390A6
:10B5C80001460148FFF7CEBFF01C0024073222F0E5
:10B5D80007022DE9F04F7F3285B01F4600F158036E
:10B5E800044622F03F020E4604213F2AA2F1400BF6
:10B5F80006F14008C0E91633129B4FF00000217491
:10B60800A381119BA060A373E073DDE90EA9C4E9CF
:10B61800060005D880F31188BFF36F8F084602DF54
:10B62800B51820462946F8F7A7FB0730109B314686
:10B6380020F007002D1AC4F8880020462A46C4E9DD
:10B64800208BCDE90193CDF800A03B46F8F798FF91
:10B658000023C4F874906365109BC4E91B7AA36740
:10B66800EFF31182102383F31288BFF36F8F094B16
:10B67800196A1C62E16782F31188BFF36F8F9B68B8
:10B688000BB1D3F88C302846C4F88C3005B0BDE82F
:10B69800F08F00BF60210024F0B5002587B0044674
:10B6A8000595109D04950F9D03950E9D02950D9D82
:10B6B80001950C9DDDE912760095FFF787FFB6F13D
:10B6C800FF3F08BFB7F1FF3F05D056EA070305D192
:10B6D800204600F087FA204607B0F0BD3A463346C8
:10B6E80004F11800014900F029FCF4E78D73039078
:10B6F8000123037483810023C0E92033C0F88C3010
:10B70800014B9860704700BF602100240A4A6FF01F
:10B718000A019368C3F898100849C3F894004B6865
:10B7280043F080534B60002383F31188BFF36F8F7E
:10B738009368D3F8980070476021002400ED00E07A
:10B7480070B590F91020037C002A36DBD90634D175
:10B758001B4C63F07F0322460374E16952F8183FDB
:10B76800934207D1C0E900210860E06111E09942E5
:10B77800F8D01B68002BF5D090F90E5093F90E60A5
:10B78800B542F4D0AE42F2DD5968C0E90031086034
:10B798005860A569954200D005B9E568A3681A7C88
:10B7A800D20604D1DA897F2A01D9AA6932B1AB421B
:10B7B80002D0284600F024FB656170BD6361FCE798
:10B7C8006021002438B590F910200146037C002A36
:10B7D80004DA03F07F0303742BF066FD0D4D2A464F
:10B7E800AB6852F8184F944200D004B9EC688B4209
:10B7F80007D01A7CD20604D1DA897F2A01D9A26936
:10B808002AB1A34202D0204600F0FAFA23466B611F
:10B8180038BD00BF60210024B3F1FF3F08BFB2F17B
:10B82800FF3F03D00249183000F088BB704700BFC3
:10B838008D73039038B5194CA168E0690B68814293
:10B8480014BF1A46002249680B605960A368E16971
:10B858002AB9134AC3E900210B60E3610CE093F9AC
:10B868000E0092F90E50A84214D0854212DD51689C
:10B87800C3E900210B605360A569094B9D4200D0C4
:10B8880005B9E568A3689D4202D0284600F0B8FAD9
:10B89800656138BD9142DCD01268D9E76021002487
:10B8A80078210024F8B50E4B0C4611460D4A9868CD
:10B8B800DDE906671060EFF31182102282F3128827
:10B8C800BFF36F8F9D6828462BF000FD284632464F
:10B8D8003B46FFF7A1FF2046BDE8F840FFF716BF3B
:10B8E800602100248C210024F8B50446EFF3118769
:10B8F800102383F31288BFF36F8F037C49B203F0E0
:10B908001F02002A0CBF0126002639D103F07F034D
:10B918002D4D03742BF0C8FC037C2A46817363F019
:10B928007F03037452F8183F934227D1E869C4E9AA
:10B9380000200460EC610FE09842F8D01B68002BEF
:10B94800F5D093F90EC06145F6D08C45F4DD596801
:10B95800C4E900310C605C60AC69944200D004B961
:10B96800EC68AB689C4202D0204600F049FA6C6152
:10B9780087F31188BFF36F8F3046F8BDE869DEE7BB
:10B988009B071ED585682BF08FFC81732B689D4221
:10B9980009D16B68C4E900531C606C60E8E76A6809
:10B9A8009342F6D01B68002BF3D093F90E209142F6
:10B9B800F5D08A42F3DD5A68C4E9003214605C604D
:10B9C800D6E78173D4E700BF6021002449B9EFF3BB
:10B9D800058030B9054B5A699B689A4201D0FFF738
:10B9E80095BE81F31188BFF36F8F704760210024E3
:10B9F800034648B9EFF3058232B9064A516992689D
:10BA0800914201D0FFF782BE83F31188BFF36F8F95
:10BA1800704700BF60210024EFF31181102383F3E6
:10BA28001288BFF36F8F054B9A68D37B013BD373A2
:10BA380081F31188BFF36F8F704700BF6021002426
:10BA480070B5EFF31186102383F31288BFF36F8F5D
:10BA5800144DAB68DA7B0132DA732A4652F8184F74
:10BA6800944200D004B9EC681A7CD20604D1DA8971
:10BA78007F2A01D9A2692AB1A34202D0204600F048
:10BA8800BFF923466B6186F31188BFF36F8FEFF31D
:10BA98001180102383F31288BFF36F8FBDE87040C5
:10BAA800FFF7A6BF60210024024B03F11802C3E987
:10BAB800062270476021002408B5FFF715FF70B112
:10BAC800074B9B68DB7B53B9EFF31180102383F39B
:10BAD8001288BFF36F8FBDE80840FFF789BF08BD24
:10BAE8006021002470B5EFF31186102383F31288C8
:10BAF800BFF36F8F1B4CA168E0690B68814214BFCC
:10BB08001A46002249680B605960A368E1692AB99E
:10BB1800154AC3E900210B60E3610CE093F90E00BC
:10BB280092F90E50A84218D0854216DD5168C3E933
:10BB380000210B605360A5690B4B9D4200D005B9ED
:10BB4800E568A3689D4202D0284600F059F93046BE
:10BB58006561BDE87040FFF7D9BD8A42D8D0126848
:10BB6800D5E700BF6021002478210024F8B550EA09
:10BB7800010306460C4603D1FFF7B4FF0020F8BDC9
:10BB8800EFF31187102383F31288BFF36F8F124DE1
:10BB9800124BA8681860FFF715FEA86823463246BE
:10BBA8000F49183000F0CAF9AA6804463846137CD1
:10BBB80043F004031374FFF7A9FDAB68D3E90A2324
:10BBC800B3F1004F08BF002AD8D12BF0E0FC201AAF
:10BBD80020EAE070D3E700BF602100248C21002414
:10BBE8008D73039038B50446EFF31185102383F362
:10BBF8001288BFF36F8F037C5B070FD518302BF0CB
:10BC08009EFC237C204623F004032374FFF798FD51
:10BC180029460548BDE83840FFF7D8BE85F31188A6
:10BC2800BFF36F8F38BD00BFA3280024014B98686D
:10BC3800704700BF602100242DE9F8430446878936
:10BC4800EFF31185102383F31288BFF36F8F037C02
:10BC5800190705D585F31188BFF36F8FBDE8F88301
:10BC6800D90943F0080260D10274A36813B12046D1
:10BC78002BF022FB04F1180004F158082BF05FFCAC
:10BC8800A66DB04511D04FF0000976B130462BF0C3
:10BC980013FB06F118002BF052FC3046C6F89890BA
:10BCA800FFF74EFDA66DB045EFD1DFF8C480D8F898
:10BCB80008309C4241D1EFF30589B9F1000918BF5A
:10BCC8004FF00109D8F818602A4A964200D00EB9F8
:10BCD800D8F80C60B34202D0304600F091F8204604
:10BCE800C8F8146028F0D3FD204600F0DBF8B9F15D
:10BCF800000F02D02048FFF7FBFCD8F808309C4220
:10BD080031D1EFF3058373BBA289D20718D4284633
:10BD1800FFF7FCFCFB07A1D5002383F31188BFF3D1
:10BD28006F8F0423184602DF98E703F07F0343F080
:10BD3800080303742BF0B8FA97E74FF00009C1E73E
:10BD480085F31188BFF36F8F83F31188BFF36F8F6B
:10BD58000423184602DFEFF31180102383F31288BF
:10BD6800BFF36F8FD4E785F31188BFF36F8FD1E7E7
:10BD78006021002478210024301C0024D3B5DDE99B
:10BD88000667089CCDE90067FFF78CFD1CB1034BE3
:10BD98009B685B69236002B0D0BD00BF60210024AE
:10BDA800027C034612F01F0210D10A4988420DD0C6
:10BDB8000949086868B1D9897F2909D893F90E20FB
:10BDC800064B1B689A42B8BF002070470020704796
:10BDD80010467047F01A0024B8030024902100246C
:10BDE800044B0122C01A044BC0105843034B1A5489
:10BDF800704700BFD01C0024ABAAAAAAA32800241D
:10BE08000D4B70B51E7CFFF7CBFF0C4D044606EBBF
:10BE1800460305EBC30528462BF091FB084B00228F
:10BE28009A553CB1621E28460649D317BDE87040B2
:10BE380000F084B870BD00BF60210024D01C00242D
:10BE4800A3280024E9BD009038B5EFF3118510232D
:10BE580083F31288BFF36F8F0F4B104A9C681068EA
:10BE6800A04206D1FFF7CCFF85F31188BFF36F8F8F
:10BE780038BD00211B7C1160094AD35C002BF3D02C
:10BE88002046FFF78DFF0028EED0237CDB0601D18A
:10BE9800FFF7D0FC2046E5E7602100248C21002430
:10BEA800A3280024EFF31181102383F31288BFF332
:10BEB8006F8F0A4A136A834207D1DB6F136281F3DB
:10BEC8001188BFF36F8F70471346002BF7D0DA6FD6
:10BED8008242F9D1C26FDA67F1E700BF602100241E
:10BEE800024B1868984208BF00207047BC03002422
:10BEF800034B1B680BB9FDF7AFBA0020704700BFB2
:10BF08009421002430B570B10B4B5B6898420AD07D
:10BF1800036843B1D3E90421D0E90445121941EB80
:10BF28000501C3E90421D0E9003213605A600023F7
:10BF3800C0E9003330BD00BFBC030024B3F1FF3FAC
:10BF480008BFB2F1FF3F2DE9F84F04469946154660
:10BF58001F467AD08160EFF31188102383F312888B
:10BF6800BFF36F8FB9F1000FDFF8E4A020DBFFF714
:10BF7800BFFF0135064649F100092D18DAE9002707
:10BF880049EBE0734FF00109C4E90453AD1843EBE2
:10BF98000707FFF7A5FFDFF8BCE00346DEF804A0BB
:10BFA800EBB9C4E900EACAF80040CEF8044028E03A
:10BFB800DAE900126FF001035B1A4FF0FF3161EB11
:10BFC80002025B1B62EB0902012B4FF0000972F1C0
:10BFD8000001BCBF01230022C0E90432D9E7D3E93C
:10BFE800041CD4E904208A4270EB0C0B24DA891A69
:10BFF8005A686CEB0000C3E90410C4E9003214600D
:10C008005C60FFF76DFF84420ED1134B1B685BB970
:10C01800B9F1000F02D1FFF76BFF064630462BF04F
:10C0280077FA0021FDF79AF988F31188BFF36F8F2B
:10C0380028463946BDE8F88F521A60EB0C009A453D
:10C04800C4E90420ADD01B68AAE700252F46EFE716
:10C05800E81C0024BC030024942100242DE9F047A7
:10C06800EFF31185102383F31288BFF36F8FDFF886
:10C07800A4900026DFF8A0800027C9F80000FFF789
:10C088002FFFD9F80030D8E900ECD91750B1D0E922
:10C098000442A34271EB020A1CDAE41A62EB0102C1
:10C0A800C0E9044213EB0E034FF000044CEB01010E
:10C0B8002046C9F80040C8E900312BF029FA21468A
:10C0C800FDF74CF985F31188BFF36F8FBDE8F04792
:10C0D800FFF7BABE14EB0E024CEBE473C0E9046739
:10C0E800C8E90023FFF70EFF85F31188BFF36F8FB0
:10C0F80083689847EFF31185102383F31288BFF301
:10C108006F8FD9F800301B1BC9F80030FFF7E8FE25
:10C11800B7E700BF94210024E81C002410B5EFF312
:10C128001184102383F31288BFF36F8FFFF7E0FEAB
:10C13800054A0346D2E90001181841EBE37184F37C
:10C148001188BFF36F8F10BDE81C0024F8B50646B0
:10C15800EFF31187102383F31288BFF36F8F026800
:10C1680022B187F31188BFF36F8FF8BDD0E90A5465
:10C17800691C44F10003022973F1000334D3013D23
:10C1880044F1FF34002CBCBF15462C462BF003FAB3
:10C19800013041F10001401944EB0101012871F11E
:10C1A80000014ADB2BF0F7F901306FF0020341F18F
:10C1B8000001401944EB010183426FF000438B41B9
:10C1C80040DB2BF0E8F901306FF001024FF0FF334C
:10C1D80041F10001401944EB0104121A63EB040316
:10C1E8001A493046FFF7AAFE336B01333363336ACB
:10C1F8006BB187F31188BFF36F8F336A3046984766
:10C20800EFF31187102383F31288BFF36F8F334640
:10C2180053F8184F9C42A4D0002CA2D020462BF0F3
:10C228008CF80023C4F8983087F31188BFF36F8F18
:10C238002046BDE8F8402BF071B86FF001024FF0CE
:10C24800FF33CDE700224FF00043C9E755C1009006
:10C258002DE9F04105461C4690461F46EFF311862E
:10C26800102383F31288BFF36F8FB4F1FF3F08BF29
:10C27800B2F1FF3F05D186F31188BFF36F8FBDE898
:10C28800F081002C09DB012A74F10003BCBF0122F4
:10C29800002412F1FF3844F1FF3728462BF04FF9FC
:10C2A800002342462B633B46DDE90601C5E90A0146
:10C2B80028460249FFF742FEDDE700BF55C100905E
:10C2C80038B50346EFF31185102282F31288BFF3C5
:10C2D8006F8FC160012181600068834206D185F3B8
:10C2E8001188BFF36F8F0024204638BDD0E9003293
:10C2F80013605A600023C0E900332BF0BCF92946CB
:10C3080004460248FFF762FBEEE700BFA4280024BA
:10C31800F8B507460C4616462AF0BBFF08B10020C0
:10C32800F8BD0E4B9B68D3F88C50002DF7D0221D1A
:10C33800F5D2EFF31184102383F31288BFF36F8FC4
:10C3480047F004012846B04784F31188BFF36F8F84
:10C358000028E4D040F8045BE2E700BF6021002435
:10C368000146024A0020FFF7D3BF00BF713C03908B
:10C37800014827F0E3BD00BF65600590074B07B58E
:10C388004FF48062009306494FF0FF330548FFF7EA
:10C3980079F8002003B05DF804FB00BF70A1049099
:10C3A800C0A30024F01C00240428F0B504468BB078
:10C3B8002BD0344D286818B114F05EFE00232B6092
:10C3C8001CB3314B9C4220D001AB0026214602A869
:10C3D80002932E4B019603932EF018FF01983146D5
:10C3E800013014F029FE0246286070B106AF0199A9
:10C3F80038462DF05BFA264B214604A8059304978E
:10C408002EF004FF2A68019BD654224D02F0EEFB61
:10C4180032F0FCFA2BF04EFA01F04EFF1E4B0022D0
:10C42800D5F8F0401A7084B120460EF021FC30B3E4
:10C43800A06804F0F1FBD5F8F040002CF4D1D5F851
:10C44800F0301C46DB68002BFBD1C5F8EC4000251A
:10C45800124C01F0DDFA08F0CFFA0EF0FBFC206870
:10C4680014F00AFE25600E4C206814F005FE2560C5
:10C478002BF09AF90BB0BDE8F0402BF018BAE4683D
:10C48800DBE700BFF02200246C23002461770390CF
:10C498002D980390F4220024A4280024D4210024F9
:10C4A800D021002470B5164B0022044600EB81050C
:10C4B8009A60C3E900222646043430682DF076F9E4
:10C4C800022818D130680F4C206098B10E482BF024
:10C4D8006AFC20682BF090F90C4802F0B9F902F0D8
:10C4E80007F9074920682BF082F90023236002F03E
:10C4F800FFF8012070BDA542DDD10020E3E700BFB1
:10C508009C210024CC210024FC61059066B505908F
:10C5180010B5044608482BF06FF902F0A5F840B1B1
:10C52800064802F095F934B10548BDE8104002F01C
:10C538008FB90448F5E710BDFC61059051B305902B
:10C5480016AE05907EB3059073B506462BF0AFF98D
:10C5580008F00CF814F06EFC054614F077FC04465D
:10C5680008F00CF8641B0025A4F58060244C08F042
:10C578000BF801F0A1FE00F053FC6B464FF400628B
:10C588002049304600952BF0EBF81F4B0146186008
:10C59800009B194409F094FD4FF4005201AB1B496C
:10C5A800304601952BF0DCF8194B01461860019BC9
:10C5B80019440EF02FFB05F05FFD2946D4F8E8007A
:10C5C80012F076FB1621D4F8E80030F067FF6621F8
:10C5D800D4F8E80030F062FF40F6B651D4F8E8002D
:10C5E80030F05CFF294604F1D80012F061FB0948DD
:10C5F80003F050FF084B01221A7002B070BD00BF53
:10C60800F42200249C600590D0210024B36005909A
:10C61800D4210024634D0590A428002409282DE97D
:10C62800F0470446A4B000F08B8001F05FFE0028BC
:10C638007DD0002C7BD1444BD3F8F030002B76D042
:10C6480002AD2046DFF80481FFF77EFF02F0BAF85A
:10C658004FF400712846DFF8F8A02DF00CF9C8F85F
:10C66800005001F04BFE0121064600F180072BF037
:10C67800E4F9384B384A06AD384939482DF09AFA6A
:10C68800DFF8DC9006A800F035FB364934482DF079
:10C69800B6FA013415F8012B514648462DF0AFFA89
:10C6A800202CF6D130492E482DF084FA32F0AFF91B
:10C6B80002212E48FFF7F6FE0023C8F8003002F0EA
:10C6C80087F801232A4A0EA9384633F03CF9A0B965
:10C6D80002982FF0F2FA039A0446014601AB0132A0
:10C6E8000EA833F056FA40B9039A019B9A4204D136
:10C6F800214604983CF004FDA0B14FF47A702BF069
:10C70800E7F90A231A4A0EA9384633F01CF901AB97
:10C718000EA8DDE9032133F0EEFA0EA833F053FC3E
:10C7280001F0CAFD002130462BF087F902E02046CF
:10C73800FFF70AFF0F4C6068FFF736FE00236360BF
:10C7480024B0BDE8F08700BFF4220024982100241B
:10C7580053B50590CD600590DE6005903D6105906C
:10C7680050CA049005AD0590089F0590ACA10490AF
:10C778004D6105909C2100242DE9F04F89B00746B2
:10C788002BF0ECFA804640B1B0482BF00CFB384651
:10C79800FFF7BEFE384601F013FADFF8B492CDF881
:10C7A8000880002F40D0D9F80030B3F5007F40F062
:10C7B800D580002520262C464FF002094FF4401B57
:10C7C8002BF082F94FF4C873039003FB09F3049329
:10C7D80003F59C5308330093002C40F07481A24663
:10C7E8004FF0010901F0E2F801F044FF054601901D
:10C7F800002800F0BB8046F0100601F00DFF954CB4
:10C80800206828B103781E4002D114F035FC266058
:10C81800BAF1000F04D0002001F0D0FD01F0C8FDEE
:10C82800284609B0BDE8F08F01F046FD01F040FF51
:10C838000546002840F08480864EFFF785FE336861
:10C84800002B5DD01A7822F020021A7033689A689B
:10C858001C78127892B1586808B103F01BFE33684F
:10C86800012107A89B680793FFF71CFE98B9336856
:10C8780098682BF098FA784801F0EAFF0421774885
:10C88800FFF710FE38B908217548FFF70BFE10B105
:10C89800744801F0DDFFD9F800301B0532D501F0EE
:10C8A80009F801282ED1704801F0D2FF4FF0000A94
:10C8B8006E4BD9F8040083F800A0FFF775FD3268C5
:10C8C800C9F804A02AB11378980644BF43F020039E
:10C8D8001370D9F80030190516D500F0EBFF441E87
:10C8E8004FF0300618BF0124D9F80030DA051AD500
:10C8F800B3F5007F4FF001043FF45EAFA1462AE094
:10C908003C46BBE75A48CFE71BB904F0010424268C
:10C91800EAE714F002044FF028061CBF83F4806392
:10C92800C3F38024E0E7B3F5007F254615BF4FF039
:10C9380001094FF002094FF4405B4FF4401B3FE7F9
:10C94800D9F80030B3F5007F3FF433AF3D463C469D
:10C9580020264FF001094FF4405B31E700252026DF
:10C968004FF00309DFF80CB12C4629E72BF0F6F954
:10C97800059080B12BF00FFA68B101F099FE0546D9
:10C9880048B92BF0F8F904287FF439AF032000F0F8
:10C9980097FF059D33E7CCB92BF0E0F90546A8B120
:10C9A80001F086FE90B9B8F1000F02D13846FFF7C2
:10C9B800AFFD029B13B9384601F002F923482C4613
:10C9C8002BF0F1F92C4801F043FF02952BF0C6F942
:10C9D8000546002814BF45462C46B9F1000F05D07E
:10C9E80001F066FE10B902F063FE81462BF06CF888
:10C9F800039B049A8046C31A9A423FD94FF4C871E0
:10CA0800B3FBF1F201FB1238B8F1630F11D9BAF197
:10CA1800000F04D0002001F0D1FC01F0C9FCC8F5DA
:10CA2800C870B9F1000F47D114F034FA14F07CFA49
:10CA38002CE0BAF1000F04D101F0DAFC584601F0FD
:10CA4800BDFC0123C8F164000193EAE77762059011
:10CA58009C210024EC2200246DB505909CA1049033
:10CA68007CA1049034AC0590A8AB0590A4280024C0
:10CA7800C1AB05900030300095AE0590009A9A42FF
:10CA880008D22BF021F8CDF804A00390DDF804A01B
:10CA9800A846A7E6BAF1000F04D0002001F08EFCEA
:10CAA80001F086FC009B039A1344A3EB0800B9F13C
:10CAB800000F05D00028E9D0484528BF4846B3E70D
:10CAC8000028E3D0B0E74FF0000A98E607B5114A0E
:10CAD800114B1068596820B103B05DF804EB2BF0D6
:10CAE80062B91A6892050ED59A68002A0BDD51B111
:10CAF80009680C330948C988009109492DF05AF88A
:10CB080003B05DF804FB074803B05DF804EB01F0DF
:10CB18009FBE00BFCC2100249C21002450CA049051
:10CB28005B610590DAB105902DE9F74314F066F9D9
:10CB380000F0B4FF2AF038FE14F018FA2BF013F8BE
:10CB480001F0D2FC52482AF057FE00F0A1FF18B9B4
:10CB580000F0AAFF00F0A2FF2BF048F901F042FE16
:10CB680000F096FFB0FA80F00021400901F0ECFADD
:10CB780010B9082000F092FF31F048FF2AF09AFE21
:10CB880000F0D0FE02F07EF941482AF035FE002080
:10CB980000F096FE00F07CFF08B901F043FD01208B
:10CBA800012501F09DFB002001F094FB4FF48074F7
:10CBB80000F06EFF374EFFF731FD374F2AF078FE51
:10CBC800012001F089FDDFF8D480284614F41069AB
:10CBD80055D015B9384601F03BFE3578002D3CD1CB
:10CBE80000F056FFFFF7C8FD0028EFD100F050FF16
:10CBF800044601F061FB2046FFF7A6FC012001F086
:10CC080023FD00F045FF28B9254B012101A8019318
:10CC1800FFF748FC01F0ECFB404601F0CFFB01F0C8
:10CC2800C7FB3378012B1AD101F0CCFD00F0BEFC14
:10CC3800044601F0CDFD0420FFF7B6FB01F0D8FB58
:10CC4800002001F0BBFB01F0B3FB012001F004FD63
:10CC5800032000F035FE0020B8E70025C6E7114B99
:10CC6800DFF84490C9F8003001F042FD00F02EFDD5
:10CC780000230446C9F8003001F03AFDDBE7002C38
:10CC8800B2D02DF0EEF8484603B0BDE8F08300BFFF
:10CC9800FC610590A5280024D6A30590303030000B
:10CCA800646105906C610590CC21002408B50DF0F5
:10CCB800EFFF00F035FB042106482EF06BFE2AF04A
:10CCC8006BFF00F0D9FE02F017F8BDE808400DF040
:10CCD800F3BF00BFE4230024014B1878704700BF5E
:10CCE800A42800240048704700389C1C004870475E
:10CCF8003333534038B505462021FBF71BFF041E8C
:10CD080011DA21460024094827F018F92146202283
:10CD1800074827F013F9C4F1200228190021BDE8BB
:10CD280038403CF0E5B91F2CF0DD38BD05620590B0
:10CD38001F6205900428034607B506D801460F4828
:10CD480003B05DF804EB01F013BC06210C4A6846F9
:10CD580024F066FB011E0DDD052901DD27F0BFFD6E
:10CD680001F108034422013168466B4403F8082C9A
:10CD780001F0FEFB03B05DF804FB00BF46620590BE
:10CD88004B620590F8B5244DAB7DDB0732D52E6894
:10CD9800706801282ED9B168431ECA5C0A2A29D1B5
:10CDA8004A1E002B01DC1A4608E0D45C0A2CFAD093
:10CDB800013BF6E78C5C202C02D101329042F9D875
:10CDC800002B0CDD541CA04209D15C1E0C44A1426E
:10CDD80005D014F8017D0A2F0CD0202FF7D001447C
:10CDE800D21A0E4F11F8023C94083A2B08BF0134AE
:10CDF800013C00D2F8BD0422394630462CF012FD21
:10CE08000421384601F0B4FB2B6904332B61AB7D58
:10CE180043F00203AB75EBE7D8210024E0B7059097
:10CE28002022002101483CF063B900BFAC23002454
:10CE380038B500220B4C05460846A2606B6862753F
:10CE48004FF0FF3263602560A161C4E903232AF033
:10CE5800D3FC6B680BB90123A375BDE83840FFF715
:10CE680091BF00BFD8210024F8B503780446DBB190
:10CE78000E4FD7F8B80018B12146F4F771FC98B1F5
:10CE88002046F4F77FFC461C30462EF019FF054675
:10CE980050B1324621463CF003F905491C22081DD1
:10CEA8003CF00CF9C7F8B850F8BD00BFF4220024D4
:10CEB800AC2300242DE9F347AB4C06462368D3E99D
:10CEC800011030F0CBF8A5680746002D40F03881F6
:10CED800731E042B1AD8D4E900325B689A4278D0C2
:10CEE800012E15D1236865689868D4F8108000EB86
:10CEF80008012844A8EB050800252AF060FC06462E
:10CF0800A845A56040F3BA80A946A8E00D2E13DC19
:10CF1800022E40F3B380F31E0A2B00F28F80DFE865
:10CF280013F058008D00CD018D008D005F008D003D
:10CF38008D008D003D004D001B2E4ED07F2E4FD012
:10CF4800A37D99077FD41F2E40F39880206821691C
:10CF580083685A5C06F0C003802B16BFF2B2237DAB
:10CF6800002302F1400508BF0133EDB208BFDBB270
:10CF7800372D194423759BBFD208E525002502F0FB
:10CF8800060298BF1541324698BF05F003052CF0FC
:10CF980033FD237DAB4271D1013596E073482AF009
:10CFA8002BFCA0692AF028FC226863682169906834
:10CFB800C91A184401F0DCFA002586E06C480026FE
:10CFC8002AF01AFC20682CF0A6FC63681844FFF7C6
:10CFD8004BFF304602B0BDE8F0870123A3604DE067
:10CFE800226961688A4249D92068561A0023D0F814
:10CFF80008E0B34203EB010C17D1032BCCBF042686
:10D008000126961B33461EF803C01946013B0CF057
:10D01800C00CBCF1800FF6D0A2EB0108761A42468C
:10D028002CF0F7FC4FF0010919E01EF80CC0BCF118
:10D03800200F01D10133DCE70126E2E7A37D9A073F
:10D0480023D5092E18D0202E7FF47DAF00264FF06F
:10D05800030803212068B146A6752CF0D3FCA8EB81
:10D068000600FFF767FE2369A3EB08032361B9F104
:10D07800000F00F0298128E00023A375A37D4FF05D
:10D08800FF3623F00203A375A3E7092E7FF45BAFF5
:10D0980022682169D2E90123002A40D00B4413F801
:10D0A800010C10F023FA002839D0324B04250193E3
:10D0B8000026019B21695A1C2068314401360192DF
:10D0C8001A782CF093FCB542F3D12368D3E9011008
:10D0D8002FF0C4FFB84203D20321274801F048FAD1
:10D0E80023682769D3F80880D3F80490781908EBE7
:10D0F800090140442AF063FBA9EB0701064608EB47
:10D10800070001F035FA236822695B689B1A5B1BEC
:10D11800981BFFF70FFE23692B442361AEE72368B2
:10D1280060689D6801AB2169144A091A28440BF00C
:10D1380095FA05460028A1D0431C3FF432AFB7E763
:10D14800013D032D00F2E880DFE815F004001A0025
:10D15800A000E1004F2E04D05B2E40F0DD800223BA
:10D168003CE704233AE700BFD82100245062059029
:10D1780077620590E0B705905962059050CA04900F
:10D18800A6F13003092B03D803236675A36075E75E
:10D198000023412EA3602ED1E368062B3FF76EAF24
:10D1A80003F1010A5D4D2D3305EB8305AB68002BB8
:10D1B8003FF464AFD4F80080D4F80490D8F808009D
:10D1C8002169014448442AF0FAFAC8F8049006464E
:10D1D800A9684046C4F80CA02CF0FBFB63682269E0
:10D1E800A2EB03082268B8F1000F5568A5EB030508
:10D1F8007FF76BAF16E7423E062E3FF63FAF01A31F
:10D2080053F826F029D200906FD200907FD2009078
:10D2180085D00090C5D2009085D00090EDCE0090CA
:10D22800E568002DFFF62AAFD4F80080013DD4F858
:10D238000490D8F808002169014448442AF0BFFA4C
:10D24800D8F8041006464046A1EB0901E5602CF029
:10D25800D9FBE268002AC1DB304B206803EB82036C
:10D26800D3F8B810B8E7236822695B689A42BFF41C
:10D2780005AF01252BE0226963689A427FF6FEAE6E
:10D2880000254FF00108A9462E46E8E67E2E43D138
:10D29800637D312B3FF426AE333B052B3CD801A2EE
:10D2A80052F823F0E7D20090C5D2009021D3009025
:10D2B80021D30090EDCE0090C5D2009023685D6820
:10D2C8002369ED1A0023A360002D7FF7D7AE2368EA
:10D2D800294698682369184401F04AF91BE7206831
:10D2E80021694368994217D285685B1A01220D4467
:10D2F80015F8016F06F0C006802E01D19A4204D1BC
:10D308002CF087FB0023A36056E60132F0E7462E97
:10D31800D4D0482E3FF4E6AD00235FE6F422002483
:10D328002DE9F04F0B4B8BB019686846CDF820C03B
:10D33800091ACDF824D08908CDE90045CDE902675E
:10D34800CDE90489CDE906AB2EF024FB0BB0BDE88E
:10D35800F08F00BFF422002470B5067804461EB191
:10D368004FF0FF35284670BD2AF027FDC31E05463D
:10D37800012B0CD801210C48217001F0F9F8032D7C
:10D38800EED10A48836E60309E600EF0EBFAA388F7
:10D39800013B9BB2A380002BE4D10121044801F09A
:10D3A800E7F86388A380DDE75D620590F422002436
:10D3B8007B6205902DE9F04391B017461D46002386
:10D3C800044603A80493884607F001060EF0B6FA4F
:10D3D800034600285BD1F90641D5DC20D4E90121B8
:10D3E8002CF0F3FF0446B8F1010FD4F8009007D1F0
:10D3F8004FEA09114FF4437041F0060104F0A4FE0E
:10D408002146424601A811F04FF9C7F38002494668
:10D4180001A80FF09BFEB8F1010F044601D1FFF7F8
:10D4280045FC380602D4032000F0FCF914B120466C
:10D438002CF04FFD4FF0FF3000F0F4F9012012F00E
:10D44800C9FE07F069F8EEB9CDB900241EB1012173
:10D45800474801F08DF8204611B0BDE8F0837A0600
:10D4680005D5DC2094E80E002CF067FFBAE7BB0670
:10D47800B9D520462CF087FE2CF0B5FFB2E7002383
:10D488002B60E2E701213A4801F072F8DCE74FF03F
:10D49800FF3000F0C7F9022012F09CFE790602D591
:10D4A800A368206898471EB10121314801F060F84F
:10D4B800049C20460BF0A4FE2E490DF083F90028A9
:10D4C80041D004982DF0A2FA0E283AD0C20705D40C
:10D4D80083072BD10268284B9A4227D12DF052FDA1
:10D4E80040F48074002DB1D0049F4FF0FF332C60BE
:10D4F80038466F60AB602DF074FA0028A6D001AAF8
:10D50800694638462DF09CFA019B002B9ED05A683C
:10D51800AA60002285F82C2018682CF054FE2022DE
:10D52800014605F10C003BF01AFE8FE70146002288
:10D5380012480BF081FE124910482CF0B8FA01206D
:10D54800CEE70020CCE70F4B9C420DD004990B4846
:10D558002DF05CFE049B0C4918680DF033F908B1F6
:10D568008224BFE70124BDE74FF40064BAE700BF97
:10D578005D62059058F004904800059050CA0490E8
:10D58800089F05906C23002434F0049008B50378B4
:10D598004BB901210170044800F0EAFF2AF00DFCA4
:10D5A80003380128FAD808BD5D6205902DE9F043DB
:10D5B8008BB0DFF8F48000263C4F202106A82CF021
:10D5C8005AF940462AF018F9384607962AF014F90D
:10D5D8002AF0F3FB0128044635D107990229F0D136
:10D5E800089B1A78052AECD193F80190B9F1410FFC
:10D5F80006D02F4800F0BCFF00232C480793E5E72E
:10D6080080252C4800F0B4FF03216846ADF800508F
:10D618008DF8024000F0ACFF01AA0023214603A8C0
:10D628000392254A8DF804300492244AADF8065036
:10D6380005924A46ADF80850FFF7BCFEC305DBD596
:10D648000BB0BDE8F083022809D11D482AF0D4F8B0
:10D6580006A82CF032F900201A4B1870F0E70328BE
:10D6680002D100230793B3E7042804D0C1B206A867
:10D678002CF060F9ACE714482AF0BEF8079B43B9D0
:10D688000F482AF0B9F806A82CF017F94FF4807063
:10D69800D6E700231122012106A8FFF78BFE10F41C
:10D6A800106F91D0CCE700BF5F620590159F059081
:10D6B800209904907A62059061D3009095D50090E6
:10D6C80077620590A52800247D6205902DE9F04138
:10D6D80092B04B4EDFF82C81202101A82CF0CBF81A
:10D6E8003046494F2AF088F848482AF085F83046ED
:10D6F8002AF082F8BA8A002302B1BB8205A80293F5
:10D7080006930EF01BF9044690B9414901A82AF086
:10D7180064F8012805462CD139482AF06DF801A88B
:10D728002CF0CBF83B4B20461D7012B0BDE8F081C1
:10D73800022012F04FFD30462AF05EF8069936486E
:10D748002DF064FD029B002BD4D001A82CF0E3F847
:10D758000AF0C0FE58B10A2101A82CF0EBF84146A6
:10D7680001A82AF03AF803280BD00428EDD10021AB
:10D778002CE0022803D122482AF03EF8B0E703281B
:10D7880001D1304619E0042808D11D482AF034F8A0
:10D7980001A82CF092F84FF48070C6E70528D1D183
:10D7A8001E482AF029F802941D4C2AF006FBC1B243
:10D7B80003298DF8031003D111482AF01DF899E7C1
:10D7C80004290CD10E482AF017F80121002316224B
:10D7D80001A8FFF7EFFD10F4106F8BD0A5E701A8A3
:10D7E8002CF0A8F89DF803300D2B03D120462AF021
:10D7F80003F8DAE701210DF1030000F0B9FED4E7E0
:10D8080077620590BC620590F4220024DE600590E2
:10D8180080620590A528002450CA0490856205906E
:10D82800B5620590014B1860704700BFC40300241F
:10D83800024B986A003818BF01207047F422002470
:10D848002DE9F04106460D4600270DB9BDE8F081E7
:10D8580033780A2B16D1AFB9012401210F4800F003
:10D8680087FE06EB040843461FB998F800200A2AE9
:10D8780001D0A54208D1304621462D1B464600F06E
:10D8880077FEE2E70024ECE71F7808F1010801348D
:10D89800A7F10D035F425F41E5E700BFC162059054
:10D8A800024B034819782FF042BF00BFA628002476
:10D8B800CCC70490014B1878704700BFA6280024F5
:10D8C800014B1870704700BFA628002410B5064CFD
:10D8D80020680E2806D1054B80220549054801F02D
:10D8E8005BF8206010BD00BFC8030024A7280024EF
:10D8F80030960490B01D002410B5064C20680E2800
:10D9080006D1054B80220549054801F045F82060FD
:10D9180010BD00BFCC030024272900244C96049096
:10D92800001E002470B501F027FA044698B10A4B8E
:10D9380003600A48FDF718F8054660B129F04FFA68
:10D9480048B1074B29462046002223600123BDE841
:10D95800704003F069B870BD88F60490C759059007
:10D96800C0C8049010B5044602F0E8FBE3681BB990
:10D978000C4A1168A14203D1BDE8104002F0F8BB7F
:10D98800A360094B1968E160196809B119688C60CE
:10D99800116801B914601C6002F0EAFB13F044FA44
:10D9A80010BD00BFFC210024F82100242DE9F0411E
:10D9B800144E33F01AFD33680BB3134D02F0BEFB5F
:10D9C8002C681CB1BDE8F04102F0D2BB01230F4A1C
:10D9D8002B603368346014601BB92B68013B2B60E3
:10D9E800F0E7D3E900689F68C3E9024402F0C0FB8E
:10D9F8000EB14046B04702F0A1FB3B46ECE7BDE85C
:10DA0800F08100BFFC210024F4210024F821002427
:10DA18002DE9F7430025154E01AF0195A84602F000
:10DA28008DFB346854B9019B3360114B1D60114B59
:10DA38001C6003B0BDE8F04302F09ABBD4F808902C
:10DA48002046C4F808800DF013F918B10023E360EC
:10DA58004C46E7E760680DF00BF90028F6D12B4635
:10DA68003C60254604F10807F1E700BFFC210024CB
:10DA7800F8210024F4210024044B10B51C6804B9D3
:10DA880010BD60682DF0BAFFA468F8E7FC210024F7
:10DA9800014B1878704700BFA7290024014B187064
:10DAA800704700BFA72900242DE9F04130F0B1FFED
:10DAB800044620F47F00284B284E20F47F409842EB
:10DAC8000AD114F47F4FC4F3072505D030F0A0FF26
:10DAD80035702846BDE8F0810023337029F06DFECB
:10DAE80028B1062833D85423C340DB072FD51C4858
:10DAF80030F08EFFDFF86C8000F07AFC29F0D5FF5B
:10DB0800064600200F460146FA220023F3F70EFED0
:10DB18007D2A73F1000334BF4046002000F04EFC1C
:10DB28002AF038F8054648B929F0BFFF801B61EB99
:10DB38000701B0F57A7F71F10003E5D3002000F00A
:10DB48003DFC00F035FC25B9204630F061FF00258A
:10DB5800BFE71125BDE700BFAF0000ADA72900242E
:10DB6800AF1100AD00303000024B43EA002030F026
:10DB78004FBF00BFAF0000AD0D4D044608B52B7870
:10DB8800012B0FD901280DD90A4826F0D7F92146CB
:10DB9800094826F0D3F92978084826F0CFF926F065
:10DBA80080FEFCE72046FFF7DFFF30F02BFF00BFC9
:10DBB800A7290024C3620590D9620590E562059003
:10DBC80010B50446002838D01C4800F041FE631EFA
:10DBD800112B12D8DFE803F02D1111111111112B9F
:10DBE8001129111127212523091F154800F030FE9E
:10DBF8001448BDE8104000F02BBE023C124800F06B
:10DC080027FEE4B20A2C16D8104B53F8240000F073
:10DC18001FFE0F48EAE70F48E8E70F48E6E70F4816
:10DC2800E4E70F48E2E70F48E0E70F48DEE70F4870
:10DC3800DCE70F48DAE70F48E9E710BD53AB05907A
:10DC4800DBAB059067AB059055B2059028C00490F2
:10DC580078AB0590A7B005901CB30590D5AC05909E
:10DC6800EBAC0590D7AD0590BBAD0590BDB2059066
:10DC7800B5AE059091AC05900129024610B50C4649
:10DC880017D9042915D00B490B482BF0B8FF022CE3
:10DC980003D0052C0BD0094900E0094906482BF0B0
:10DCA800AEFF08490448BDE810402BF083BF064981
:10DCB800F4E710BD8AB3059050CA0490B8B0059037
:10DCC80068B00590089F059073B005902DE9F04F56
:10DCD8009DB080460C46924600AF00F00FFB28B975
:10DCE800012528467437BD46BDE8F08F01239F4AB9
:10DCF80007F11801803031F026FE0028F0D1D7E96D
:10DD08001402D7E90A139A4208BF884200F02B810F
:10DD180097F84930002B40F0268107F1180029F0C8
:10DD2800D9FD5B28064606D107F11800D7E90A2372
:10DD380032F01EFAE3E7002EF6D008F1FF3919F8A1
:10DD4800015F2DBB30460FF0D1FB20B107F1180061
:10DD580029F0C0FD06463D2E1CD107F1180029F018
:10DD6800B9FD22280CBF012300238AF8003040F0B7
:10DD7800CA8007F1180029F09EFD22282AD016D85B
:10DD880030B30A2824D0C1B2204629F0BBFDF0E701
:10DD9800B54206D00A2EB2D007F1180029F0A9FD25
:10DDA800ADE707F1180029F086FD0646C7E75C28AD
:10DDB800E9D107F1180029F07EFD7628E3D861281B
:10DDC8001DD80A2804D0552800F089800028DAD107
:10DDD800052509E007F1180029F07CFD0A2803D081
:10DDE800232807D00028F3D1EDB207F1180032F04C
:10DDF800EAF876E707F1180029F07BFDF4E7A0F1CF
:10DE08006203142BBFD801A252F823F00BDF009055
:10DE18008FDD00908FDD00908FDD009079DE00901F
:10DE28008FDD00908FDD00908FDD00908FDD0090FA
:10DE38008FDD00908FDD00908FDD00906DDE00900B
:10DE48008FDD00908FDD00908FDD009069DE0090FF
:10DE58008FDD009071DE00907DDE009075DE009011
:10DE68000D2090E70A208EE709208CE70B208AE72F
:10DE78000C2088E73B1D6E464FF004099B46D846A8
:10DE880009EB0B0A07F1180029F015FD08F8010B3A
:10DE9800D045F7D100233946102258460BF80930EF
:10DEA80023F05EFB3B680146434528D1B0F5881F47
:10DEB80022D27F281AD9B0F5006F19D3B0F5803F68
:10DEC80034BF03230423227B22B1626813442268EF
:10DED8009A420FD920462BF034FDB54649E707F1A1
:10DEE8000C036E464FF008099B46C8E70123EAE792
:10DEF8000223E8E76360F0E70225B54674E7B54614
:10DF080066E708203FE70A283FF462AF00283FF49D
:10DF18005FAF00250D281CD009DC092819D00A2874
:10DF280000D040B963685B1B636000255CE720286C
:10DF38000FD0232805D0C1B22046002529F0E2FCE5
:10DF48000CE0636807F118005B1B636029F0D1FCE3
:10DF5800EBE70135C1B2204629F0D4FC07F11800DF
:10DF680029F0A9FCD6E704253FE700BFFC6205902D
:10DF780070B586B00E4610220DF1070302A929F0EC
:10DF8800CCFC044648B99DF807507DB9084902A859
:10DF9800F3F7E6FB20B901253570204606B070BDC1
:10DFA800044902A8F3F7DCFB0028F5D00524F4E7C0
:10DFB8000B630590106305902DE9F0418EB00E4675
:10DFC800302202AC0DF10303214629F0A6FC0546D8
:10DFD80028B99DF80380B8F1000F04D0052528461C
:10DFE8000EB0BDE8F0812046F3F7CCFB2718A74216
:10DFF8000CD99DF808302B2B01D02D2B06D12D3BA9
:10E008000DF10904D3F1000848EB0308391B022974
:10E0180021DD2378692B13D163786E2B1BD1A3786C
:10E02800662B18D1E01C4FF0FF430193B842D5D1BD
:10E03800019BB8F1000F01D003F100433360CEE734
:10E048006E2B08D16378612B05D1A3786E2B02D192
:10E05800E01C054BE9E701AA204606F055FB00281D
:10E06800BCD08442E2D1B9E70000C07F70B588B067
:10E0780004460E46202104A82BF0FDFB0DF10602F4
:10E0880004A92046FFF722FE054630B99DF8063060
:10E0980033B104A808F09AFC3060284608B070BD77
:10E0A8000DF107012046FFF763FF30B99DF80730EF
:10E0B800002B0CBF1E203E20EEE702A9204629F0C7
:10E0C80051FC18B902982CF020FFE5E703A9204677
:10E0D800FFF772FF70B9039C21462046F3F77AFADE
:10E0E80030B924F0030444F00204A4F1FF40D3E75C
:10E0F8000148D1E70525D0E70200400010B5064CDD
:10E1080023783BB1054B4FF47A721A6000F0B6F9E8
:10E118000023237010BD00BFA8290024D0030024C9
:10E12800074B1A683AB11A68012A05D105490A70DD
:10E138004FF47A721A6070471A68013AFAE700BF1A
:10E14800D0030024A82900242DE9F0414D4E4FF0BA
:10E158000008ADF5287D07464B4C30460D46A6F81D
:10E16800048000F099F906F18000C4F8048031F0C9
:10E17800E6FB0D2806D13FB935B900200DF5287DFD
:10E18800BDE8F081002D79D04FF4007300220721FB
:10E198003E48009328AB14F093F80028EDD100F026
:10E1A8006DF93B49394813F0A3FF0028E5D13949F7
:10E1B800364832F0B9FA384B03AA03F13807186821
:10E1C800083353F8041C1546BB4203C52A46F6D14A
:10E1D8001B8812A9314A2B8039232C4802930A2321
:10E1E80031F0B1FB02AB029A03A912A831F083FD0A
:10E1F80012A831F0E8FE0A23294A12A9234831F06F
:10E20800A2FB12A831F0DFFE264B03AA03F1100788
:10E218001868083353F8041C1546BB4203C52A4640
:10E22800F6D1186899889B792860AB711623A98064
:10E2380012A91D4A02930A23144831F084FB02AB49
:10E2480003A91A6812A831F056FD12A831F0BBFED6
:10E2580016490E4832F068FA00288ED100F00EF9FF
:10E26800134B012523600023E360124BC4E90156D8
:10E27800C3E93B442AF060FC28467FE70028EFD03A
:10E288007BE700BF800D002400220024000E00243C
:10E298006A6B0590166305903C6305901A630590B8
:10E2A800FC620590766305902E63059037630590B0
:10E2B800634D0590F422002408B54FF47A72044B9C
:10E2C8001A6000F0DBF8BDE8084012F049BC00BF56
:10E2D800D00300240146014829F092BB800D002498
:10E2E8000146014829F09FBB800D0024024B586865
:10E2F800003818BF0120704700220024034B04484F
:10E308005B68002B08BF0020704700BF0022002474
:10E31800800D002408B533F065F829F069FD00F098
:10E32800CBFBFFF7EBFE33F05FF829F061FD00202F
:10E3380030F071FB034BC3E90001BDE8084033F03E
:10E3480052B800BF501E002408B5FFF7E9FE0022AE
:10E3580002490348BDE8084029F0A5BA1DE300902A
:10E368001422002410B5074C01F0E8FE23680BB90D
:10E3780012F07CFD236801332360BDE8104001F0F2
:10E38800F7BE00BF1022002408B501F0D7FE074BE6
:10E398001A6812B11A68013A1A601B680BB912F0B0
:10E3A80073FDBDE8084001F0E3BE00BF1022002461
:10E3B800014829F064BD00BF2822002438B5094D62
:10E3C80004462B6883420CD0074B197829F0B4FB1C
:10E3D800B0FA80F12C6049090448BDE8384000F0E3
:10E3E80031BB38BD24220024B5060024282200248D
:10E3F80038B50B4D2C7894B901230A490A482B707B
:10E4080000F004FB22462146074829F060FD074B2F
:10E418004FF0807218681A60FFF7D0FF2C7038BD73
:10E42800A929002440B20490282200242422002490
:10E43800014B1870704700BFB5060024014B1878CF
:10E44800704700BFB5060024F8B50E461C461546B1
:10E458006AB1094F3B781BB9FFF784FF01233B7072
:10E468002246691E3046BDE8F84012F003BC012B75
:10E4780094BF00200120F8BDAA29002410B5054C3E
:10E4880012F056FB23780BB1FFF77EFF00232370B1
:10E4980010BD00BFAA2900240F4B10B50360044625
:10E4A800838843F00503838030F0A0FA01230E220D
:10E4B8000A4984F88430231D616123610849A060FA
:10E4C800C4F88040E260A162C4E90823C4E90D23CE
:10E4D800044BE36310BD00BFE8040590A37B0390E1
:10E4E80051E40090057D039010B5054C23782BB9B5
:10E4F80029F024FC12F04AFE0123237010BD00BF4E
:10E50800AB29002473B505460C4669B10D4B1B7841
:10E518006BB90A4601AB01460B482AF067FD06466F
:10E528000A4B1B782BB13446204602B070BD0E460C
:10E53800F6E72146284629F009FC2146284612F02C
:10E548004DFEF0E7AC290024E0030024AD290024A7
:10E55800024B1A7818701046704700BFAD29002486
:10E56800024B1A7818701046704700BFAC29002477
:10E578002DE9F843DFF87C8000AF05460E4629F008
:10E58800F4FAD8F8003043B31B4829F032FCC0F540
:10E5980000720446D8F8000043689919914223D9BB
:10E5A8000734D21A2946E94624F007042BF03AF931
:10E5B8001148ADEB040DD8F80040694600F052F957
:10E5C800014620462BF005FA0A21D8F800002BF066
:10E5D800B1F90023C8F80030CD4631462846FFF788
:10E5E80091FFBD46BDE8F883324629462BF01AF95B
:10E5F800F3E700BF98210024CEAB059008B5FFF7DC
:10E608005FF9044B03F178029A62BDE8084012F002
:10E618000BBC00BFF4220024014B00221A60704793
:10E6280034220024034B01221A700022024B1A6084
:10E63800704700BFAE29002434220024014B002279
:10E648001A707047AE290024024A13680343136006
:10E65800704700BF38220024024A136823EA0003E7
:10E668001360704738220024014B1878704700BFA8
:10E67800AE29002410B50C4C206890B10B4B1B68D8
:10E6880083B929F021FA236883422368A0EB0300A9
:10E6980040F2EE2388BF00F1FF30984294BF00207B
:10E6A800012010BD0020FCE7342200243822002479
:10E6B800024B1868003818BF012070473422002424
:10E6C800034B1B7813B9034829F06DBB704700BF93
:10E6D800AF2900248D63059010B1034B01221A70F5
:10E6E8000248FFF73FB900BFB02900243C220024AC
:10E6F800F8B5254B1D7825B10120BDE8F840FFF796
:10E70800EBBF224B22481D702AF05DFB20482AF0FF
:10E7180040FB58B91E4801272AF04DFB80F0010440
:10E728000120FFF715FF0546E4B20AE029F016FBC1
:10E738000028EFD016482F462AF03DFB80F0010450
:10E74800E4B2F4B10120FFF70BFF0646114829F0A7
:10E758002AFB114829F027FBFEF7B8F90F4829F0E2
:10E7680022FB0F4829F01FFB0E4829F01CFB17B1AC
:10E778002846FFF7EDFE34B13046BDE8F840FFF714
:10E78800EFBE2646E2E7F8BDAF290024B0290024F1
:10E79800D803002494630590996305909E630590BF
:10E7A800A263059091630590044B1B7823B9044B31
:10E7B8001B780BB1FFF79CBF704700BFAF2900243F
:10E7C800B0290024014B01221A707047AF29002498
:10E7D800024B002202481A70FFF7C4B8AF29002480
:10E7E8003C220024034B044A04481A6000225A6061
:10E7F8002AF0E3BA3C220024B1E70090D8030024B1
:10E80800A1F180034F2B70B5064618D819460E485B
:10E818000E4C022310F8012B914205DA03FB014448
:10E82800E518A54205D870BD03FB0244891A0133D7
:10E83800F0E714F8011B3046FFF7E2FFF1E7BDE807
:10E8480070402BF07EB800BFB4630590BE6305909E
:10E858000246024902482BF0ADB900BFB1630590EA
:10E8680088FB04902DE9FF4105460A466846802446
:10E8780015F8011B274F0131DFF89C802BF016F8A3
:10E88800009E013E019B9E4205D868462BF043F846
:10E8980004B0BDE8F0810023184619461A4695F8D9
:10E8A80000C05200013114EA0C0FC9B214BF4FF076
:10E8B800010C4FF0000C64084CEA020204BF013559
:10E8C8008024824205D317F801C00CEB4000634452
:10E8D800E5E71B1A4244D15C012917D10B2300201C
:10E8E8002A784000144214BF01220022640840EA3A
:10E8F800020004BF01358024013BF1D101302BF027
:10E9080062FC014668462BF064F8BBE76846FFF7EF
:10E9180077FFB7E7E16505903B650590F7B50446D5
:10E928000D4683685B6CD3B9A3685B6BE3B9194F79
:10E93800A3689B69B3B101220DF1070120469847EE
:10E94800012806460ED19DF807203B689A4210D14F
:10E9580005F1080028F043FB11F02CFCE8E7984784
:10E968000028E1D103B0F0BD204698470028DED149
:10E97800F8E795F84830002BDAD1002200230DF192
:10E98800070105F1080028F023FB0028D0D085F8FE
:10E998004860CDE7C4030024F8B51E46174B04466B
:10E9A8000D461746C0E900318B68F3B19B6CE3B1A3
:10E9B80002461349284698473B460122314604F14E
:10E9C800080028F0F2FA4FF0FF324FF0FF33C4E9A5
:10E9D8000E23C4E91023002384F84830AB689B6AEF
:10E9E8000BB1284698472046F8BD6FF05703054AF3
:10E9F8000121054825F0DDFDDEE700BF54C0049085
:10EA080025E90090EE650590F897049038B50C4616
:10EA18000546084628F0CCFE6C60606828F0DFF9EF
:10EA280020B9074825F08AFA012038BD4FF4803212
:10EA3800217A606829F012FA0028F5D12872F4E7E3
:10EA48001D66059038B543680C460546012158688F
:10EA58001B7A994003691B68194214BF84F00103AB
:10EA680023464BB18368DB689847014610B10448D8
:10EA780025F064FA6C7238BD83681B69F4E700BF3F
:10EA88003466059038B501294368094A04460D469D
:10EA980018BF4FF40032197A586829F0DFF9014697
:10EAA80020B1044825F04AFA012038BDA572FCE7D8
:10EAB800060002004C66059008B5FEF7B9FE10B9CD
:10EAC800FFF7D8FDA8B108BD114A934203D1BDE8AC
:10EAD800084029F02CBE0F4A934203D1BDE80840F4
:10EAE80000F07EBD0C4A9342EDD1BDE808402AF003
:10EAF800FEBD0A480368002BE5D0094A9342E2D0DC
:10EB0800084A9342E0D1BDE8084032F09EBF00BFFA
:10EB1800B8C3049090C10490C0C80490581E002443
:10EB280088F604908C13059070B54FF0FF33244E8F
:10EB3800244C336023682BB933681BBBBDE8704095
:10EB480015F080BD204DAB42F6D0204A934204D147
:10EB5800204632F093FF2560EEE71D4A934203D129
:10EB6800204600F06DFDF6E71A4A934203D120468D
:10EB780001F0C8F8EFE7184A9342ECD1204602F0BA
:10EB88001FF8E8E7154C2368002BD7D00E4DAB4291
:10EB9800D4D0134A934204D1204629F0A3FA256021
:10EBA800CCE7104A934203D1204601F023FAF6E756
:10EBB8000D4A9342F3D1204601F02CFDEFE700BF48
:10EBC800D4030024581E002488F604908C13059062
:10EBD80090C10490B8C30490C0C804904C2200248B
:10EBE80030C3049034C5049084C70490F8B5374CFA
:10EBF800374E23680BB1B3420DD126603548036800
:10EC0800002B61D0B3425FD0334A934247D1BDE86D
:10EC1800F84016F0EFBF314A934216D16568A54215
:10EC280003D304F198039D42E8D928460CF020F854
:10EC38000028E3D02A4B6C22294618463AF030FACD
:10EC48006060284632F098FFD8E7264A93421FD1E1
:10EC58006568A54203D304F198039D42CED928469E
:10EC68000CF006F80028C9D01D4A2B4605F1200EE5
:10EC780094461868083353F8041C1746734503C7AD
:10EC88003A46F6D12846C4F804C033F0B6F8B5E7DA
:10EC9800154A9342B2D1204629F0D0FFAEE7134A75
:10ECA800934203D1BDE8F84000F0F6BC104A934205
:10ECB80003D1BDE8F84001F037B80E4A934203D1BA
:10ECC800BDE8F84001F08CBFF8BD00BF4C2200241D
:10ECD80088F60490581E00248C13059030C30490C5
:10ECE8005422002434C5049084C7049090C1049031
:10ECF800B8C30490C0C80490174808B503681BB986
:10ED0800164803684BB908BD154A9342F8D0154A0E
:10ED18009342F5D12AF026F8F2E7114A9342F2D04D
:10ED2800114A934203D1BDE8084032F0B6BE0F4AFB
:10ED3800934203D1BDE8084029F012BD0C4A934222
:10ED480003D1BDE8084029F063B90A4A9342DAD1F1
:10ED5800BDE808402AF0E4BC4C220024581E0024D8
:10ED680088F6049084C704908C130590B8C3049067
:10ED780090C10490C0C80490084B10B5084C1B689B
:10ED8800A34200D043B9074BB422002118463AF0F9
:10ED9800AFF940F8044D10BD0020FCE7581E0024D0
:10EDA80088F604905C1E002408B5FFF7E5FF10B94B
:10EDB800014803F0EFFA08BD22AD0590084B10B5E5
:10EDC8001B68084C0BB1A34208D1074B94220021C1
:10EDD80018463AF08DF940F8044D10BD0020FCE7C4
:10EDE8004C22002488F604905022002408B5FFF72E
:10EDF800E5FF10B9014803F0CDFA08BD28AD05902C
:10EE0800094B1B685A1C0DD0002B0BDCB82253434E
:10EE1800064A9818D358064A934203D0002B08BFD5
:10EE28000E2070470E207047D4030024581E00247B
:10EE380088F604900E2807B513D00E4A904213683E
:10EE480003D10D4A934200D093B90AF0D9F9C38887
:10EE5800E7224FF48A71009340F25513074803F0F4
:10EE6800D5FA4FF0FF33064A136003B05DF804FB90
:10EE78000023F8E7581E002488F60490EFB40590A4
:10EE8800D4030024074A1368013304D1064B074909
:10EE98001B688B4200D17047002BFCD00023136005
:10EEA800704700BFD4030024581E002488F604903D
:10EEB8002DE9F04F044685B01F464FF0000800F1D9
:10EEC8005009CDE90212B84502D305B0BDE8F08F6C
:10EED800039B03EB080694F8B530757896F901B0F2
:10EEE800002B37D0B57806F1030A484618F048F9E0
:10EEF800A8B3012300210093334694F8B620206D6F
:10EF0800D4F860C0E0470095534694F8B620012134
:10EF1800206DD4F860C0E047484633F060FABBF192
:10EF2800000F23DB00202AF0EFF9029B3BB1D4F855
:10EF38008430164A934202D0204628F0F8FFFEF7A4
:10EF480077FC0028C1D194F8B5304544DBB905F108
:10EF58000208B8E706F1020A05F07F05C5E7FEF7E3
:10EF680067FC0028C5D1FEF721FDBEE76B1C94F8AD
:10EF7800B520DDB256FA83F313445878FF2808BF4A
:10EF88004FF4FA70CFE705F103089CE788F6049080
:10EF9800F0B54B6B8BB005460C46002B00F0C980D2
:10EFA800012380F84030486B33F0A6FF85F83C0019
:10EFB800636B002B00F0C080A36B002B00F0BC80BB
:10EFC8004FF48073A5F84030A06B33F095FF85F8B7
:10EFD8003D00B4F85630002B16BF0123002304214E
:10EFE80085F8B43094F8573085F8423094F85630A4
:10EFF80085F8433008BF012394F8556018BF0026F0
:10F00800626B0CBF194633460AB9A26B32B1228E25
:10F01800B2F5807F02BF002602213346012205F1A6
:10F0280008000027CDE90422CDE90222CDE900132A
:10F03800638C228BE18A33F0A6FC94F85930089748
:10F0480005F15000099394F85430CDE90673638DA7
:10F058000593238D0493E38C0393A38C0293B4F953
:10F0680020300193B4F91E300093628BA38B216882
:10F0780017F0FEFFA38D3249A5F8AA3094F82E3078
:10F0880085F8B030238EA5F8AC3094F8323085F886
:10F09800B130606CF2F7D8F8F2F7D8FAA5F8A80002
:10F0A80094F84C30264985F8AF3085F8B270206D59
:10F0B800F2F7CAF8F2F7CAFAC5F8900094F8543093
:10F0C80085F8B36085F8B63063681D49C5F8943093
:10F0D8002389A5F8A030E068F2F7B6F8F2F7B6FA97
:10F0E800A5F8A6002369C5F89830A38AA5F8A23028
:10F0F800E36BC5F89C30B4F84030A5F8A430114B48
:10F10800C5F8843094F8583085F8B530A36C4BB105
:10F1180028460D4B40F8843FA16CFFF777FCA06CA4
:10F1280028F044FB094928460BB0BDE8F04028F018
:10F1380043BF80F840303BE7002385F8413048E77B
:10F1480000007A4488F6049074180590D4050024C9
:10F1580010B50B680446C0F894304B680549A0F810
:10F16800A0301046F2F770F8F2F770FAC4F8900081
:10F1780010BD00BF00007A4410B5038F04465A2B17
:10F1880002D0B3F5877F19D15A2902D0B1F5877F0C
:10F1980019D104F1080033F0B5FB0E4B9C4205D1A0
:10F1A80015F050FAE18EA08E15F0EEF8A06878B14F
:10F1B80004F11801BDE8104033F011B85A2902D003
:10F1C800B1F5877FE5D1A38EE28EE386A286E0E7DC
:10F1D80010BD00BF581E00242DE9F04F97B004461B
:10F1E80090F8B23002AFE3B1D0F88420B14B9A4224
:10F1F80017D1843028F04EFE94F8AF30834204D102
:10F2080000205437BD46BDE8F08FFFF7BDF8002158
:10F21800B4F8A2302046D4F8982084F8B210FFF74A
:10F2280047FEA368002B00F0BF81204628F0CDFEE2
:10F238000028E5D104F1500A504633F0C5F80028FB
:10F24800DED094F84810002900F099800023236349
:10F2580004F12803FB6294F8B430002B40F0A0803E
:10F26800FEF7E6FA78610028CAD1204628F071FE38
:10F2780004F1080B07F13802F96A5846C7F810D0AC
:10F2880033F01FFC002800F0848107F138002025A6
:10F2980033F079FD94F83A30064607F13800B5FBAB
:10F2A800F3F533F075FD814607F138004FEAC518CC
:10F2B80033F06EFDB0EBC51F00F2C98001231FFAC1
:10F2C80089F03B6280239B0000254009BB6107331E
:10F2D800013023F007037863ADEB030D7B6B9B00D4
:10F2E8000DF10808073323F00703ADEB030D02AB5C
:10F2F800BB62B4F8AC30B3F5807F14BF022301239E
:10F30800BB60BB694344FB6007F1380033F03BFD49
:10F31800B4F87A307862B3F5807F05D007F1380207
:10F328005946504633F05EF8B4F8AA3087F83330BF
:10F338001DB1B4F8AC3087F83330504617F020FFD1
:10F34800002800F02681012394F8B62000210093BC
:10F3580007F13303206DD4F860C0E047504633F01E
:10F368003EF800239946FB61BB8B3A6A9A4200F249
:10F37800A3806B1CBA6801259A42C5D809E1A06828
:10F38800002800F0118117F023FEF862002800F031
:10F398000B81B4F87A30B3F5807F7FF45CAF55E722
:10F3A80004F10806204628F0D4FDC7F828D03046D6
:10F3B80033F04CFB05463046C5F34F0533F048FBA8
:10F3C80077218046EB1D2A4623F00703ADEB030D9A
:10F3D8000DF10809484639F08BFEB4F8AA305046BA
:10F3E80087F8443017F0CCFE834688B12046D7F81A
:10F3F80028D028F0CDFD94F8B230002B3FF430AF80
:10F40800FEF716FA00287FF42BAFFEF7CFFAF2E7E3
:10F41800012394F8B6200146009307F14403266EB1
:10F42800206DB047504632F0DAFF1FFA8BF398454B
:10F43800DCD950460BF1010B17F0A2FE0028D5D0FD
:10F4480094F8B6204B4600950121266EE8E707F1AF
:10F45800380033F093FCB8FBF0F0002808BF012017
:10F4680086B207F1380033F08EFCB0FBF6F083B2B9
:10F4780007F138003B6233F086FCB0FBF6F303FB80
:10F48800160080B218B13B6A01339BB23B6207F1A8
:10F49800380033F073FC16FB00F080B2B0FBF5F2D5
:10F4A80093B205FB1202002A3FF40DAF01339BB261
:10F4B80009E700BF741805907B697A8F786AFB6446
:10F4C8003B8F8642B7F93C1007F14400A7F8443057
:10F4D80002EB090394BF92197A6A9BB2A7F8481005
:10F4E80098BF4A44A7F846308ABF9B1813B21BB28C
:10F4F800A7F84A307B6A9B1B9BB27B6233F048FCBF
:10F5080094F83A3008220021B2FBF3F3B0FBF3F38E
:10F518007A6BB86A92007B6039F0EAFDBA6900211B
:10F52800404639F0E5FD94F8B43013B940F20713BA
:10F53800E387D5B194F8B33063B1062384F83E303D
:10F548004346BA6A07F14401584633F0ADFA94F8D5
:10F55800B13013E094F8402012B184F83F30EFE75F
:10F56800B4F84230002BF2D0EAE74346BA6A07F112
:10F578004401584633F098FA94F8B030B3B950467D
:10F58800B14417F0FDFDFB691FFA89F90133FB61EE
:10F59800A8B9FB6AD7F810D09B68FB62002B7FF4F0
:10F5A80067AE204628F0F4FC01202AE64346FA68B4
:10F5B8009342E4D01A68D24343F8042BF7E7BB8898
:10F5C800012194F8B62000934346206DD4F860C01A
:10F5D800E047504632F003FFFEF7E8F9C4E600BF03
:10F5E80010B590F8B23004463BB3D0F88420134BE2
:10F5F8009A4214D1843028F04DFC94F8AF308342FD
:10F608001BD0FEF7C1FE0021B4F8A2302046D4F882
:10F61800982084F8B210BDE81040FFF749BC28F0E4
:10F6280044FAD4E90432C01AB4F8A83061EB0201F4
:10F6380083424FF000038B41E3D310BD741805904B
:10F6480010B590F8B230044693B1D0F88420104B2E
:10F658009A4201D028F06BFCFEF796FE0021B4F820
:10F66800A2302046D4F8982084F8B210FFF720FC86
:10F6780004F1080033F00CFAD4F88420054B9A42C0
:10F6880005D104F18400BDE8104028F0F8BB10BD96
:10F6980088F604907418059010B50449044608309B
:10F6A80033F0A6F9012384F8483010BDD4050024AE
:10F6B80010B50B4C0B4B22689A420ED1A2680A4B2C
:10F6C8009A420AD1204628F080FC28B92046FFF744
:10F6D80083FD80F00100C0B210BD0020FCE700BF30
:10F6E800581E002490C10490D4050024014808B590
:10F6F80002F048FEB9B3059010B504492BF0CEFED0
:10F7080004460BF041F8204610BD00BF90C104909C
:10F71800F0B50C4689B00646174654F8040BFFF7B7
:10F72800EBFF03AB05463A46019321460A4B701E90
:10F738000093022304F05CFD05A9052203980AF052
:10F7480009F9049809F00CFF05A902462846FFF7B5
:10F75800FFFC0E2009B0F0BD80C1049008B5FFF78A
:10F76800CBFFFFF739FD10B9024802F013FE0E2057
:10F7780008BD00BF4DAE059010B5FFF7BDFF28F0DE
:10F7880024FCA0B16430F1F7C5F800220A4BF1F768
:10F7980065FAF1F7FBFB01460446F1F71BFF40B998
:10F7A80024F0030040F00200A0F1FF4010BD034820
:10F7B800FCE70348FAE700BF00408F400200808062
:10F7C800020040002DE9F04FCBB0084611461A461A
:10F7D8002AAB01936A4B009320232AF0ACFC2A9BA6
:10F7E80005220AA92B9803930AF0B4F805220DA95B
:10F7F8002C980AF0AFF840F25631409829F0EFF80B
:10F80800339F5A22049097FBF2F302FB137313B150
:10F818005C4802F0A1FDFFF7C7FA05463F9809F0DA
:10F828009FFE8346429809F09BFE8246489809F05D
:10F8380097FE3C9B80463A9805930E283D9B06937D
:10F8480000F08C802BF0E5FC06463E9C09A99DF84B
:10F858001C91204609F006FE002800F08280032053
:10F868002CF033FA099B044603700023437083701D
:10F8780009F10203444A00210DF1560007932A605A
:10F88800522239F035FC0A9A039B2846149213A990
:10F898000B9A1393ADF854200D9ACDF8588017920F
:10F8A8000E9AADF86E70ADF860202D9AADF8622012
:10F8B8002E9AADF864202F9AADF86620309AADF8EC
:10F8C8006820319AADF86A20329AADF86C20349AE3
:10F8D800ADF87020359AADF87220369AADF87420DC
:10F8E800379AADF87620389A059BADF878202093A2
:10F8F800069B9DF8E420ADF87C608DF87A209DF891
:10F90800EC20CDF890B08DF87E20CDF89CA08DF835
:10F91800A490CDE92134079BADF88C30049B259346
:10F928009DF804318DF898309DF80C318DF8A03091
:10F938009DF810318DF8A1309DF814318DF8A23062
:10F948009DF818318DF8A3309DF824318DF8A53035
:10F95800FFF71EFB28464BB0BDE8F08F4FF48076CA
:10F9680073E7012210A9204609F0F4FF10B1DDE980
:10F9780010437FE740F29C41044802F033FD00BF8A
:10F9880080C00490DEB1059090C1049088B00590C5
:10F9980070B58AB00C460138043104AB01931A4B98
:10F9A8000093032304F024FCFF22002140F2723369
:10F9B800049804F0B9FC05228DF80F0007A90598F2
:10F9C800246809F0C7FF204628F049FCC0B19DF81B
:10F9D800186001250DF10F032046324600210095DD
:10F9E80028F05DFC089B3246294620460093079B79
:10F9F80028F055FC204628F0D3FC0E200AB070BD34
:10FA0800FDF7D4FFDFE700BF18C3049070B58CB0D2
:10FA1800084611461A4605AB0193184B0093072375
:10FA28002AF089FB4FF49E621549059804F0E0FC22
:10FA38000646FFF7DBF9134B044601220360002159
:10FA480040F27D430A9804F06FFC40F27243054689
:10FA5800012200210B9804F067FC099BC0B23146D3
:10FA68000193EDB2089B0390204600930295DDE9CF
:10FA7800062328F080FB20460CB070BDE0C204903D
:10FA8800D015059030C3049008B528F058FB20B96C
:10FA98004FF49561024802F085FC0E2008BD00BFB6
:10FAA800BBAF0590436DDB6B0BB1006D1847014888
:10FAB800704700BF000080BF10B5038F04465A2B63
:10FAC80002D0B3F5877F19D15A2902D0B1F5877FC3
:10FAD80019D104F1080032F015FF0E4B9C4205D1F4
:10FAE80014F0B0FDE18EA08E14F04EFCA06878B141
:10FAF80004F11801BDE8104032F071BB5A2902D058
:10FB0800B1F5877FE5D1A38EE28EE386A286E0E792
:10FB180010BD00BF581E0024F8B590F87830044690
:10FB28000D46174643B100230126204684F8793054
:10FB380028F046FC3046F8BD90F87960002EF2D1E6
:10FB48004B1CF0D027F0B1FF2369C31ABB4202D97E
:10FB58000D4802F01FFCA26E821A9542C4E91A01F0
:10FB6800E8D3B3FBF5F205FB1233ED1A27F09DFF3E
:10FB7800D4E91A32C01A61EB0201A84271F10001FE
:10FB8800D1D2FDF713FFF1E742B305902DE9F04F0D
:10FB98001F4600230446016580F878308BB040F298
:10FBA8008540904602F0C8F86065C369002B00F0F4
:10FBB8009180206D984786B2636D04F1080B206D23
:10FBC8001B69984783B2206D0793636D5B699847FB
:10FBD80083B20893636D5B6A002B7DD0206D9847D4
:10FBE8008146636DDD6A15B1206DA8470546636DD2
:10FBF8009B69002B77D0206D98475FFA80FA636D78
:10FC08001B6B13B1206D98470346626D526B22B18E
:10FC1800206D09939047099B02465846CDE9043266
:10FC2800CDE9025A0023DDE90712CDE9006932F077
:10FC3800AAFE636D1B6A13B1206D984783B2A4F8BE
:10FC48007430636D206D9B6B002B4FD1A38E94F89D
:10FC58003A205343DB10A4F87630636D04F1580161
:10FC6800206D5B689847E28EB4F87610013AB4F8D4
:10FC78007430E06D01FB023394F83A20A18E5143B1
:10FC880040F2DD3203EBD10104F08AFB87F0010377
:10FC980084F87930636D9B6A7BB3206D984780B296
:10FCA8004FF47A73A4F87000B3FBF0F3A4F8723041
:10FCB800B8F1000F03D041462046FFF7FDFE10497A
:10FCC800584632F095FE394620460BB0BDE8F04F55
:10FCD80028F019BD10266FE7072E8CBF4FF00009DA
:10FCE8004FF001097DE74FF0020A88E7984780B294
:10FCF800A4F876000028B0D1A8E73C20D0E700BFE0
:10FD0800D405002410B50446002128F0FCFC04F1B9
:10FD1800080032F0BDFE636D206DDB689847014B2B
:10FD2800236010BD88F6049010B50446006D09F0F4
:10FD380067FA78B10A4B98420CD00121204628F086
:10FD4800E2FC084904F1080032F052FE012384F86D
:10FD5800483010BD2046BDE81040FFF7D3BF00BFB4
:10FD680088F60490D405002408B5083032F040FE27
:10FD780010B9024802F0F0FA0E2008BD2AB1059029
:10FD8800014808B502F0FEFAB9B3059010B5044968
:10FD98002BF084FB04460AF0F7FC204610BD00BF98
:10FDA800B8C3049030B585B00C460138043102ABB5
:10FDB8000193144B0093022304F01AFA2068FFF70A
:10FDC800E5FF039B05460298002BCABF4FF47A74DF
:10FDD8004FF0FF3494FBF3F40E280FD02BF019FAF0
:10FDE8004FF47A7191FBF0F122462846FFF794FE12
:10FDF80000280CBF1E203E2005B030BD4FF0FF315B
:10FE0800F2E700BFA8C3049010B5FFF7BFFFFFF7E4
:10FE180049FE00210446F1F7B5FB10B1084802F08D
:10FE2800B9FA21462046F1F7D5FB30B924F0030092
:10FE380040F00200A0F1FF4010BD0248FCE700BFFF
:10FE48000DB30590020040002DE9F0418CB00C463E
:10FE58000138043102AF07F1080301932B4B0093DB
:10FE6800022304F0C5F92068FFF790FF0622054633
:10FE780007F11001D7E90286304609F06BFDBB692E
:10FE8800012B02D0224802F067FA95F83A30102B7D
:10FE980001D02048F7E70023AC8E07F11C00FB6176
:10FEA800A7F81E8008F101087B623C846408A7F863
:10FEB800228032F06DFFC30782B248BF0134D7E910
:10FEC8000431B1EB840F1FD35209002101328C4653
:10FED8007A607A689200073222F00702ADEB020DD1
:10FEE80002AA88B27C68013184420AD807F11C0151
:10FEF80005F1080032F0D8FD30462837BD46BDE888
:10FF0800F08142F820C0ECE70348BCE798C30490AE
:10FF180002B30590F1B10590EAB2059038B50C46E8
:10FF2800FFF734FF05460E2C0AD0204618F0C0F91A
:10FF380001462846FFF718FF20B9034802F00CFADB
:10FF48000021F6E70E2038BD2AB1059070B586B0BD
:10FF5800084611461A4603AB01930F4B009303233F
:10FF68002AF0E9F85A22DDE9036595FBF2F302FB72
:10FF7800135313B1094802F0EFF9FEF715FF084BC8
:10FF88000446AAB2036031469DF81430FFF7FEFD1F
:10FF9800204606B070BD00BF80C30490DEB1059056
:10FFA800B8C3049038B50C46FFF7F0FE0546204666
:10FFB80009F0D6FA00210446F1F7E4FA28B94FF01F
:10FFC8007E512046F1F7FCFA30B10123002240F2BD
:10FFD8004E31064802F006FA2146284628F082FBF0
:10FFE80010B9034802F0D6F90E2038BD1CB50590AB
:08FFF8000DB3059010B504469D
:02000004900169
:10000000406804F10803984201D131F0F9FE002361
:10001000A26A6360044B9A4205D104F12800BDE84E
:10002000104027F030BF10BD741805900A4B10B572
:10003000826A9A420ED000F1280400212046FEF781
:1000400005FD042028F07FFC20460121FEF7FEFC80
:10005000012010BD0020FCE788F604902DE9F04156
:1000600004460E4615461F467BB9154B8362E9B21E
:10007000304631F0C7FEE0B9114B20462360FFF750
:10008000BDFF29460F4802F0B1F90F4B80463946B3
:1000900048F8283F4046FEF7BDFC002201214046BB
:1000A00027F019FF384627F085FB2046FFF7BEFFF3
:1000B000DDE73046666031F03BFFA586BDE8F081A4
:1000C00088F60490B5AC05907418059070B586B0AC
:1000D000084611461A4603AB0193104B00930323C5
:1000E0002AF02DF84FF49561059828F07CFC40F239
:1000F000034206460A49039804F07EF90546FEF7D6
:1001000079FE084B0446294603603346BDF81020AB
:10011000FFF7A4FF204606B070BD00BF1CC50490C9
:100120004C17059034C5049008B5FFF77FFF20B940
:100130004FF49561024802F039F90E2008BD00BF66
:10014000BBAF059010B50A4C23686BB927F0A5F832
:1001500008B9FBF765FCEFF31182102383F31288D3
:10016000BFF36F8F034B1A6023680133236010BD08
:10017000E4220024E822002408B50C4B1A6812B9C6
:100180000520FDF7FDFC1A68013A1A601B6863B987
:10019000074B1B6883F31188BFF36F8F27F07DF83F
:1001A00018B9BDE80840FBF74FBC08BDE4220024A5
:1001B000E822002408B527F004FB01460248BDE808
:1001C00008402DF0B8BA00BF4CC60490F7B5184CE3
:1001D000A568E66801950025ECB2019FA74215D8F5
:1001E000144CA568E66801950025ECB2019FA74272
:1001F0001CD906EBC40C0135DCF80470B842F4D10C
:1002000040F24240086040F274410AE006EBC40C40
:100210000135DCF804708742DED10020086040F22E
:100220004931116056F8342012091A6003B0F0BD4C
:100230001CA3049044A4049010B540F2C22386B0DD
:100240000446084604AA0393059303A905ABFFF7E8
:10025000BDFF039A059B3AB100932046049B0649D3
:1002600029F0ACFC06B010BD049A2046034906B044
:10027000BDE8104029F0A2BC696605906C66059047
:100280000A46014904F0B8B8F8C604901FB5044600
:1002900088B10E280FD027F090FA60B940F2C2233F
:1002A00001A9204602AA039303ABFFF78FFF03992E
:1002B000024802F09BF804B010BD00BF4EB5059097
:1002C0000E2373B50B600D4601A900F0F5FC012863
:1002D00004460FD9019E3046F1F758FA0246012A2A
:1002E00003D9531EF15C2F2907D03146044806F08C
:1002F000B9FB2860204602B070BD1A46EFE700BF88
:100300001CCA04900E2373B50B600D4601A900F0C2
:10031000D3FC0128044609D9019E3046F1F736FA8C
:1003200031460246034806F09DFB2860204602B095
:1003300070BD00BF1CCA0490F8B5037800AF064634
:100340002F2B6BD0524CD4F8B45045B902202BF06F
:10035000C0FC05464F49F1F711FAC4F8B4502846DD
:10036000F1F714FA04463046F1F710FA204402304F
:100370002BF0AFFC04462846F1F708FA294602465E
:10038000204638F091FE2846F1F700FA054638B1CC
:10039000231813F8013C2F2B1EBF2F2301352354A4
:1003A0003046F1F7F3F93146421C601938F07CFE13
:1003B0002046F1F7EBF900222146134615469042FC
:1003C0002ED145B39B002046651E073323F007035B
:1003D000ADEB030DF1F7DAF900236E4620441A461F
:1003E000194615F801EF02F1010CBEF12F0F04F8C8
:1003F00002E002D0BEF1000F46D1012B30D115F83A
:10040000013C2E2B3BD14B1E56F823200023854266
:10041000E7D10023A3542046BD46F8BD1E4D9EE7FC
:1004200011F801CB561CBCF12F0F15D102F1020CB3
:100430000133604510D991F800C0BCF12E0F0BD1EB
:1004400091F801C0BCF12E0F06D10332904205D0C5
:100450008A782F2A08BF01253246B0E70125FBE73D
:10046000022B0CD115F8013C2E2B08D115F8023CBB
:100470002E2B04D18B1E013956F82320C6E746F8EF
:1004800021C062460131C1E701336246BFE700BFC8
:10049000F4220024634D05907C62059037B5134C1F
:1004A000FFF74AFF6946C4F8B400FFF709FFC4F834
:1004B000EC00B0B9D4F8F0400CB903B030BD6568B9
:1004C000012D0CD129460A4806F0A6FA01AB01908D
:1004D0002A464FF45871204628F091FAEDE7E46877
:1004E000EAE76B4601224FF45871F5E7F422002445
:1004F000634D0590084B10B5D3F8B4404CB120467D
:10050000F1F744F9214602460448BDE8104006F0E0
:10051000A9BA662010BD00BFF42200241CCA0490B2
:1005200037B5FFF709FF01A9FFF7CAFE28B9144B39
:10053000D3F8F000A0B96623019301AB012240F289
:10054000064128F05CFA0021054608462DF0BCF86B
:100550000446284602F024FB38B9204603B030BDDB
:100560004368012BE7D0C068E4E70422012109F0C9
:10057000B9F9014620462CF095FFFDF71BFAE8E794
:10058000F422002413B5FFF7D7FE01A9FFF798FE68
:10059000044610B9112002F083FE012807D001980B
:1005A00006F076FF0649F1F7DFF80028F2D001AB3C
:1005B00001224FF48961204628F021FA02B010BDD3
:1005C000634D059007B5FFF7B7FE01A9FFF79AFE47
:1005D000D8B9114BD3F8F00080B901460A2005F0D4
:1005E00013FB0122031D00F1280143F8042F8B4265
:1005F000FBD1C123C36203B05DF804FB4368012B48
:1006000001D0C068E8E76623019301AB012240F204
:10061000FA4128F0F4F9EEE7F422002410B50D4B6E
:10062000044602689A4214D1406804F108039842D3
:1006300001D131F0A4FAA06F27F0BDF8D4F8800002
:1006400010F01EFD204698220021BDE8104038F031
:1006500053BD10BD84C7049070B58AB008461146DA
:100660001A4604AB0193124B0093062329F067FD51
:1006700040F26131059828F0AEF94FF49E610646CC
:10068000049815F0E9FD0546FEF7B4FB094B044656
:100690003246036029469DF824300293079B01935C
:1006A000069B0093089B28F037FB20460AB070BDDC
:1006B00054C7049084C7049038B5437904460D4666
:1006C0008B4209D0837913B1044828F06EFC657120
:1006D000BDE83840FEF710B838BD00BFE003002485
:1006E00038B50C460F4D11461A460F4B9D4201D1AD
:1006F00024F0F9F80D4B9D42FAD00D4B9D42F7D0F6
:100700000C4B9D42F4D0A3070AD12368AB4207D11A
:1007100032F035F801462046BDE8384033F0A7BC3A
:1007200038BD00BF6027059068E60490480005903A
:100730001CCA049088F60490F7B514460AB1002349
:1007400013701C4BDFF870E0734501D124F0CBF837
:100750001A4FBB42FAD01A4EB342F7D0194DAB42F2
:10076000F4D010F0030210D1D0F800C09C450CD199
:100770008DF807200DF1070233F060FA14B19DF8EF
:100780000730237080B203B0F0BD0F4B7345DDD04E
:10079000BB42DBD0B342D9D0AB42D7D012B14FF677
:1007A000FF70F0E702689A42F9D133F09FF8FF2812
:1007B000E9D1F4E76027059068E6049048000590C9
:1007C0001CCA049088F60490C421059013B5002338
:1007D0000D4C0DF107008DF807302EF020F9A0FB2D
:1007E0000432400840EAC17004FB012218189DF849
:1007F000073042EB510147F236725343C01841F1C2
:10080000000102B010BD00BFB2E60E00014808B5FD
:1008100001F0BCFDB9B3059010B504492AF042FEC1
:10082000044609F0B5FF204610BD00BFC0C80490C3
:1008300030B585B00C460138043102AB0193144B3E
:100840000093022303F0D8FC2068FFF7E5FF039B29
:1008500005460298002BCABF4FF47A744FF0FF345C
:1008600094FBF3F40E280FD02AF0D7FC4FF47A71E2
:1008700091FBF0F12246284600F0A0F800280CBFBA
:100880001E203E2005B030BD4FF0FF31F2E700BF23
:10089000B0C8049010B5FFF7BFFF00F05BF800216F
:1008A0000446F0F773FE10B1084801F077FD2146C9
:1008B0002046F0F793FE30B924F0030040F0020028
:1008C000A0F1FF4010BD0248FCE700BF0DB305904A
:1008D0000200400038B50C46FFF79EFF05460E2C7F
:1008E0000AD0204617F0E8FC0146284628F024FFED
:1008F00020B9034801F034FD0021F6E70E2038BD91
:100900002AB1059038B50C46FFF786FF054620460C
:1009100008F02AFE00210446F0F738FE28B94FF00F
:100920007E512046F0F750FE30B10123002240F204
:100930004E31064801F05AFD2146284628F0C0FEF7
:1009400010B9034801F02AFD0E2038BD1CB50590F2
:100950000DB3059000487047000080BF10B5038FAD
:1009600004465A2B02D0B3F5877F19D15A2902D0F9
:10097000B1F5877F19D104F1080031F0C7FF0E4BA4
:100980009C4205D113F062FEE18EA08E13F000FDB3
:10099000A06878B104F11801BDE8104031F023BC23
:1009A0005A2902D0B1F5877FE5D1A38EE28EE38686
:1009B000A286E0E710BD00BF581E0024F8B590F8ED
:1009C000743004460D46174643B1002301262046E5
:1009D00084F8753028F0EAFC3046F8BD90F8756070
:1009E000002EF2D14B1CF0D027F063F82369C31A14
:1009F000BB4202D90D4801F0D1FCA26E821A954289
:100A0000C4E91A01E8D3B3FBF5F205FB1233ED1A82
:100A100027F04FF8D4E91A32C01A61EB0201A8425C
:100A200071F10001D1D2FCF7C5FFF1E742B30590A7
:100A30002DE9F0411E46002386B0054617460C46B8
:100A400080F87430002943D16FF0120012F06EFA72
:100A50002C6505F15408A368204641461B6A984757
:100A6000AB6DD8063AD4D9073AD41A073AD49C06C3
:100A70003AD458063AD419063AD49A073AD45B07BE
:100A80003AD495F8601095F8603085F864108B4280
:100A90000DD0286D83685B6A03B19847286D414685
:100AA00083681B6A984795F8603085F8643095F83C
:100AB0006440202C6DD0082C56D8002C51D0013C1D
:100AC000072C4DD8DFE804F06D5A4C5A4C4C4C1AA8
:100AD000084626F088F90028B6D0B9E71021D2E7F9
:100AE0000121D0E70821CEE72021CCE74021CAE749
:100AF0008021C8E70221C6E70421C4E700244FF0A3
:100B0000040C202122462046234605F10808CDE9A1
:100B1000020CCDE90013CDE904240023B5F85620DA
:100B2000B5F85410404631F032FF254B2B6786F064
:100B3000010385F875301FB139462846FFF70EFFCF
:100B4000286D83685B6803B198471E49404631F0C1
:100B500053FF3146284606B0BDE8F04128F0B7BD46
:100B600000242246204607E0402C22D0802C4FF063
:100B70000004224620461FD023460EE0E86D0123E4
:100B80000024C0F34002C0439C46194600F0010017
:100B9000BBE700220124104613464FF0020C10213F
:100BA000B3E700244FF0030C1821224620462346C9
:100BB000ABE7002422462046012308219C46A4E7F7
:100BC0003C001000D405002410B50446002128F094
:100BD0007EFD04F1080031F05FFF00232365014B27
:100BE000236010BD88F6049010B50446006D78B1FE
:100BF00026F0F9F860B10121204628F068FD074988
:100C000004F1080031F0F8FE012384F8483010BDEB
:100C10002046BDE81040FFF7D7BF00BFD405002431
:100C2000224B0340062B2DE9F743064606D010F071
:100C3000030513D102681E4B9A4204D101A9304624
:100C400006F08CFC0546DFF86C80DDF80490474622
:100C500057F8F04F24B9162002F022FB0025F2E7E6
:100C600045B163684B4505D14A462168284638F0AE
:100C70004BFA18B1D4E90223B24213D1E3683B60C6
:100C8000D8F8EC309C4202D10023C8F8EC300023A5
:100C900040F2325120461A4628F051FD0E2003B092
:100CA000BDE8F08304F10C071C46D3E70F0080FF7A
:100CB0001CCA0490F42200242DE9F0410378064672
:100CC00088462F2B0DD01A4BD3F8EC7057BB3478D5
:100CD00084B127F036FF164BD3F8F04024B9012435
:100CE00008E001360127F2E76568013D05D1F71BF1
:100CF000C8F800702046BDE8F08121682A463046D9
:100D0000013138F01EFA58B9735D72192F2B02D1D8
:100D1000C8F80020EEE71BB9064BC8F80030E9E739
:100D2000E468DBE7C8F80000D3F8EC40E2E700BF76
:100D3000F4220024634D059010B586B0084B02AC38
:100D400000930423019403F057FA2146029828F0F7
:100D500013FD23460222762128F0F1FC06B010BDD7
:100D6000F0C9049038B543680546194403689942B0
:100D700010D9037B1BB10021074829F098F801F135
:100D80001004806824F00704083421462AF0A7FFE5
:100D90002C60A86038BD00BF1CED049038B5144627
:100DA000054628F06CFD024B2560636038BD00BF2E
:100DB0002D98039038B5037B04460D461BB10021E6
:100DC000064829F074F80168806829442AF087FFF2
:100DD0002368A0601D441844256038BD1CED0490B4
:100DE000044B0B60044BC1E9013000230846CB6083
:100DF000704700BFA0F30490479A03902DE9F04F8D
:100E000087B016460446084605A905F05FFE032E86
:100E10000546059A06D10146204605F097FD07B024
:100E2000BDE8F08F26B90146636820689847F6E769
:100E30008718B84207D20346002213F8011B27295E
:100E400015D0222914D12726DFF8D4903246DFF8B6
:100E5000D4A02046DFF8D0B0324928F0AFFEAF4230
:100E60000DD832462F49204628F0A8FED7E70122A8
:100E70009F42E2D1002A0CBF27262226E4E728461B
:100E80002CF0BFF8039028462CF0D6F8039A804641
:100E9000964206D132462549204628F08FFE454627
:100EA000DDE75C2A04D15946204628F004FEF6E727
:100EB000A2F120035E2B01D85146EDE70A2A01D1A9
:100EC0001B49F1E70D2A01D11A49EDE7092A01D1A1
:100ED0001949E9E71F2A05D9A2F17F03212B01D97E
:100EE000AD2A01D14946D7E7A2F500530F2B06D909
:100EF000283B012B03D94FF6FF739A4201D10F49CA
:100F0000CAE70F4B9A4201D10E49C5E7421B202385
:100F10002946204600930023019200F0F1F8BEE735
:100F200082660590736605907666059072660590F8
:100F3000796605907C6605907F66059089660590C8
:100F4000FFFF010090660590F7B51E462B4B0D463E
:100F5000144698429DF8207002D0294B984208D13F
:100F60003B463246214608F0BFFB0544284603B005
:100F7000F0BDF3070BD57610019601992A190029C7
:100F800027DA013A00201346B1B9551CEEE701A952
:100F9000304608F06BFA0028EFD130462AF032F9DB
:100FA00018490246184828F090FF1B78013A03F0D0
:100FB000C003802B0AD11346AA42F6D200B1019198
:100FC000002FD3D11149124828F071FF01310120BF
:100FD000D9E70024954205D304B10191002FF1D047
:100FE0001546C3E70139C1D3681C01240546013009
:100FF0002B7803F0C003802BF8D0EBE734F3049098
:1010000014F904906BA305908CEC049079A30590DF
:101010003CEE04907FB505460C46164608F0F4F801
:10102000314B834201D023F05EFC284603A905F032
:101030004DFD042E054652D12C4B2D4A9342F2D041
:101040002C4A9342EFD02C4A9342ECD0A2072DD1E8
:1010500022689A422AD1E2680E2AD4E9013604D0E5
:10106000032A02D0254802F0CFF80E2B1AD0012215
:1010700029461D480092039AFFF766FF04460E2E8C
:10108000039A11D001232946174800933346FFF7EE
:101090005BFF844225D8021B2146134805F0E2FC81
:1010A00004B070BD2C46EAE7A818F2E70023039AC3
:1010B00029460D4800932346FFF746FF90F900307C
:1010C0000278002B08DB012129F022FDE8E701313D
:1010D0005B081A42FBD1F7E740230121F9E7002022
:1010E000DEE71620DCE700BF1CCA0490D0EB0490BA
:1010F00068E604904800059088F604908AA405905C
:101100002DE9F74F8A469DF8301091460D9A11F05F
:10111000DF0F8046A2EB090546D0302947D1C3F343
:101120004721002946D05F29364E14BF04270527E2
:10113000A6F1050092FBF7F107FB112108BF064657
:1011400009B901350132791E92FBF7F007FB102235
:101150008A1A164413F020022ED005EBD574012D07
:101160004FEA6403A5EB640433DC0025B9F1000FFA
:1011700007D04D44D8F804304A465146D8F800000C
:101180009847002C21DD2544A742B946D8F8043001
:101190003146A8BFA146D8F80000A4EB09044A468E
:1011A0009847002CF0DC10E0174E1027D2E70CAE69
:1011B0000127CFE7154EF8E713F001041DD1002DEC
:1011C00008DCB9F1000F1BD14D46284603B0BDE83D
:1011D000F08F1D46AB465F453A46D8F8043031469D
:1011E000A8BF5A46D8F8000001929847019AABEB85
:1011F000020BBBF1000FEEDCB8E72C461546B5E755
:101200002546B6E7B2660590B8660590A1660590DA
:101210002DE9F04F102A93B081460C4690461C9D54
:101220009DF874A00593DDE91E6703D8854BD34074
:10123000D90701D423F057FBE2070BD4A30703D14E
:101240002168814B994205D0204629F0E6FF4400F1
:1012500044F0010415F0210306D1BAF1300F03D197
:10126000BE42B8BF3E461F4620460DF1280B29F06E
:10127000F1FD00281CDBA80718D52B238DF828309A
:101280000DF129032A079DF814101FD5B8F1020F9C
:1012900010D14FF0300C184600F802CB01F1010CD0
:1012A00083F801C0034611E02023E7E76907FBD478
:1012B0005B46E7E7B8F1080F3AD1302018702806EE
:1012C00049BF01F10E0001335870023300200EAA0D
:1012D000012F1870A3EB0B030B924FF01002059334
:1012E000C5F34723C8BF15438DF82700CDE90C206F
:1012F00015F01002CDE90213079232D023460DAA51
:101300000CA9CDE900800BA80FF076F80378804691
:101310002D2B18D0012F40F391800D9C9DF8273084
:10132000BC42B8BF3C4603B10134059B1C4428E0D5
:10133000B8F1100FCAD14FF0300C184600F802CBAC
:1013400001F1170CACE70D9C012F00F101088DF89D
:10135000273004F1FF340D9470DDBC42B8BF3C4629
:10136000E2E70AAB0DAA0CA90BA8CDE9008323463E
:101370000FF042F8012F80465CDD0D9CBC42B8BFE7
:101380003C4625F00103A642069350DD15F0010A04
:10139000A6EB04044CD12023019452462B49009320
:1013A000484653465446FFF7ABFE0546079B4FF0B1
:1013B000300ADBB19DF8273053B1002301220DF133
:1013C00027014846013ECDE90032FFF799FE05446A
:1013D000059B5BB10023012259464846CDE9003206
:1013E000059AFFF78DFE059B0544F61A012FC8BF2D
:1013F0003E46069B41460D9A4846CDE900A6FFF7BA
:101400007FFE05444CB120231049484601940093C7
:1014100000231A46FFF774FE05440B980EAB984262
:1014200001D02AF069FC284613B0BDE8F08F0024F3
:101430000025BBE7079C06952546DAE700240695BC
:101440002546B7E704050100480005907C62059039
:101450002DE9F04F91B080469246002404AF0B4630
:101460001D4613F8012B0AB1252AF9D1A94208D249
:101470006E1AD8F80430D8F8000032463444984741
:1014800029460B78002B00F0FD81202301317B6180
:1014900000230A4612F8015B3DB12D2D28D021D83A
:1014A000202D2CD02B2D27D00025396111F8012BB0
:1014B000A2F13000092825D92E2A5DD13A69527847
:1014C0002A2A25D0396900220131396111F8010B2E
:1014D000A0F13006092E20D80A2606FB020BABF13C
:1014E0003002F2E7302DDFD143F010037D6101E0DF
:1014F00043F001031146CCE743F00203FAE743F05F
:101500000403F7E70A2000FB0522A2F13005CCE72F
:101510003A6902323A615AF8042B22EAE27B3A69CC
:1015200012786C2A02BF3A6901323A613A6992F83C
:101530000090B9F1000F00F0A581B9F1670F65D8EF
:10154000B9F14F0F29D8A9F14502022A00F28C8186
:101550000AF1070AFB602AF00706F6E80201EFF736
:1015600019FD4A4601464046CDE9015B7B6900937F
:10157000FB6828F0AFFA5CE04FF0FF3BCFE7082AAA
:1015800000F27281DFE812F0C5006B00700182008A
:101590007001C50070017001C500A9F15002172A41
:1015A00000F2628101A151F822F000BFDB16019028
:1015B0006918019069180190191801906918019033
:1015C000691801906918019069180190DB16019063
:1015D00069180190691801906918019069180190C3
:1015E00069180190691801906918019069180190B3
:1015F000691801901B16019047160190DB160190A7
:10160000511501905115019051150190A9F17002E9
:10161000D1B20829B3D923F066F9564656F8042BFF
:1016200001955AB17A699A49009204224046FFF71F
:1016300067FD04443969B246013110E77A6995497A
:1016400000920522F2E7564607F1200156F8042BD6
:1016500087F8202001957A6900920122E6E7564634
:1016600007F12001FB6056F8040B28F0BCFDBBF12C
:10167000FF3F0146FB6804D03A6A934538BFC7F87C
:1016800020B001957A6900923A6ACFE7564656F83B
:10169000049BBBF1000F08D0B9F1000F0FD10195E9
:1016A0007A697D4900920622C0E74846FB60F0F760
:1016B0006DF8FB6802465A4528BF5A4608E048467E
:1016C000FB60F0F763F8BBF1FF3F0246FB68F2D125
:1016D0000195796900914946A8E7B9F1500F0AF1DF
:1016E00004062BD1DAF800B04FF0410A01954046CC
:1016F0007A696A4900920222FB60FFF701FD00222D
:10170000B9F1640F0444FA774FF01002FB6823D05C
:1017100045E0B9F1700F0AF1040604D1DAF800B01F
:101720004FF0610AE2E7B9F1750FDAF800B031D095
:101730004FF0610A0022FA77102230E0DAF800B0A8
:1017400029F00F0AB9F1640FAAF10F0A5FFA8AFAB9
:10175000F0D10022FA770A22BBF1000F46DA2D21E0
:10176000CBF1000BF97707F13009AAF10A0A07F16A
:10177000200EDC46BBFBF2F002FB10B183460929C8
:101780008CBF5144303109F8011DF1450FD062453D
:10179000EFD90CE000224FF0610AFA770A22BBF180
:1017A000000FE0D1302207F12F0987F82F2013F026
:1017B000100AFA7F23D06AB301224046013D01920C
:1017C0007969009107F11F01FB60FFF799FCFB6845
:1017D0008246019549467A694046009207F13002F7
:1017E000A2EB0902FFF78CFC504422E7980702D5D0
:1017F0002B21F977D3E75907D1D52021F9E7002A22
:10180000E7D007F120018945E3D909F8012C09F156
:10181000FF39DEE79246DCE756467B60C7F80CD01E
:1018200056F8049B484626F0E8FA00F1FF3A0730E4
:1018300020F00700ADEB000D484604A9B960FDF7A4
:1018400015F8BBF1FF3FD7E9013102D0DA4528BFD7
:10185000DA46019540467A6900925246FFF750FCFD
:101860000444D7F80CD0E5E6B9F1250F7FF4D3AEE8
:10187000D8F80430012239690134D8F800005646FE
:101880009847D7E620463437BD46BDE8F08F00BF05
:101890000B63059010630590976605909E66059012
:1018A0002DE9F04F122A9BB01E46DDF890909DF86E
:1018B000944006901091079201D823F014F8069BEB
:1018C000002B2EDA0699EFF789FE50BB069B2D24DC
:1018D00003F100430693079B109D013B05F8014B64
:1018E0000793069B06F0200B9D4923F000473846DE
:1018F000EFF774FEC8B99A493846EFF751FEA0B920
:101900004BF049004BF04E01EB1C4BF04602AA7025
:101910000022287069701A70109A981A1BB0BDE8DE
:10192000F08F002CD7D1109DDBE706990846EFF722
:1019300055FE30B14BF04E024BF04101EB1C10460E
:10194000E5E746F02006662E5DD14BF0040B079BC1
:10195000B9F1000FA3F1030A5CDA53464FF0060910
:10196000062BA8BF06230C93069B002B099365D07A
:10197000C3F3C7504FF07E587F38EFF715FC794915
:10198000EFF766FCEFF740FE099B0646B3F17E5F7A
:1019900034BF0024012421184FF07E5002F08CFE49
:1019A000099BB3F17E5F2CBF01274FF0FF370699EB
:1019B000EFF7F6FD003818BF0120A04238D01BF029
:1019C000040F3CD0002E3ADD09EB0603079A0233E0
:1019D000934234DD6FEA0B028BF0040309F101043A
:1019E00012F0040243F00203089200F0A480079A68
:1019F0009B46023A94422ADA731C1C44092C48DDA7
:101A0000A4F109092DE0672E0CBF4BF0020B4BF03F
:101A1000010B9CE7B9F1630F05D0D1454B46A8BF38
:101A200053460C93A0E710234FF009090C939BE752
:101A30003E444046311902F03FFEB8E7099E1BF0D4
:101A4000040308935DD0079B023B4B450BDC002E43
:101A500053DABAF1020FD14619DDB21C0ADBA9F143
:101A60000809002711E0002E49DAB9F1020F0EDD56
:101A7000B31C3DDA77424F45A8BF4F46023FA9EB62
:101A80000704092C59DDA4F10909092404E009F12E
:101A900001044FF000094F460323079AA046121B8A
:101AA000D31A4B45A8BF4B46062CA8BF4FF00608DB
:101AB0001593A8EB0603013B0F93099B23F0030347
:101AC0001493159BE318A3EB08031293099B002BB7
:101AD00000F00181089B002B00F0F980002E80F2BD
:101AE000F380002F40D108F1FF310B970A954CE0AD
:101AF00009F10104092CCCDDB1E754467CE74C46E2
:101B00007AE71BF0020308930BD0B9F1000F17D04E
:101B10004C46092C1DDD0027A4F10909092408976A
:101B200007E009F10104092C0FDDA9F10809089F5C
:101B300009240723B1E79B46EBE74FF00009ABE729
:101B40004F460124CDF82090F3E7DDF820904F4672
:101B5000EFE74FF000094F46CDF82090E9E700BFCE
:101B6000FFFF7F7F9B209A3E2B4630212E2203F8D9
:101B7000021B18466A703A4637F0BEFA034608EB75
:101B800007013B440A93FF230B930A2201230D9282
:101B9000984500F3A580B8F1060F40F3AA8001290B
:101BA00040F3A780B8F1070F00F09F80022900F0F2
:101BB0009C8002394FF06409069802F07DFD4FF0D9
:101BC0007C51EFF73DFAEFF745FD0B9B09FB00F960
:101BD0002A460393129B48460D9902930C9BCDE92C
:101BE000046BCDE900830A9B28F01AF8079A90420B
:101BF000BFF663AE19AA01460E90284602F088FD92
:101C00001998149920F00300EFF718FA0E9B02467A
:101C1000002855D0B8F1060F4FF0010ACDF83890E2
:101C2000C8BF08EB48031190C4BF123B0AFA03FA7D
:101C30000C231393002A5FDAD1440B9B2A460D999B
:101C400048460393129B02930C9BCDE9046BCDE9AC
:101C500000830A9B27F0E4FF079A9042BFF62DAE5F
:101C600019AA01461690284602F052FD19981499B7
:101C700020F00300EFF7E2F9169B024600B317933A
:101C800020F00040119B169223F00041EFF7D6F9A7
:101C90000028DDE9162307DB4FF00A0CB9FBFCF145
:101CA0000CFB1191014302D1CDF838901192BAF199
:101CB000010F27D013994FEA5A0A01391391B9D16C
:101CC000E818109BC01A29E60F990B960EE7089B9F
:101CD0000F990B930AE7099B0A9519460B9354E752
:101CE0000D98013350430D9052E701394FF00A0926
:101CF00062E74FF001095FE7D145FFF4DEADA9EBE4
:101D00000A099AE70F9AA04502F101020F9202DA3E
:101D100008F10108D5E60E9A9145D1D00B9B2A46D1
:101D20000393129B02930C9BDDE90D10CDE9008318
:101D3000CDE9046B0A9B27F073FF0346C0E700BFA1
:101D400038B504460D4628F053F838B9284607F050
:101D50005BFA2246C188024800F05CFB38BD00BF38
:101D60009CB4059070B504460846114614F0030271
:101D700003D12568054B9D4201D022F0B4FD02F04D
:101D800013FA6368BDE87040184700BFD8CA0490D2
:101D900070B504461D4608461146A30703D12268C4
:101DA000064B9A4201D022F09EFD4FF0021202F043
:101DB000FBF963682868BDE870401847C0CA049002
:101DC00070B504461D4608461146A30703D1226894
:101DD000074B9A4201D022F086FD4FF0041202F028
:101DE000E3F96368D5E90001BDE87040184700BF1A
:101DF000A8CA049070B505461C4608461146AB07B4
:101E000003D12A68074B9A4201D022F06CFD4FF0B3
:101E1000061202F0C9F96B682068D4E90112BDE826
:101E20007040184790CA0490F0B51746820785B0F5
:101E300004460D461E4603D10268104B9A4201D05B
:101E400022F051FD42683946284602F0ADF9636838
:101E5000DB0706D4A3683146284605B0BDE8F0404C
:101E6000184706EB8502394601A828F01FFBA36836
:101E700001AA31462846984705B0F0BD78CA0490BB
:101E80002DE9F84305460E461746984602F02EFB0C
:101E9000E968002011F8012BC2F3C303C2F38004E8
:101EA00012062CD403F1010904EB44044C44A400B1
:101EB00004F1140004F010F931461E4E43463A4630
:101EC0000560A0F80C90044619F016F9F36900219A
:101ED000204623616B685B68F3610DF083F823692A
:101EE000F3610346E8B9A2681068B26894421AD355
:101EF0003269944217D83461CBB109F037FD11F83B
:101F0000012B4FEA400E02F0300C0CFA0EFC43EAB3
:101F10000C0302F0020C0CFA00FC013044EA0C0441
:101F2000BEE7022801D022F0DEFC6069DDE7BDE8F3
:101F3000F88300BFF422002470B50C46054608461D
:101F400027F067FF2346024602492846BDE8704055
:101F500027F034BEC86605902DE9F04788469146C3
:101F60009A460446002846D00768002F41D0244BEB
:101F7000244A934201D122F0B6FC234A9342FAD07C
:101F8000224A9342F7D0224A9342F4D0B907F2D1C1
:101F90003A689A42EFD17E6864687CB31D4B194A57
:101FA0009342E8D0184A9342E5D0184A9342E2D0CF
:101FB000174A9342DFD0A207DDD122689A42DAD1D4
:101FC000701C04301449800029F0EDF80546C0F873
:101FD0000C80C0E9019A2FB1B20007F1080110305E
:101FE00037F062F814B1043645F826402846BDE8BB
:101FF000F0873E46D0E707460646E2E73046E0E790
:1020000084EB049068E60490480005901CCA049094
:1020100088F6049044CE049058CA04908268024B1B
:10202000DA61C2689A617047F422002408B5054B52
:102030009A68824201D922F056FC1A698242FAD388
:10204000186108BDF42200248388024603F4C0719D
:10205000B1F5C07F0FD0190604D5C37B00EB830216
:102060001069704713F4807006D0D37B02EB8302B3
:102070001369586870470148704700BFEFB8039074
:1020800070B51B4C002528F080F81A4904F1600057
:1020900004F1A006A56204F0AFFA04F17800164935
:1020A00004F0AAFA04F190000321C4F8005101F0F1
:1020B00041FE3046012101F03DFE4FF4AB724FF47A
:1020C000BB71304628F005F829462846C4F8B050C0
:1020D000C4E906662BF0F8FA1621C4F8E8002BF0E4
:1020E000E1F9294604F1D800BDE870400CF0E4BDE8
:1020F000F422002434F0049010F0049008B5084B4A
:10210000D3F8B00008B9074808BD002243F26601C1
:10211000043003F03BF90028F5D04068F4E700BF35
:10212000F42200243CEB04900001034B0A4640F0EB
:102130000601986927F0CDBFF42200240101034B6A
:1021400041F00601986927F0D5BF00BFF4220024B2
:102150000001034B0A4640F00601D86927F0B9BFD9
:10216000F42200240101034B41F00601D86927F055
:10217000C1BF00BFF422002470B50401114E054612
:102180000022F06944F006040430214603F0FEF812
:102190000246A8B9D6F8B00030B12146043003F0A9
:1021A000F5F808B1406870BD00222146064803F0EA
:1021B000EDF8024620B92A460449054827F085FE75
:1021C0005068F0E7F4220024B8E604905AA5059080
:1021D000D0ED04900A4B10B50446D3E906039842AB
